:020000040800F2
:100000000000022069900008C9830008CD83000821
:10001000D1830008D5830008D983000800000000C0
:100020000000000000000000000000004156010830
:10003000DD83000800000000D15601083557010893
:10004000B9900008B9900008B990000889840008A8
:10005000B9900008B9900008B99000087D840008A4
:10006000B9900008C5160008B9900008B9900008BA
:10007000B9900008B9900008B9900008B99000083C
:10008000B9900008B9900008B9900008B99000082C
:10009000B9900008B9900008B99000089984000848
:1000A000B9900008B9900008B9900008B99000080C
:1000B000E1830008B9900008B9900008B9900008E1
:1000C000B9900008B9900008B9900008ED830008C5
:1000D000B9900008F9830008B99000080584000869
:1000E000B9900008B9900008B9900008B9900008CC
:1000F000B9900008B9900008B9900008B9900008BC
:10010000B99000081D840008B9900008B990000853
:1001100029840008B990000841840008B9900008BB
:10012000B9900008B9900008B99000084D84000803
:10013000B990000859840008B9900008B9900008E7
:10014000B9900008B9900008B990000865840008CB
:10015000B990000871840008B9900008B9900008AF
:10016000B9900008B9900008B9900008B99000084B
:10017000B9900008B9900008B9900008000000008C
:08018000B9900008B9900008D5
:1001900010B5054C237833B9044B13B10448AFF3C1
:1001A00000800123237010BD6006002000000000C5
:1001B000C835020808B5034B1BB103490348AFF328
:1001C000008008BD0000000064060020C835020859
:1001D00010F8012B11F8013B012A28BF9A42F7D0F1
:1001E000D01A7047034613F8012B002AFBD1181AC6
:1001F000013870470000000000000000000000000F
:1002000001F0FF01102A2BDB10F0070F08D010F8C7
:10021000013B013A8B422DD010F0070F42B3F6D1CB
:10022000F0B441EA012141EA014122F007047FF0E4
:1002300000070023F0E80256083C85EA010586EA3B
:10024000010685FA47F5A3FA87F586FA47F6A5FA77
:1002500087F68EB9EED1F0BC01F0FF0102F0070283
:1002600032B110F8013B013A83EA010313B1F8D12E
:100270000020704701387047002D06BF354603380F
:10028000073815F0010F07D1013015F4807F02BF48
:10029000013015F4C03F0130F0BC0138704700BF99
:1002A00081F0004102E000BF83F0004330B54FEA27
:1002B00041044FEA430594EA050F08BF90EA020F94
:1002C0001FBF54EA000C55EA020C7FEA645C7FEA27
:1002D000655C00F0E2804FEA5454D4EB5555B8BF4A
:1002E0006D420CDD2C4480EA020281EA030382EABB
:1002F000000083EA010180EA020281EA0303362D4D
:1003000088BF30BD11F0004F4FEA01314FF4801C1F
:100310004CEA113102D0404261EB410113F0004F31
:100320004FEA03334CEA133302D0524263EB4303E8
:1003300094EA050F00F0A780A4F10104D5F1200E86
:100340000DDB02FA0EFC22FA05F2801841F10001E1
:1003500003FA0EF2801843FA05F359410EE0A5F1B5
:1003600020050EF1200E012A03FA0EFC28BF4CF0E6
:10037000020C43FA05F3C01851EBE37101F000459C
:1003800007D54FF0000EDCF1000C7EEB00006EEBA9
:100390000101B1F5801F1BD3B1F5001F0CD3490833
:1003A0005FEA30004FEA3C0C04F101044FEA44528A
:1003B00012F5800F80F09A80BCF1004F08BF5FEA11
:1003C000500C50F1000041EB045141EA050130BDF1
:1003D0005FEA4C0C404141EB0101013C28BFB1F503
:1003E000801FE9D291F0000F04BF01460020B1FA4E
:1003F00081F308BF2033A3F10B03B3F120020CDA21
:100400000C3208DD02F1140CC2F10C0201FA0CF0FE
:1004100021FA02F10CE002F11402D8BFC2F1200C63
:1004200001FA02F120FA0CFCDCBF41EA0C01904019
:10043000E41AA2BF01EB0451294330BD6FEA040462
:100440001F3C1CDA0C340EDC04F11404C4F120024D
:1004500020FA04F001FA02F340EA030021FA04F35F
:1004600045EA030130BDC4F10C04C4F1200220FAB6
:1004700002F001FA04F340EA0300294630BD21FAF4
:1004800004F0294630BD94F0000F83F4801306BFBA
:1004900081F480110134013D4EE77FEA645C18BFAE
:1004A0007FEA655C29D094EA050F08BF90EA020F45
:1004B00005D054EA000C04BF1946104630BD91EA3D
:1004C000030F1EBF0021002030BD5FEA545C05D140
:1004D0004000494128BF41F0004130BD14F580047F
:1004E0003CBF01F5801130BD01F0004545F0FE41F3
:1004F00041F470014FF0000030BD7FEA645C1ABF28
:10050000194610467FEA655C1CBF0B46024650EA5E
:10051000013406BF52EA033591EA030F41F400218A
:1005200030BD00BF90F0000F04BF0021704730B510
:100530004FF4806404F132044FF000054FF00001E5
:1005400050E700BF90F0000F04BF0021704730B5A6
:100550004FF4806404F1320410F0004548BF40427B
:100560004FF000013EE700BF42004FEAE2014FEAD0
:1005700031014FEA02701FBF12F07F4393F07F4FAB
:1005800081F06051704732F07F4208BF704793F0AE
:100590007F4F04BF41F40021704730B54FF46074C1
:1005A00001F0004521F000411CE700BF50EA0102C4
:1005B00008BF704730B54FF000050AE050EA01026D
:1005C00008BF704730B511F0004502D5404261EBDD
:1005D00041014FF4806404F132045FEA915C3FF41E
:1005E000D8AE4FF003025FEADC0C18BF03325FEABB
:1005F000DC0C18BF033202EBDC02C2F1200300FA6C
:1006000003FC20FA02F001FA03FE40EA0E0021FA90
:1006100002F11444BDE600BF70B54FF0FF0C4CF47E
:10062000E06C1CEA11541DBF1CEA135594EA0C0F30
:1006300095EA0C0F00F0DEF82C4481EA030621EA6B
:100640004C5123EA4C5350EA013518BF52EA0335A6
:1006500041F4801143F4801338D0A0FB02CE4FF058
:100660000005E1FB02E506F00042E0FB03E54FF088
:100670000006E1FB03569CF0000F18BF4EF0010E80
:10068000A4F1FF04B6F5007F64F5407404D25FEA7C
:100690004E0E6D4146EB060642EAC62141EA55512F
:1006A0004FEAC52040EA5E504FEACE2EB4F1FD0C71
:1006B00088BFBCF5E06F1ED8BEF1004F08BF5FEAEF
:1006C000500E50F1000041EB045170BD06F00046A1
:1006D00046EA010140EA020081EA0301B4EB5C044E
:1006E000C2BFD4EB0C0541EA045170BD41F4801146
:1006F0004FF0000E013C00F3AB8014F1360FDEBF6B
:10070000002001F0004170BDC4F10004203C35DA46
:100710000C341BDC04F11404C4F1200500FA05F3C9
:1007200020FA04F001FA05F240EA020001F000426A
:1007300021F0004110EBD37021FA04F642EB0601E0
:100740005EEA430E08BF20EAD37070BDC4F10C040A
:10075000C4F1200500FA04F320FA05F001FA04F2CE
:1007600040EA020001F0004110EBD37041F10001BA
:100770005EEA430E08BF20EAD37070BDC4F12005C5
:1007800000FA05F24EEA020E20FA04F301FA05F22D
:1007900043EA020321FA04F001F0004121FA04F2D5
:1007A00020EA020000EBD3705EEA430E08BF20EAA5
:1007B000D37070BD94F0000F0FD101F000464000DF
:1007C00041EB010111F4801F08BF013CF7D041EA61
:1007D000060195F0000F18BF704703F00046520065
:1007E00043EB030313F4801F08BF013DF7D043EA36
:1007F0000603704794EA0C0F0CEA135518BF95EAEC
:100800000C0F0CD050EA410618BF52EA4306D1D172
:1008100081EA030101F000414FF0000070BD50EA91
:10082000410606BF1046194652EA430619D094EA1B
:100830000C0F02D150EA013613D195EA0C0F05D105
:1008400052EA03361CBF104619460AD181EA030159
:1008500001F0004141F0FE4141F470014FF0000011
:1008600070BD41F0FE4141F4780170BD70B54FF0AC
:10087000FF0C4CF4E06C1CEA11541DBF1CEA13552C
:1008800094EA0C0F95EA0C0F00F0A7F8A4EB05040E
:1008900081EA030E52EA03354FEA013100F0888005
:1008A0004FEA03334FF0805545EA131343EA1263CE
:1008B0004FEA022245EA111545EA10654FEA002683
:1008C0000EF000419D4208BF964244F1FD0404F53C
:1008D000407402D25B084FEA3202B61A65EB030598
:1008E0005B084FEA32024FF480104FF4002CB6EB55
:1008F000020E75EB030E22BFB61A754640EA0C00D5
:100900005B084FEA3202B6EB020E75EB030E22BF14
:10091000B61A754640EA5C005B084FEA3202B6EB55
:10092000020E75EB030E22BFB61A754640EA9C0014
:100930005B084FEA3202B6EB020E75EB030E22BFE4
:10094000B61A754640EADC0055EA060E18D04FEAA2
:10095000051545EA16754FEA06164FEAC30343EA42
:1009600052734FEAC2025FEA1C1CC0D111F4801F0F
:100970000BD141EA00014FF000004FF0004CB6E708
:1009800011F4801F04BF01430020B4F1FD0C88BFA7
:10099000BCF5E06F3FF6AFAEB5EB030C04BFB6EBB2
:1009A000020C5FEA500C50F1000041EB045170BDA5
:1009B0000EF0004E4EEA113114EB5C04C2BFD4EBD2
:1009C0000C0541EA045170BD41F480114FF0000E56
:1009D000013C90E645EA060E8DE60CEA135594EAD2
:1009E0000C0F08BF95EA0C0F3FF43BAF94EA0C0FD5
:1009F0000AD150EA01347FF434AF95EA0C0F7FF44A
:100A000025AF104619462CE795EA0C0F06D152EA9D
:100A100003353FF4FDAE1046194622E750EA410681
:100A200018BF52EA43067FF4C5AE50EA41047FF492
:100A30000DAF52EA43057FF4EBAE12E74FF0FF3CF7
:100A400006E000BF4FF0010C02E000BF4FF0010CC8
:100A50004DF804CD4FEA410C7FEA6C5C4FEA430C41
:100A600018BF7FEA6C5C1BD001B050EA410C0CBF90
:100A700052EA430C91EA030F02BF90EA020F0020F2
:100A8000704710F1000F91EA030F58BF994208BF59
:100A900090422CBFD8176FEAE37040F00100704716
:100AA0004FEA410C7FEA6C5C02D150EA013C07D16D
:100AB0004FEA430C7FEA6C5CD6D152EA033CD3D0B8
:100AC0005DF8040B704700BF8446104662468C46B2
:100AD0001946634600E000BF01B5FFF7B7FF0028E5
:100AE00048BF10F1000F01BD4DF808EDFFF7F4FF0E
:100AF0000CBF012000205DF808FB00BF4DF808ED99
:100B0000FFF7EAFF34BF012000205DF808FB00BFBB
:100B10004DF808EDFFF7E0FF94BF012000205DF8DD
:100B200008FB00BF4DF808EDFFF7CEFF94BF012092
:100B300000205DF808FB00BF4DF808EDFFF7C4FF8B
:100B400034BF012000205DF808FB00BF4A0011D22D
:100B500012F5001211D20DD56FF47873B3EB625217
:100B60000ED44FEAC12343F0004343EA505323FA23
:100B700002F070474FF00000704750EA013002D198
:100B80004FF0FF3070474FF0000070474FEA4102CE
:100B9000B2F1E04324BFB3F5001CDCF1FE5C0DD9DB
:100BA00001F0004C4FEAC0024CEA5070B2F1004F25
:100BB00040EB830008BF20F00100704711F0804F28
:100BC00021D113F13872BCBF01F00040704741F4ED
:100BD00080114FEA5252C2F11802C2F1200C10FAF1
:100BE0000CF320FA02F018BF40F001004FEAC123D5
:100BF0004FEAD32303FA0CFC40EA0C0023FA02F379
:100C00004FEA4303CCE77FEA625307D150EA01334E
:100C10001EBF4FF0FE4040F44000704701F000401E
:100C200040F0FE4040F40000704700BF80F00040FC
:100C300002E000BF81F0004142001FBF5FEA4103B4
:100C400092EA030F7FEA226C7FEA236C6AD04FEAB4
:100C50001262D2EB1363C1BFD218414048404140F9
:100C6000B8BF5B42192B88BF704710F0004F40F4AB
:100C7000000020F07F4018BF404211F0004F41F4C7
:100C8000000121F07F4118BF494292EA030F3FD093
:100C9000A2F1010241FA03FC10EB0C00C3F12003A6
:100CA00001FA03F100F0004302D5494260EB400035
:100CB000B0F5000F13D3B0F1807F06D340084FEAA0
:100CC000310102F10102FE2A51D2B1F1004F40EB95
:100CD000C25008BF20F0010040EA030070474900FD
:100CE00040EB0000013A28BFB0F5000FEDD2B0FA9A
:100CF00080FCACF1080CB2EB0C0200FA0CF0AABFBD
:100D000000EBC25052421843BCBFD040184370475A
:100D100092F0000F81F4000106BF80F40000013260
:100D2000013BB5E74FEA41037FEA226C18BF7FEA37
:100D3000236C21D092EA030F04D092F0000F08BF79
:100D40000846704790EA010F1CBF0020704712F060
:100D50007F4F04D1400028BF40F00040704712F19F
:100D600000723CBF00F50000704700F0004343F004
:100D7000FE4040F4000070477FEA226216BF08463A
:100D80007FEA23630146420206BF5FEA412390EAFD
:100D9000010F40F4800070474FF0000304E000BFF3
:100DA00010F0004348BF40425FEA000C08BF7047A4
:100DB00043F0964301464FF000001CE050EA010268
:100DC00008BF70474FF000030AE000BF50EA01027D
:100DD00008BF704711F0004302D5404261EB41016A
:100DE0005FEA010C02BF84460146002043F0B6438F
:100DF00008BFA3F18053A3F50003BCFA8CF2083AB4
:100E0000A3EBC25310DB01FA02FC634400FA02FCBC
:100E1000C2F12002BCF1004F20FA02F243EB0200C3
:100E200008BF20F00100704702F1200201FA02FC25
:100E3000C2F1200250EA4C0021FA02F243EB020018
:100E400008BF20EADC70704753B94AB9002908BFCF
:100E500000281CBF4FF0FF314FF0FF3000F0BEB94B
:100E6000ADF1080C6DE904CE00F03CF8DDF804E0CB
:100E7000DDE9022304B0704738B5002200230446A0
:100E80000D46FFF73BFE28B920462946BDE838400D
:100E900000F00AB8204605F1004100F005F8404294
:100EA00061EB410138BD00BFD0B50C4B00220646B6
:100EB0000F46FFF7B1FBFFF749FE0446FFF732FB91
:100EC000074B0022FFF7A8FB02460B463046394687
:100ED000FFF7EAF9FFF73AFE2146D0BD0000F03DEA
:100EE0000000F0412DE9F047089D8E4604468846F3
:100EF000002B4AD18A42174662D9B2FA82F64EB125
:100F0000C6F1200301FA06F820FA03F3B74043EADA
:100F10000808B4404FEA174E1FFA87FCB8FBFEF1F1
:100F2000230C0EFB118843EA084301FB0CF29A42A2
:100F300009D9FB1801F1FF3080F0EA809A4240F2B3
:100F4000E78002393B449A1AA3B2B2FBFEF00EFBD3
:100F5000102243EA024300FB0CFC9C4509D9FB1814
:100F600000F1FF3280F0D6809C4540F2D3803B44B4
:100F7000023840EA0140A3EB0C0300211DB1F3400D
:100F80000022C5E90032BDE8F0878B4205D90DB1DA
:100F9000C5E9000100210846F5E7B3FA83F100290D
:100FA00046D1734502D3824200F20581841A6EEB6A
:100FB000030201209046002DE5D0C5E90048E2E794
:100FC000002A00F09080B2FA82F6002E40F0A48051
:100FD0008A1A030C4FEA174E80B2BCB20121B2FB51
:100FE000FEFC0EFB1C2243EA024304FB0CF29A4275
:100FF00007D9FB180CF1FF3802D29A4200F2E080C8
:10100000C4469B1AB3FBFEF20EFB123340EA0343C5
:1010100002FB04F49C4207D9FB1802F1FF3002D214
:101020009C4200F2CA8002461B1B42EA0C40A5E724
:10103000C1F120068B4022FA06F71F430EFA01F495
:1010400020FA06F32EFA06FE4FEA1749234300FA68
:1010500001F81FFA87FCBEFBF9F01C0C09FB10EE2F
:1010600044EA0E4400FB0CFEA64502FA01F209D93F
:101070003C1900F1FF3A80F09C80A64540F299802F
:1010800002383C44A4EB0E041FFA83FEB4FBF9F3D0
:1010900009FB13444EEA044403FB0CFCA44508D9A5
:1010A0003C1903F1FF3E80F08280A4457FD9023BCA
:1010B0003C4443EA0040A4EB0C04A0FB02EC644572
:1010C0007346E14662D35FD05DB1B8EB030264EBD7
:1010D000090404FA06F622FA01F31E43CC40C5E9DE
:1010E000006400214FE7B1FBF2FC010C41EA0E4124
:1010F00080B240EA01423B4638463C46B846BE46CE
:101100002026B1FBF7F1A2EB080241EA0C4166E7A9
:10111000014618E710462CE7C6F120022EFA02F32A
:10112000B740B14020FA02F24FEA174E0A43B3FB30
:10113000FEF8BCB20EFB1833110C41EA034108FB68
:1011400004F9B04089454FEA104380B23ED979187E
:1011500008F1FF3C01D289451FD8A1EB0901B1FB81
:10116000FEF909FB04F80EFB191192B242EA0142A2
:10117000424529D2BA1809F1FF31C4D24245C2D240
:10118000A9F102013A44BEE7F0459DD2BEEB02034D
:101190006CEB070C0138E14696E7A7EB09094944D7
:1011A000A8F1020CB1FBFEF909FB04F8DBE773467A
:1011B0007FE7504666E70846FDE63B44023A33E7E0
:1011C000ACF1020C3B441CE749469CE7A1EB09014A
:1011D000C446B1FBFEF909FB04F8C4E7704700BF41
:1011E000044B026800211970D36843F02003D360D8
:1011F000704700BF8806002038B50B4C23784FF4A9
:101200001652054643F00103426023700DF08AF840
:101210002A68D36843F08003D3602378DB07FCD4CB
:101220002078C0F3400038BD8806002010B4084C78
:101230000068237843F001032370064CC3682160E3
:10124000054943F080030A705DF8044BC3607047A2
:1012500088060020840600208206002030B554074E
:101260004FEAD20319D001334FF0FF0E01EB030C0C
:10127000013B13F0FF030CF801ECF7D1084C0068B8
:101280002378084D43F001032370C368064C29609E
:1012900043F080032270C36030BD002BE4D1EDE742
:1012A000880600208406002082060020E9B100B5EF
:1012B0008646084400211EF801CB08228CEA01036F
:1012C00043F3000323F0730383EA5101531E13F029
:1012D000FF02C9B24FEA5C0CF0D17045EBD1007847
:1012E000401A18BF01205DF804FB0078401A18BFAF
:1012F0000120704738B503681968DC688906024622
:1013000001D5A5062FD41968D8680C062AD5010680
:1013100028D55268B2F5165F49D04548027832B9EF
:10132000444C454924680A70444924780C70444967
:101330000978914245D0414C2178013211F00105E4
:1013400018BFFF25D2B25D604908530721700270B3
:1013500008D1394A3749137809680133DBB2137071
:10136000CB5C237038BD44685968B4F5165FC9B2C8
:1013700048D0344C344D20782B784008FF2908BFE2
:1013800040F0800020702E485A1C0078D2B2904263
:101390002A7002F007011BD00029E3D12B4B25490D
:1013A0001A78086824788454511C197038BDF022CA
:1013B0005A60DA681E49002022F080020870DA6064
:1013C00038BDDA68002122F080020170DA6038BD91
:1013D00002332278DBB239B103F00701013352083E
:1013E000DBB20029F8D12270184812490378096845
:1013F000CA5417490B78002262F300032A70027066
:101400000B7038BD124CB1F1F003217818BF0123E5
:1014100063F341014FF4E133217043600CF082FF2C
:1014200023780949002262F300030A70237038BD53
:101430007E060020840600207D0600207C06002019
:101440008206002080060020810600207F06002002
:10145000880600200000000000B51F481F499FEDCE
:101460001A7B4FF4803285B00023C0E900120122BC
:10147000CDE90033CDE9023380ED0A7B836003615F
:10148000037680F82030C360C26180F8303042615A
:1014900007F0EEFE68B99FED0E7B00230E48029325
:1014A00069468DED007B08F06FF828B905B05DF84E
:1014B00004FB06F02BFAEEE706F028FA05B05DF81B
:1014C00004FB00BFAFF300800100000F000000002C
:1014D0000A000000010000009006002000200140EA
:1014E00000B5194A016889B000239142CDE9023361
:1014F000CDE90433069302D009B05DF804FB02F590
:101500008C320093506C40F480705064506C00F446
:101510008070009000980193136B0C4843F0040313
:101520001363136B9FED067B03F00403019302A981
:101530008DED027B019B09F0A3F909B05DF804FB76
:1015400001000000030000000020014000080240EC
:10155000064A08B5536943F008030920536108F0AF
:101560003BF9BDE80840092008F004B9003C0140FF
:10157000092008F00DB900BF10B4144B1B689A681D
:101580009207FCD50022DA609A68D407FCD5D968A6
:101590009A689007FCD50022DA609A68D207FCD5D9
:1015A000D8689A689407FCD50022DA609A68D20756
:1015B000FCD5DC6802020B0403F47F0392B2E0B2B4
:1015C000134318435DF8044B704700BFC89D0020CB
:1015D00010B51D4C23787BB11C4BD3ED007AF4EE93
:1015E000C07AF1EE10FA08D9194BD3ED007AF4EE77
:1015F000C07AF1EE10FA13DA10BD164B012293E80F
:10160000030005F097FB144A0121042004F076FF43
:10161000114A0121082004F071FF0023237010BD3E
:101620000C4B012293E8030005F084FB0A4A0121D8
:10163000042004F063FF084A0021082004F05EFF44
:101640000023237010BD00BF1561002000000020A2
:10165000F460002028690208249C002030B4174D53
:10166000174C226829682B682868D205490401F0C4
:10167000007102F080729B020A4303F080631343FF
:1016800080052A6800F000601843D30623682168AB
:1016900022684FEA83434FEA017103F0005301F0DF
:1016A00080414FEA027243EA010302F0004218BF90
:1016B00040F080501343184330BC7047289C0020F2
:1016C000249C00202DE9F0432DED028B9A4A9B4B80
:1016D0009B4D9C4C83B04FF4007100200190C2F8E8
:1016E00080115A69110744BF08225A61FFF744FF6D
:1016F000296803464FF40050236004F0F9FE0028E7
:1017000040F0A6802368904C904E1A02D4E9002144
:1017100048BF43F07F43D21841EBE371C4E9002195
:101720008B4A3368126801339342336071D3894F17
:101730003B6801333B60884B1B78002B40F0B28044
:10174000864B1B78002B40F0A18029684FF4005095
:1017500004F0CEFE002840F08A80814BDFF84092F2
:1017600093ED008A7F4BD4E90001D3ED008AFFF7A7
:101770002DFB7D4B07EE900A93ED007A77EEC77A4A
:101780000022F5EEC07AF1EE10FAA8BF87EE887A53
:101790004FF000034FF00008C4E90023C6F80080B2
:1017A000B8BF87EEA87A89ED007A99ED000AFFF7B5
:1017B0000FFF6E4B0120196804F09AFE04460028C2
:1017C00038D06B4C6B4EFFF749FF23783268DFF857
:1017D000D4C13F68D9ED007A9CF800E04FF4B461C1
:1017E00001FB03F3644903EBC20367F31700013203
:1017F00003EB0109C9ED017A3260C850BEF1000F58
:1018000003D05E4B1B689F426CD25D4B1B689342BA
:1018100056D9019B4BB14FF0E0234FF08052C3F8F3
:10182000042DBFF34F8FBFF36F8F03B0BDEC028B5E
:10183000BDE8F08300F010F9524A137803F0FF017D
:10184000002B3BD1504B1A78002A69D01970E0E781
:1018500029684FF4805004F04BFE00287FF452AF0B
:101860004A4B024693E8030005F064FA4AE7296808
:101870004FF4805004F03CFE00287FF46EAF434BE1
:10188000012293E8030005F055FA66E7092007F006
:101890007FFF29684FF4005004F02AFE00283FF42F
:1018A0005CAFE4E7394B002293E8030005F042FA0D
:1018B0002A4B1B78002B3FF448AFE7E71470A8E7EA
:1018C000334B34491A60237808680133DBB2237044
:1018D0002378002203F00F0301A93260237012F075
:1018E00061FC96E78CF8008000F0B6F8284B32686F
:1018F0001A602378274AC6F800800133DBB22370D0
:101900002378106803F00F0301A9237012F04AFC3A
:1019100029684FF4805004F0EBFD38B1326874E769
:101920001D4B01A9186812F03DFC72E71B4B1868AB
:1019300013F040F9F2E700BF00E100E0003C014095
:10194000209C002008610020006100201861002018
:10195000040000201C610020176100201661002097
:10196000EC600020E8600020F0600020249C002053
:10197000E4600020E0600020D80600201061002014
:10198000D860002061610020606100203869020891
:10199000DC600020149C0020109C0020009C002093
:1019A000F86000200C610020174B10B593E803008D
:1019B000012205F0BFF9154B154C93E803000022F6
:1019C00005F0B8F9134B002293E8030005F0B2F9D3
:1019D000114B012293E8030005F0ACF90F4B0022F4
:1019E00093E8030005F0A6F994E80300002205F04F
:1019F000A1F90A2007F02AFC94E803000122BDE8BF
:101A0000104005F097B900BF78360208703602081A
:101A100080360208683602086036020888360208F6
:101A200008B50A4BDA6822F00202DA609A6842F0DE
:101A300002029A605A6942F0020207205A6107F0D6
:101A4000CBFEBDE80840072007F094BE003C0140F3
:101A5000072007F09DBE00BF08B5FFF789FDFFF71F
:101A6000F7FF08480CF04EF9074B002293E80300FB
:101A700005F060F9BDE80840044A0021012004F0A7
:101A80003DBD00BFB89E002038690208249C00209C
:101A900038B5674C4FF48070216804F029FD0028A8
:101AA00056D121684FF4005004F022FD00284FD198
:101AB000604B00221A7021685F4D4FF4805004F093
:101AC00017FD01286BD15D4B01221A702968042093
:101AD00004F00EFD002871D0594B00221A702168C5
:101AE0004FF4805004F004FD01284CD1554B9FED7C
:101AF000566AD3ED006A9FED557A554BC6EE267AAD
:101B000067EE877AFCEEE77AC3ED007A04F0E6FA36
:101B1000504B186004F070F94F48504A5049002368
:101B200003609FED417B4F4813704F4A0B60036089
:101B300021684FF4805082ED007B04F0D9FC01282D
:101B4000216846D04FF4805004F0D2FC50B138BD2B
:101B500021684FF4805004F0CBFC0128A8D1354B0C
:101B60001870A8E72168802004F0C2FC002856D134
:101B700021684FF4807004F0BBFC002844D1BDE81C
:101B80003840FFF7E5BC21684FF4805004F0B0FC0A
:101B90000028BBD1354A2E4B12681A60B6E7296877
:101BA000012004F0A5FC00288DD0244B00221A70DF
:101BB0002968042004F09CFC00288DD121684FF492
:101BC000007004F095FC002886D01D4B01221A708D
:101BD00085E7802004F08CFC98B91A4B93ED000A3D
:101BE00004F08EFA2168202004F082FC0128AED196
:101BF0002968202004F07CFC0128A8D11C4B187017
:101C000038BDFFF70DFFEDE71A4B002293E8030004
:101C100005F090F8B3EE040A04F072FAAFE7FFF7AC
:101C2000FFFEA5E7AFF30080000000000000000009
:101C3000209C002017610020249C002016610020B9
:101C400015610020406300200050C3476666663F70
:101C500004000020D860002018610020E46000200B
:101C6000E06000201C61002000610020486300202B
:101C7000146100203869020870B59A4C237882B04C
:101C800000224F2B019211D0974D0120296804F0BA
:101C90002FFC00286ED123784F2B31D023783F2B97
:101CA00079D0012004F0FCFA02B070BD6378462BB5
:101CB000EAD1A378462BE7D1E678002EE4D1FFF7EE
:101CC00057FCFFF7C5FE8948874D894C0CF01AF880
:101CD000884B324693E8030005F02CF801202A4691
:101CE000314604F00BFC21684FF4805004F000FCF6
:101CF00001286BD08049814804F0C4FA02B070BD5D
:101D000063784E2BCAD17E4B1B78002BC6D1296835
:101D1000012004F0EDFB002840F09180774C744ED8
:101D20002378042B00F0B3802378012B00F08B8004
:101D300031684FF4805004F0DBFB012800F08F8005
:101D400001210846684A04F0D9FB6E496B4801231B
:101D5000052204F0F1F931684FF4805004F0C8FB1B
:101D600010B9694B03221A70642007F06FFAFFF76D
:101D70008FFE99E75E4E1020316804F0B9FB002811
:101D800089D031684FF4805004F0B2FB012882D131
:101D900004F09EFA88E76378002B82D1296801203D
:101DA00004F0A6FB58B92968012004F0A1FB002823
:101DB00066D05649514804F065FA02B070BD544AE5
:101DC000524B92E8030018601971F2E72168202055
:101DD00004F08EFB01288DD12968202004F088FBB7
:101DE000012887D14B4B1A78012A83D14A4A1E70A9
:101DF00013684A4C83F00103136004F063F8484B06
:101E000048491A680968484B1268484811F09EF81A
:101E1000207000285DD1454811F0DCF920700028C1
:101E200040F0BE80414811F051FA01462070002870
:101E300040F0BF802C4A102004F060FB5AE70B20D2
:101E400004F02EFA30E731684FF4805004F050FB74
:101E500000287FF46DAF1A2004F022FA24E73168DD
:101E6000202004F045FB012804467FF469AF29686F
:101E7000202004F03DFBB0B9102004F011FA13E764
:101E80002B4A224B92E803001860998091E7316851
:101E90004FF4805004F02CFB00287FF445AF07205E
:101EA00004F0FEF900E723481C4E202104F02CF832
:101EB00020491E480A2210F06BFD307000283DD0EA
:101EC0001D4A2146022004F019FB0C2004F0E8F919
:101ED000EAE6194A0121042004F010FB0E2004F068
:101EE000DFF9E1E65C9B0020249C0020B89E0020E6
:101EF000209C00203869020894360208DE87002002
:101F00005E9B002008690208DD8700202061002018
:101F1000A4360208146100206C6300207083002046
:101F2000586300205C630020546300207483002009
:101F3000AC3602081C620020289C002004F018F82F
:101F40002048FEF74FF91F49024601AB1E4810F02A
:101F5000FDFF30700028BCD11B4811F03BF905464D
:101F60003070E8B92146194A102004F0C7FA184B1E
:101F7000184A19491D60194B15600D60204621460D
:101F8000124A1D6004F0BAFA154916482346052284
:101F900004F0D2F8642007F059F9FFF779FD83E6E1
:101FA000114A0121082004F0A9FA0F2004F078F961
:101FB0007AE60D4A0121102004F0A0FA0D2004F069
:101FC0006FF971E67063002074830020249C002068
:101FD000646300206C63002060630020686300205D
:101FE00008690208DE870020289C002070B5174C85
:101FF0000120216804F07CFA28B1154D10202968D1
:1020000004F076FA70B92168012004F071FA28B161
:102010000F4B1020196804F06BFA70B1BDE87040E6
:10202000FFF736BD29684FF4805004F061FA0128AB
:10203000E9D1BDE8704004F04BB9064A0346BDE85B
:102040007040106819461A4611F034BF249C0020D5
:10205000209C0020109C002038B523481DF005FD71
:10206000224B04461968012004F042FA20BB621E8C
:1020700041F287339A421AD81D4B1C4A1C60012139
:10208000084604F03BFA1B4A1B4B012111701968EA
:102090004FF4805004F02CFA00B3184B0222642055
:1020A0001A7007F0D3F8BDE83840FFF7F1BCBDE87F
:1020B0003840012004F0F4B80F4D1020296804F0D6
:1020C00017FA0028D3D029684FF4805004F010FA92
:1020D0000128CCD1BDE8384004F0FAB8084B1868A4
:1020E00013F00CF8D9E700BF5C9B0020249C002073
:1020F000106100200C610020209C0020DD87002062
:10210000009C002030B5544C8BB02168012004F0B5
:10211000EFF9002834D1514B1A783F2A1BD01A7896
:102120004E2A40D02168012004F0E2F9044600283C
:102130006AD109AA08ABCDE900324949474807AB43
:1021400006AA1EF097FC43B2042B63D0012004F0D2
:10215000A7F80BB030BD5A78002AE0D1414A424975
:10216000D478907853781278CDE900043F481EF077
:102170005FFC3E493E480BB0BDE8304004F082B8F9
:102180003C4D1020296804F0B3F90028C3D0296819
:102190004FF4805004F0ACF90128BCD10BB0BDE87D
:1021A000304004F095B85B78452BBBD1324B1A78A0
:1021B000572AB7D15B78002BB4D1304B1A783F2A1D
:1021C000C4D15B78002BC1D105AB4FF47A710422E6
:1021D000CDE90121009330220123A021284809F0F4
:1021E00023F99DF816209DF817401F499DF81530DA
:1021F0001E48CDE900249DF814201EF019FC1B494F
:102200001B4804F03FF8A4E703200BB0BDE83040C2
:1022100004F046B8DDE90601089A60F3070461F3AB
:102220000F24099862F317444FF47A7105AACDE997
:10223000002360F31F64029101233022A021104883
:10224000059409F055F8322007F000F80D490848C8
:1022500004F018F87DE700BF249C00205C9B002060
:10226000C836020854A00020B436020820610020BD
:10227000DE870020209C00205E9B00203C9B0020ED
:10228000A09B00209436020830B5544C8BB02168D6
:10229000012004F02DF9002834D1514B1A783F2A3F
:1022A0001BD01A784E2A40D02168012004F020F972
:1022B000044600286AD109AA08ABCDE90032494991
:1022C000474807AB06AA1EF0D5FB43B2042B63D0E8
:1022D000012003F0E5FF0BB030BD5A78002AE0D1B1
:1022E000414A4249D478907853781278CDE9000475
:1022F0003F481EF09DFB3E493E480BB0BDE83040D4
:1023000003F0C0BF3C4D1020296804F0F1F800280C
:10231000C3D029684FF4805004F0EAF80128BCD1FA
:102320000BB0BDE8304003F0D3BF5B78452BBBD189
:10233000324B1A78572AB7D15B78002BB4D1304B87
:102340001A783F2AC4D15B78002BC1D105AB4FF47A
:102350007A710422CDE90121009334220123A021C6
:10236000284809F061F89DF816209DF817401F498C
:102370009DF815301E48CDE900249DF814201EF06C
:1023800057FB1B491B4803F07DFFA4E703200BB05C
:10239000BDE8304003F084BFDDE90601089A60F330
:1023A000070461F30F24099862F317444FF47A711C
:1023B00005AACDE9002360F31F64029101233422B2
:1023C000A0211048059408F093FF322006F03EFF4C
:1023D0000D49084803F056FF7DE700BF249C00200C
:1023E0005C9B0020C836020850A00020B4360208CA
:1023F00020610020DE870020209C00205E9B0020C2
:102400003C9B0020A09B00209436020830B5544C21
:102410008BB02168012004F06BF8002834D1514BB7
:102420001A783F2A1BD01A784E2A40D02168012002
:1024300004F05EF8044600286AD109AA08ABCDE989
:1024400000324949474807AB06AA1EF013FB43B2C6
:10245000042B63D0012003F023FF0BB030BD5A786A
:10246000002AE0D1414A4249D478907853781278D2
:10247000CDE900043F481EF0DBFA3E493E480BB070
:10248000BDE8304003F0FEBE3C4D1020296804F04A
:102490002FF80028C3D029684FF4805004F028F8A2
:1024A0000128BCD10BB0BDE8304003F011BF5B7810
:1024B000452BBBD1324B1A78572AB7D15B78002B0A
:1024C000B4D1304B1A783F2AC4D15B78002BC1D1EC
:1024D00005AB4FF47A710422CDE901210093382233
:1024E0000123A021284808F09FFF9DF816209DF8A1
:1024F00017401F499DF815301E48CDE900249DF86E
:1025000014201EF095FA1B491B4803F0BBFEA4E7FC
:1025100003200BB0BDE8304003F0C2BEDDE9060188
:10252000089A60F3070461F30F24099862F31744D3
:102530004FF47A7105AACDE9002360F31F6402917C
:1025400001233822A0211048059408F0D1FE322042
:1025500006F07CFE0D49084803F094FE7DE700BFBD
:10256000249C00205C9B0020C83602084CA0002060
:10257000B436020820610020DE870020209C002065
:102580005E9B00203C9B0020A09B0020943602080C
:1025900030B5644C8DB02168012003F0A9FF0028FC
:1025A00033D1614B1A783F2A16D01A784E2A3FD081
:1025B0002168012003F09CFF054600286FD12168A7
:1025C0004FF4007003F094FF00286ED117200DB077
:1025D000BDE8304003F064BE5A78002AE5D1534A82
:1025E000534950791379D478CDE9023090785378F3
:1025F0001278CDE900044F481EF01AFA4D494E48B2
:102600000DB0BDE8304003F03DBE4C4D10202968B0
:1026100003F06EFF0028C4D029684FF4805003F007
:1026200067FF0128BDD10DB0BDE8304003F050BEBA
:102630005B78452BBCD1424B1A78572AB8D15B78CE
:10264000002BB5D13F4B1A783F2A3FD15B78002B46
:102650003CD104AB4FF47A710622CDE901210093FD
:1026600040220123A021384808F0DEFE9DF8152005
:102670009DF814309DF813402D492E48CDE90232C3
:102680009DF812209DF81130CDE900249DF810200E
:102690001EF0CEF92749284803F0F4FD19E0032085
:1026A0000DB0BDE8304003F0FBBD0BA80AA909AA94
:1026B00008ABCDE90210CDE9003224491A4807AB36
:1026C00006AA1EF0D7F940B2062804D0012003F074
:1026D000E7FD0DB030BDDDE90612089B61F307058B
:1026E00062F30F25099A0A998DF8141063F31745C0
:1026F0004FF47A7404ABCDE90030029462F31F65A5
:102700000B9C1148049501234022A0218DF815400F
:1027100008F0EEFD322006F099FD0D49064803F061
:10272000B1FDD6E7249C00205C9B0020C8A00020BF
:10273000D836020820610020DE870020209C00207F
:102740005E9B00203C9B0020A09B0020F8360208E6
:102750009436020830B5334C87B0002321680593C6
:10276000012003F0C5FE00283DD12F4D2B783F2BD3
:102770002AD02168012003F0BBFE002849D12B7824
:102780002A4AD35C5B073FD527481DF06EF94FF608
:10279000FE73421E9A42059040D8254C05AB4FF47B
:1027A0007A710422CDE90121009360220123A02146
:1027B0002060204808F09CFD322006F047FD1E49AD
:1027C0001E4803F05FFD0CE06B78002BD1D1184B55
:1027D0001B491A681B481EF02BF91A49174803F0C9
:1027E00051FD07B030BD184D1020296803F080FE60
:1027F0000028BAD029684FF4805003F079FE0128F0
:10280000B3D103F065FDECE7012003F049FD07B00B
:1028100030BD032003F044FD07B030BD022003F0BB
:102820003FFDDEE7249C00205C9B0020997102089C
:1028300074030020A09B002094360208DE8700204D
:10284000303A020820610020209C00202DE9F0434E
:10285000624C85B02168012003F04AFE00283FD178
:102860005F4D2B783F2B10D05E495D48FDF7B0FCE3
:102870000446002842D02B78432B00F083800120AF
:1028800005B0BDE8F04303F00BBD6B78002BEBD136
:1028900021684FF4007003F02BFE38B921684FF423
:1028A000805003F025FE002800F093804E4C4F4BE3
:1028B0000C2293ED000A40210023204603F00EFA7B
:1028C0002046FDF78FFC4A4B0219198821529B784C
:1028D00048489370214605B0BDE8F04303F0D2BCF0
:1028E000454B4FF48050196803F002FE01286BD06D
:1028F000062005B0BDE8F04303F0D2BC3E4E3F4D8C
:102900003F4F404BD7F800803B6001222A700146C0
:1029100032464FF48050D6F8009003F0EFFD324677
:1029200021464FF4006003F0E9FD32462146802045
:1029300003F0E4FD324621464FF4807003F0DEFDE3
:10294000FFF7A6F82B78002BFCD12F4BC6F8009090
:1029500093ED007ADFED2D7AC7F80080B4EEE77AC8
:10296000F1EE10FA08DB93ED007ADFED297AB4EE90
:10297000E77AF1EE10FA2ED9182005B0BDE8F04341
:1029800003F08EBC6B784C2B7FF479AF214B1A7817
:10299000522A7FF474AF5B78002B7FF470AF13483A
:1029A000002404234FF47A72CDE901320090A02173
:1029B000012328220460184808F09AFC322006F00F
:1029C00045FC16490B4886E705B0BDE8F04303F027
:1029D0007FBC172054E705481C68E2E7249C0020D0
:1029E0005C9B002010370208206100206C610020F1
:1029F00040380208DE870020209C00206161002012
:102A000048630020A0860100F86000200050C3C782
:102A10000050C3475E9B0020A09B00209436020814
:102A2000D0B57348734C84B01DF01CF821680120A8
:102A300057EC106B03F05CFD68B16F4B4FF48050A6
:102A4000196803F055FD012822D0062004B0BDE826
:102A5000D04003F025BC21684FF4007003F048FD1E
:102A6000002842D0654C2378432B47D03046394666
:102A7000FEF78CF82378502B07EE900A64D0237869
:102A80004E2B0AD0012004B0BDE8D04003F008BCB2
:102A900004B0BDE8D04003F01BBC6378452BF1D1F6
:102AA000574B1A78472AEDD15B78002BEAD1504B6F
:102AB0001A783F2A00F09580B7EE007AF4EEC77AD4
:102AC000F1EE10FADEDB9FED4F7AF4EEC77AF1EE0D
:102AD00010FAD7D804234FF47A724B4C4B48009429
:102AE000CDE901320123502254E021684FF4805097
:102AF00003F0FEFC0028B5D11720A7E763784C2B24
:102B0000B4D1A378522BB1D1E378002BAED1404B96
:102B10003D4C00934FF07E524FF47A770426CDE976
:102B20000167A0211A60226001234A22374808F079
:102B3000DFFB322006F08AFBCDE9016733480094C1
:102B400001235022A02128E063784F2B97D12C4BF2
:102B50001A78532A93D15B78002B90D1244B1A78A2
:102B60003F2A26D0B7EE007AF4EEC77AF1EE10FADB
:102B700088DB9FED247AF4EEC77AF1EE10FA81D863
:102B800004234FF47A72224C20480094CDE901329C
:102B900001234A22A021C4ED007A08F0A9FB3220CB
:102BA00006F054FB1B491C4804B0BDE8D04003F0BC
:102BB00069BB5B78002BD5D1154A184C92ED000A01
:102BC00040210A22204603F089F82046FDF70AFB3F
:102BD000134B021919889B7821520F489370214694
:102BE000E2E75B78002B7FF467AF074AE5E700BFB9
:102BF0003C9B0020249C0020209C00205C9B00200B
:102C00005E9B00200050C34764610020A09B002011
:102C10006861002094360208DE87002020610020D1
:102C2000403802082DE9F04F2DED028B87B0844823
:102C3000844C05A91DF060FD2168012057EC106B44
:102C400003F056FC78B1804C4FF48050216803F0BB
:102C50004FFC012825D0032003F022FB07B0BDEC78
:102C6000028BBDE8F08F21684FF4007003F040FC48
:102C700008B3059B724A93420BD01B784BB9734C37
:102C80002378502B22D023784E2B02D16378452B0A
:102C900053D0012003F004FB07B0BDEC028BBDE86C
:102CA000F08F22460021102003F028FC07B0BDEC75
:102CB000028BBDE8F08F21684FF4805003F018FCC0
:102CC0000028D6D1172003F0EBFAC7E763784F2B23
:102CD000D9D1254615F8023F532BD4D1A04618F878
:102CE000033F002BCFD130463946FDF74FFFDFEDD4
:102CF000587A08EE100AB4EEE78AF1EE10FA0BDB10
:102D0000DFED547AB4EEE78AF1EE10FA04D8B5EEAE
:102D1000408AF1EE10FA1AD1022003F0C1FA00261F
:102D2000494FDFF85491B246C9F80060C7F800A0D7
:102D300007B0BDEC028BBDE8F08F474D2B78472BD9
:102D4000A7D1A84618F8013F002BA2D1CBE73E4FF0
:102D5000DFF828B1DFF8209101238BF800303A46E4
:102D60003E4BD9F80060D7F800A0C9F80030002128
:102D70004FF4805003F0C2FB3A4600214FF400604C
:102D800003F0BCFB3A460021802003F0B7FB3A4633
:102D900000214FF4807003F0B1FBFEF779FE9BF841
:102DA0000030002BFBD12378502B06D023784E2BFC
:102DB00029D0012003F074FAB6E763784F2BF5D1E0
:102DC0002B78532BF2D198F80030002BEED1244B06
:102DD000244893ED007A244B0093C7EE087A4FF411
:102DE0007A714A22C3ED007A0423CDE9013101232F
:102DF000A02108F07DFA322006F028FA1B491C4871
:102E000003F040FA90E76378452BD2D12B78472B1B
:102E1000CFD198F80030002BCBD1114B114893ED56
:102E2000007A144B0093C7EE087A4FF47A72C3ED20
:102E3000007A0423CDE9013201235022D8E700BFF4
:102E40003C9B0020249C0020209C00205C9B0020B8
:102E5000000096C4000096445E9B0020A0860100FE
:102E6000F8600020A09B00206861002094360208D2
:102E7000DE8700206461002048630020606100203C
:102E8000174B10B51968012003F032FBB0B9154B90
:102E90001A783F2A04D0BDE81040012003F000BAA0
:102EA0005B78002BF7D11049104A11481DF0C0FD86
:102EB000BDE810400E490F4803F0E4B90E4C102055
:102EC000216803F015FB0028E1D021684FF4805001
:102ED00003F00EFB0128DAD1BDE8104003F0F8B989
:102EE000249C00205C9B0020243702081C37020829
:102EF00020610020DE870020209C00202DE9F04F7B
:102F0000DFF8749185B0D9F80010012003F0F0FAD1
:102F1000002872D1534B1A783F2A05D0012005B002
:102F2000BDE8F04F03F0BCB95D78002DF6D1DFF8B5
:102F30004C81D8F80030002B52D0DFF844B14A4C15
:102F4000DFF840A12E460DE0D9F800104FF40070D4
:102F500003F0CEFA98B906EB8603354658F82330CD
:102F6000002B3DD005EB850308EB830301361A7A6D
:102F7000022A4FEA8507F6B253D0042AE4D03D4432
:102F800008EB850758F82530FA68009240215A4628
:102F900020461DF017FDD9F800104FF4007003F023
:102FA000A7FA012848D02046FDF71CF95146C0F188
:102FB0003F0220461DF010FE2046FDF713F92B4F6F
:102FC000054601232A462146384603F0B5F8002875
:102FD000F7D106EB8603354658F82330002BC1D1D4
:102FE000224C322006F032F92149204603F04AF9FA
:102FF0000023237005B0BDE8F08F1E4C102021681F
:1030000003F076FA002885D021684FF4805003F051
:103010006FFA01287FF47EAF05B0BDE8F04F03F0F2
:1030200057B9D9F8001003934FF4007003F060FA19
:10303000039B58B11A7AA0E72046FDF7D3F8396907
:10304000C0F13F0220461DF0C7FDACE7D9F80010E3
:1030500003934FF4805003F04BFA039B0028E9D10F
:1030600079E700BF5C9B002020610020DE87002004
:1030700094360208209C0020249C00205800002048
:10308000383702084038020838B56D4D01202968EC
:1030900003F02EFA002833D16A4C23783F2B19D045
:1030A0002968012003F024FA002840F08780237863
:1030B000492B37D023784F2B00F08D802378532B6A
:1030C00050D023784F2B00F09E80BDE8384001207F
:1030D00003F0E6B86378002BE2D15B4C80202168D6
:1030E00003F006FA002857D0584A594B1068127955
:1030F00018601A71BDE838405549564803F0C2B807
:10310000514C1020216803F0F3F90028C4D0216845
:103110004FF4805003F0ECF90128BDD1BDE83840F0
:1031200003F0D6B863784E2BC4D14B4B1D78002DDD
:10313000C0D1454A8020012103F0E0F9424A4FF412
:103140008070294603F0DAF93F4A4FF400502946CF
:1031500003F0D4F903F0DCF9BDE838403F493D48BD
:1031600003F090B86378592BABD13B4B1A78542AB3
:10317000A7D15D78002DA4D1334A29464FF4807041
:1031800003F0BCF9304A8020294603F0B7F92E4AF3
:1031900001214FF40050DBE721684FF4807003F009
:1031A000A7F980B12E4A2A4B1068928818609A803D
:1031B000BDE838402649274803F064B8BDE83840E8
:1031C000062003F06DB821684FF4005003F090F929
:1031D000B8B1244AE7E76378552B7FF46FAF1E4BF5
:1031E0001A78542A7FF46AAF5D78002D7FF466AFB9
:1031F000154A4FF48070012103F080F9124A8020B3
:103200009FE7194ACFE76378462B7FF45EAF124BF6
:103210001A78462A7FF459AF5C78002C7FF455AFBA
:10322000094A21464FF4807003F068F9064A80206D
:10323000214603F063F9044A4FF40050214687E722
:10324000249C00205C9B0020209C00204437020826
:1032500020610020DE8700205E9B0020943602085B
:103260004C37020854370208AC36020838B53E4CD9
:103270000120216803F03CF930B13C4D1020296851
:1032800003F036F900284AD121684FF4007003F0AA
:103290002FF970B1364B1A784F2A16D01A784F2A68
:1032A0004FD01A783F2A24D0BDE83840012002F0E0
:1032B000F7BF21684FF4805003F01AF90028E9D1D4
:1032C000BDE83840172002F0EBBF5A784E2AE5D10E
:1032D0009A78002AE2D1254A01214FF4006003F0D8
:1032E0000DF903F015F9BDE838402249224802F0F3
:1032F000C9BF5B78002BD7D11C4C4FF4006021680C
:1033000003F0F6F8B0B921684FF4006003F0F0F86C
:1033100018B3BDE838401949174802F0B3BF29680F
:103320004FF4805003F0E4F80128ADD1BDE83840F7
:1033300002F0CEBF124A114B1068127918601A7150
:10334000E7E75A78462AACD10E4A11784629A8D127
:1033500051780029A5D1054ABFE70B4A074B1068F1
:10336000928818609A80D4E7249C0020209C00203A
:103370005C9B002094360208DE870020206100203C
:10338000A43602085E9B0020AC36020810B53D4B07
:103390008CB01968012003F0ABF800285ED13A4BDD
:1033A0001A783F2A3CD005AB0024009337493648B1
:1033B000059404AB03AACDE903441DF05BFB40B2C6
:1033C000032828D1039B04993148172B94BFDCB202
:1033D0000394059B8DF818403B2986BF002104917A
:1033E000C9B23B2B88BF00234FF0000298BFDBB26D
:1033F0008DF8191006A9CDE9092288BF05938DF82B
:103400001A308DF81B2009F095FB2249224802F062
:1034100039FF0CB010BD012002F042FF0CB010BD0E
:103420005C78002CBFD1224606A9194809F084FA1D
:10343000224605A9164809F0BBFA9DF81A409DF8E6
:1034400019309DF818201549009415481DF0F0FA20
:103450001349114802F016FF0CB010BD114C10209A
:10346000216803F045F8002899D021684FF4805076
:1034700003F03EF8012892D10CB0BDE8104002F0F4
:1034800027BF00BF249C00205C9B0020CC36020894
:10349000489C002094360208DE8700206837020826
:1034A00020610020209C002010B53A4B86B019689E
:1034B000012003F01DF8002858D1374B1A783F2A15
:1034C0003CD005AB0024009334493348059404AB49
:1034D00003AACDE903441DF0CDFA40B2032828D158
:1034E00003980499059B1F2886BF01200390C0B252
:1034F0000C2986BF01210491C9B2632B8CBF002324
:10350000DBB24FF000028DF80A008DF809104FF081
:10351000010402A9224888BF05938DF80B308DF86D
:10352000084009F085FB1F491F4802F0ABFE06B0BA
:1035300010BD012002F0B4FE06B010BD5A78002A7A
:10354000BFD102A9164809F033FA9DF80B409DF847
:1035500009309DF80A201549009415481DF068FAB5
:103560001349114802F08EFE06B010BD114C102018
:10357000216802F0BDFF00289FD021684FF48050E1
:1035800002F0B6FF012898D106B0BDE8104002F065
:103590009FBE00BF249C00205C9B00209037020847
:1035A000489C002094360208DE8700207C37020801
:1035B00020610020209C002038B53A4D0120296868
:1035C00002F096FF50BB384C23783F2B10D029686F
:1035D000012002F08DFF002853D123784F2B2FD0EC
:1035E00023784F2B52D0BDE83840012002F058BE5E
:1035F0006378002BEBD12D4C2020216802F078FF5E
:10360000002831D02A4A2B4B1068127918601A71A1
:10361000BDE838402749284802F034BE234C10202A
:10362000216802F065FF0028CDD021684FF480505A
:1036300002F05EFF0128C6D1BDE8384002F048BE66
:1036400063784E2BCCD11D4B1B78002BC8D1174A69
:103650000121202002F052FF02F05AFFBDE838405D
:103660001749154802F00EBE2168202002F040FFE5
:103670000028CDD1134A0F4B1068928818609A80A9
:10368000C6E7BDE83840032002F00ABE6378462B47
:10369000A9D10A4B1A78462AA5D159780029A2D176
:1036A000024AD6E7249C00205C9B0020209C00203E
:1036B000A436020820610020DE8700205E9B0020E7
:1036C00094360208AC3602083E4B10B5196801204A
:1036D00002F00EFF30BB3C4B1A784F2A0AD01A7802
:1036E0004F2A31D01A783F2A44D0BDE8104001203B
:1036F00002F0D6BD5A784E2AF1D19A78002AEED13E
:10370000324933480123052202F016FD322005F02C
:103710009DFD304A0121102002F0F0FEBDE810406E
:1037200002F0F6BE2B4C1020216802F0E1FE0028CA
:10373000D1D021684FF4805002F0DAFE0128CAD1BE
:10374000BDE8104002F0C4BD5A78462ACAD1224AC8
:1037500011784629C6D151780029C3D110201D4ABD
:1037600002F0CCFE02F0D4FEBDE810401B49184820
:1037700002F088BD5B78002BB7D1164C1020216871
:1037800002F0B6FE50B92168102002F0B1FE88B1F7
:10379000BDE8104012490E4802F074BD114A104BAA
:1037A0001068127918601A71BDE810400C49084879
:1037B00002F068BD0C4A0A4B1068928818609A8023
:1037C000E6E700BF249C00205C9B002010690208F3
:1037D000DE870020209C00205E9B0020943602089B
:1037E00020610020A4360208AC36020870B5654D91
:1037F0000120296802F07CFE002840F0A280624B84
:103800001A783F2A04D0BDE87040012002F048BD7C
:103810005B78002BF7D12968012002F069FE04468D
:10382000003C29684FF0020018BF012402F060FE3E
:1038300008B144F002042968042002F059FE08B1DE
:1038400044F004042968082002F052FE08B144F054
:1038500008042968102002F04BFE08B144F010045F
:103860002968202002F044FE08B144F02004474EAD
:103870004FF40060316802F03BFE08B144F480442C
:1038800029684FF4007002F033FE08B144F400449C
:1038900031684FF4805002F02BFE08B144F48034BC
:1038A0003168022002F024FE08B144F4003431688B
:1038B000042002F01DFE08B144F4802429684FF46E
:1038C000007002F015FE002852D13168102002F07D
:1038D0000FFE08B144F480143168202002F008FE85
:1038E00008B144F4001431684FF4007002F000FE97
:1038F00008B144F480043168802002F0F9FD28B951
:1039000031684FF4807002F0F3FD38B131684FF444
:10391000807002F0EDFD40B344F0C07429684FF4AC
:10392000006002F0E5FD08B144F000741849194840
:1039300022461DF07DF8BDE870401649164802F099
:10394000A1BC124C1020216802F0D2FD00283FF4E7
:1039500056AF21684FF4805002F0CAFD01287FF471
:103960004EAFBDE8704002F0B3BC44F40004D5E7AC
:103970003168082002F0BCFD0028A6D044F40024E1
:10398000A3E700BF249C00205C9B0020209C00201B
:10399000A037020820610020DE87002038B51D4CCA
:1039A0000120216802F0A4FD28B11B4D10202968D8
:1039B00002F09EFD10BB21684FF4007002F098FDEC
:1039C000B8B1164B1A783F2A04D0BDE83840012020
:1039D00002F066BC5B78002BF7D10F4B10491A68D8
:1039E00010481DF025F8BDE838400E490E4802F099
:1039F00049BCBDE83840172002F052BC29684FF49A
:103A0000805002F075FD0128D5D1BDE8384002F0A4
:103A10005FBC00BF249C0020209C00205C9B0020F9
:103A2000A037020820610020DE87002038B5284C2E
:103A30000120216802F05CFD00BB264D2B783F2B56
:103A40000DD02168012002F053FD00283AD12B78D7
:103A5000432B25D0BDE83840012002F021BC6B7813
:103A6000002BEED11C4B1D491A681D481CF0E0FFCD
:103A7000BDE838401A491B4802F004BC1A4D10201A
:103A8000296802F035FD0028D7D029684FF480500E
:103A900002F02EFD0128D0D1BDE8384002F018BC5C
:103AA0006B784C2BD6D1114B1A78522AD2D15B7835
:103AB000002BCFD1084A0E4913600A48BDE83840B0
:103AC00002F0E0BBBDE83840062002F0E9BB00BFD1
:103AD000249C00205C9B0020289C0020A03702082A
:103AE00020610020DE870020209C00205E9B0020BB
:103AF0009436020870B53F4C0120216802F0F8FCB2
:103B000060BB3D4D3D492846FCF762FBD0B13C49C6
:103B10002846FCF75DFB002844D03A492846FCF7CC
:103B200057FB064600284CD02B783F2B23D019207A
:103B300002F0B6FBBDE870402E4A00214FF4007041
:103B400002F0DCBC224601214FF4007002F0D6FCEA
:103B5000BDE870402C492D4802F094BB2C4C4FF42A
:103B60008050216802F0C4FC012820D0BDE87040DC
:103B7000062002F095BB6B78002BD8D121684FF45A
:103B8000007002F0B5FC28B3224A234B106818607D
:103B900021491E4802F076FBBDE870401A491B48D7
:103BA00002F070BB224601214FF48050CEE721681D
:103BB000102002F09DFC0028D8D0BDE8704002F033
:103BC00087BB014622464FF4007002F097FC224664
:103BD0003146E9E721684FF4805002F089FC20B1BA
:103BE0000E4A0D4B10681860D2E70D4A0A4B106858
:103BF0001860CDE7249C00205C9B00200C62002014
:103C0000FC610020AC37020894360208DE870020F1
:103C1000209C0020B437020820610020B837020839
:103C2000BC37020870B5854C86B00023216801209E
:103C3000CDE9043302F05CFC00286CD1804B1A788B
:103C4000552A46D01A78532A7AD07E497C48FCF708
:103C5000BFFA002838D17C4B4FF48070196802F00D
:103C600047FC002840F0C380784B1A783F2A00F0C8
:103C7000C68021684FF4007002F03AFC00285BD047
:103C80002168012002F034FC0446002840F0B38093
:103C90006F496E4805AB04AA1CF0ECFE022813D154
:103CA000DDE904136B4A6C485370C3F3042343EA01
:103CB00041136A49137001220A60234622462146B5
:103CC000006810F0F7F802E0012002F0E9FA06B00F
:103CD00070BD5A78492AB5D19A78442AB2D1DA7897
:103CE000002AAFD1594B1A783F2AEDD15B78002BCF
:103CF000EAD15B4B5B4AD3E90001D2E90032CDE95E
:103D00000010594959481CF093FE5849584802F090
:103D1000B9FA06B070BD574D1020296802F0E8FBD3
:103D200000288BD029684FF4805002F0E1FB012875
:103D300084D102F0CDFACAE7172002F0B1FAC6E743
:103D40005B784E2B81D14C4B1B78002B7FF47DAFE1
:103D50003E4B1A783F2A38D021684FF4007002F0A9
:103D6000C7FB0028E8D02168012002F0C1FB002831
:103D700041D13648FCF736FA1428A5D83F4C3349D0
:103D80001025421C4FF47A7620461DF040F800942E
:103D900001232022A221CDE90156394807F0A8FAD3
:103DA0002C44322005F052FA01233022A221CDE921
:103DB00001560094324807F09BFA322005F046FA8B
:103DC00030492B4802F05EFA81E75B78002BC3D1C3
:103DD0002A4926481CF038FF2B4A24491488927837
:103DE000034623481C809A7002F04CFA6FE70820C3
:103DF00002F056FA6BE7032002F052FA67E75B78AD
:103E0000002B7FF436AF2168012002F071FB18B15E
:103E1000062002F045FA5AE70E4B1C491A785878EA
:103E2000130203F4F8530343520910481CF000FE38
:103E30000E490F4802F026FA49E700BF249C0020F3
:103E40005C9B0020383C0208289C00203C9B002002
:103E5000F0370208C8610020049C00208461002023
:103E6000CC610020D4610020C4370208206100200A
:103E7000DE870020209C00205E9B0020DC6100206B
:103E8000A09B00209436020840380208E43702085C
:103E900070B5914D88B02968012002F029FB0028F7
:103EA0004DD18E4C8E492046FCF792F9B8B98D4C15
:103EB00023783F2B34D16378002B31D18A498B484A
:103EC0001CF0C2FE8A4A89491488927803468948C0
:103ED0001C809A7008B0BDE8704002F0D3B98649E2
:103EE0002046FCF775F900283CD17E4B1A783F2A12
:103EF00040F08B805B78002B40F087807F4A8049C0
:103F0000D2E90040D2E90232CDE9000477481CF042
:103F10008FFD7649774808B0BDE8704002F0B2B92D
:103F20007048FCF75FF90F2803D82378002B40F086
:103F3000AD800A2008B0BDE8704002F0B1B9714C04
:103F40001020216802F0D4FA0028AAD021684FF48A
:103F5000805002F0CDFA0128A3D108B0BDE870402E
:103F600002F0B6B92378532B55D067495B48FCF76C
:103F70002FF9002849D15B4B1A783F2A00F0A28024
:103F800029684FF4007002F0B3FA002800F0938023
:103F900007AB002400935D495248079406AB05AA7D
:103FA000CDE905441CF066FD40B2032840F0908046
:103FB000059A069B079C56494C481F2A84BF01223C
:103FC00005920C2B84BF01230693632C88BF002429
:103FD000009488BF07941CF02BFD4E4B43491846B4
:103FE0001CF00DFF4FF47A7103461022CDE9012138
:103FF0000093A22148480123802207F079F947491C
:104000003C4802F03FF908B070BD012008B0BDE89F
:10401000704002F045B963784E2BA6D1A378002BEF
:10402000A3D1304B1A783F2A47D029684FF400704B
:1040300002F05EFA00283ED02A48FCF7D3F8142894
:10404000E3D8374C2749421C102520464FF47A7696
:104050001CF0DDFE01234022A2210094CDE901568F
:104060002D4807F045F92C44322005F0EFF8A22145
:1040700001235022CDE901562748009407F038F972
:10408000322005F0E3F825491A4823E7164B154975
:10409000421C18461CF0BBFE102203464FF47A71F6
:1040A000CDE901210093A2211B48012307F020F94B
:1040B0001A4910480EE717203CE75B78002BB4D173
:1040C0001749FCE65B78002B7FF45AAF1149F6E6FE
:1040D000012002F0E5F896E7249C00205C9B00207C
:1040E000F83702083C9B00208861002020610020F6
:1040F00040380208DE87002000380208986100205E
:1041000008380208209C0020203802089037020856
:104110002838020870610020A09B00209436020815
:10412000A861002030B5484C85B02168012002F01C
:10413000DFF930B1454D1020296802F0D9F9002887
:1041400051D121684FF4007002F0D2F948B3404DCC
:104150002B783F2B0DD03F493D48FCF739F830B361
:104160002B78432B4BD0012005B0BDE8304002F046
:1041700097B86B78002BEED12168802002F0B8F957
:10418000002854D0344A354B1068918892791860D1
:1041900099809A713149324805B0BDE8304002F04B
:1041A00071B8172005B0BDE8304002F079B82D4A4B
:1041B0002D4B92E803004FF47A7483E80300082241
:1041C0002A480294CDE90032A2210123702207F08F
:1041D0008FF8322005F03AF82549214805B0BDE8AE
:1041E000304002F04FB829684FF4805002F080F957
:1041F0000128A6D105B0BDE8304002F069B86B785F
:104200004C2BB0D11B4B1A78522AACD158780028CD
:10421000A9D1154C009408234FF47A72CDE90132EC
:10422000A221C4E90000012310487022CFE72168D1
:10423000802002F05DF90028ACD10F4B074A03CB78
:1042400010605160A6E700BF249C0020209C002045
:104250005C9B00204C3802083C380208206100209A
:10426000DE870020D4610020CC610020A09B0020CC
:10427000943602085E9B00204438020870B5524E06
:10428000524C316882B0012002F032F930B121681D
:10429000102002F02DF9002840F0828021684FF4B0
:1042A000805002F025F9002874D0494D2B783F2B1F
:1042B00031D02A78474B995C490765D569785B5CB2
:1042C0005B0761D5302A0CBF002101213F4A042041
:1042D00002F014F96B783D4A302B0CBF002101210C
:1042E000022002F00BF931684FF4007002F000F97F
:1042F00040B1AB78354A302B0CBF0021012108209A
:1043000002F0FCF83449354801F0BCFF02B0BDE8CA
:10431000704002F0FDB86B78002BCAD121680420F0
:1043200002F0E6F821680546022002F0E1F82A468C
:1043300003462B492B481CF07BFB31684FF400707F
:1043400002F0D6F80246002837D02168082002F093
:10435000CFF86C460246244920461CF069FB2146F2
:1043600020481CF02AFC214B1E481B68ADF8003089
:104370001A0C21468DF802201CF01FFC1949174821
:1043800001F080FF02B070BD012002B0BDE87040B6
:1043900001F086BF052002B0BDE8704001F080BF8B
:1043A00021684FF4805002F0A3F801287FF476AF23
:1043B00002B0BDE8704001F08BBF6C460C4920464E
:1043C0001CF036FBCBE700BF249C0020209C002083
:1043D0005C9B00209971020894360208DE87002059
:1043E00054380208206100205C3802084038020876
:1043F0006038020838B52F4D0120296802F078F89E
:1044000008BB2D4C2D492046FBF7E2FE68B323780C
:10441000452B0DD029684FF4007002F069F810B1F7
:104420002378412B3AD0BDE83840012001F038BF55
:104430006378582BEED1A378542BEBD1E378002B83
:10444000E8D11F4B12E01F4C1020216802F050F8F9
:104450000028D6D021684FF4805002F049F8012896
:10446000CFD1BDE8384001F033BF174B174C93ED67
:10447000000A012203234021204601F02FFC2046A0
:10448000FBF7B0FE124B0219198821529B789370EA
:1044900021461048BDE8384001F0F4BE6378442B53
:1044A000C1D10D4B1A78432ABDD15B78002BBAD10C
:1044B0000A4BDBE7249C00205C9B00206438020848
:1044C00008000020209C00200C000020206100201B
:1044D00040380208DE8700205E9B0020100000208C
:1044E00038B53B4C0120216802F002F8002830D199
:1044F000384D2B783F2B13D02168012001F0F8FFB5
:10450000002860D134493348FBF762FE002832D0DE
:104510002B784F2B3DD0BDE83840012001F0C0BEC4
:104520006B78002BE8D12D4C4FF48050216801F0BE
:10453000DFFF002839D02A4A2A4B106891889279E7
:10454000186099809A71BDE838402649264801F0E4
:1045500099BE224D1020296801F0CAFF0028C7D05B
:1045600029684FF4805001F0C3FF0128C0D1BDE895
:10457000384001F0ADBE194A01214FF4805001F0DE
:10458000BDFF01F0C5FFBDE838401849164801F0ED
:1045900079BE6B78532BBED1154B1A78432ABAD10A
:1045A00059780029B7D10D4AE7E721684FF48050C8
:1045B00001F09EFF0028C6D10E4A0A4B106892886F
:1045C00018609A80BFE7BDE83840032001F068BE5C
:1045D000249C00205C9B002084380208209C002042
:1045E0007438020820610020DE870020943602081B
:1045F0005E9B00207C38020810B51B4C012021680E
:1046000001F076FF216820B1012001F071FFA0B90F
:1046100010BD4FF4007001F06BFF20B9BDE81040F1
:10462000172001F03DBE02F0A7F801F08BFFBDE8B6
:1046300010400E490E4801F025BE0E4C4FF480503C
:10464000216801F055FF012804D0BDE81040062084
:1046500001F026BE2168102001F04AFF0028F4D0A6
:10466000BDE8104001F034BE249C002094360208BE
:10467000DE870020209C0020194B10B5196801200E
:1046800001F036FFA8B917491748FBF7A1FD58B943
:104690001649174801F0F6FD4FF47A7004F0D6FD84
:1046A000BDE8104005F086B8BDE81040012001F0DB
:1046B000F7BD104C4FF48050216801F019FF01281C
:1046C00004D0BDE81040062001F0EABD21681020AA
:1046D00001F00EFF0028F4D0BDE8104001F0F8BD55
:1046E000249C00204C3802085C9B00209436020871
:1046F000DE870020209C0020F0B5554C87B0216853
:10470000012001F0F5FE216830B1012001F0F0FE3A
:10471000002840D107B0F0BD4FF4007001F0E8FE72
:10472000002867D04B4C23783F2B69D049480A2298
:1047300005A91CF069F8059EA642054655D03378B8
:104740002E2B36D0002B50D1FE284ED8FF20424BC6
:10475000424E0124CDE900341D704FF47A7530705B
:104760002346FF22A02102953D4806F0C1FD3220DC
:1047700004F06CFDFE222346A021CDE90145009600
:10478000374806F0B5FD322004F060FD3549364863
:1047900001F078FDBEE7354C4FF48050216801F000
:1047A000A7FE012845D0062007B0BDE8F04001F083
:1047B00077BD771C0A22384605A91CF025F8059B11
:1047C000DF1B7A1E012A10D87278A2F13001092964
:1047D0000BD8022F38D0A34207D01B782BB9FE2D5F
:1047E00003D8FF28B2D06328B1D9012001F058FDC9
:1047F00007B0F0BD172007B0BDE8F04001F050BD94
:104800006378002B92D1154B134A1B781278FF2B3B
:104810000AD0174917481CF00BF91649124807B07F
:10482000BDE8F04001F02EBD134912481CF000F91C
:10483000F3E72168102001F05BFE0028B3D007B039
:10484000BDE8F04001F044BD302AC4D1CDE700BF3F
:10485000249C00205C9B002081610020806100205E
:10486000A09B002094360208DE870020209C0020B8
:104870009038020820610020543A02082DE9F041E6
:10488000AF4C82B0002321680193012001F030FE7B
:10489000002878D1AB4D2B783F2B5FD021680120C9
:1048A00001F026FE002840F0C380A749A548FBF789
:1048B0008FFC00287AD0A549A248FBF789FC064660
:1048C000002800F09C802B78522B00F0BB802B78C6
:1048D0004C2B00F01E812B78522B00F063819C49F9
:1048E0009848FBF775FC002800F0FF80994995482F
:1048F000FBF76EFC002840F06D8197499748984F70
:1049000001220EF045F83870002840F08081954D66
:10491000DFF84882944E01AB4FF48072294640463E
:104920000EF0E2F93870019A01232946304601F071
:1049300003FC0446052010F04BFB002CF3D1019B37
:10494000B3F5807FE7D0884C84480EF0BFFC8749E0
:10495000204601F097FC0023237011E06B78002BB8
:104960009CD12168202001F0C3FD002852D0804B4B
:10497000804A03CB106051607E497B4801F082FC85
:1049800002B0BDE8F0817C4D4FF48050296801F001
:10499000AFFD01287FF47EAF2968102001F0A8FD4B
:1049A00000283FF477AF01F093FCE9E7216820206D
:1049B00001F09EFD0446002840D1704B024693E86A
:1049C000030002F0B7F9C82004F040FC03F018FB24
:1049D0006B496C4801220DF081FF614B1870002873
:1049E00065D001210846684A01F088FD544A20201C
:1049F000214601F083FD122001F052FCC0E721683E
:104A0000202001F075FD012804465AD01C2001F039
:104A100047FCB5E72168202001F06AFD0028ABD1F2
:104A20005A4B544A03CB1B88106051601381A3E793
:104A3000062001F035FC02B0BDE8F0811B2001F03A
:104A40002FFC9DE76B78532B7FF441AF504B1A78C6
:104A5000542A7FF43CAF5C78002C7FF438AF2146B9
:104A6000374A464D202001F049FD22464449204660
:104A70000DF034FF474808F047FA464803F086FB3C
:104A8000454B95E8030001221C7002F053F9C82041
:104A900004F0DCFB95E80300224602F04BF9C82045
:104AA00004F0D4FB3149304801F0ECFB68E7244ABC
:104AB0000121202001F022FD2C492B4801F0E2FBCE
:104AC0005EE72F49324630460DF008FF244B014681
:104AD0001870002800F0828020462B4A214601F001
:104AE0000DFD132001F0DCFB4AE71C4C1A490122A2
:104AF00020460DF04DFF1A4B187000287ED120463D
:104B0000E4680EF0E3FB25491A4822461BF090FFAB
:104B100032E76B78532B7FF4DEAE1D4B1B78002BF6
:104B20007FF4D9AE1E4801F09DFC0D4B1870002893
:104B30004BD0112001F0B4FB194B00221A701FE773
:104B4000249C00205C9B0020AC380208B43802088A
:104B5000C8380208D03802083C9B0020748300202B
:104B6000708300203C620020DE870020943602081B
:104B70009838020820610020209C0020306902083B
:104B800048370208A4850020289C0020A03802088D
:104B90005E9B0020409D0020D4EC0020303A0208AB
:104BA0003C6300206B784D2B7FF499AE1C4B1B7837
:104BB000002B7FF494AE1B480EF0BAFC1A4B187011
:104BC000B8B1142001F06CFBDAE61849184801F07E
:104BD00059FBB1E7012001F063FBD1E6154B164A02
:104BE0001970202001F08AFC1049114801F04AFB9D
:104BF000C6E60E490E4801F045FBC1E60F4A012109
:104C0000022001F07BFC152001F04AFBB8E60B4ABC
:104C10000121022001F072FC162001F041FB92E616
:104C20005E9B00203C9B002070830020943602088D
:104C3000DE870020D4EC0020249C0020289C00204B
:104C400030B53B4C85B02168012001F051FC0028B3
:104C500052D1384D2B783F2B3BD02168012001F0F9
:104C600047FC00285BD12B78334AD35C5B072AD5FD
:104C700030481AF0FAFE314BA0F10A029A4254D899
:104C800003F1CC532E4A2F4903F5252303F2627317
:104C900002FB0033B1EB730F15D92B4C0094A2FB30
:104CA000002004234FF47A72C008CDE90132A0211C
:104CB00001231C222060254806F01AFB322004F054
:104CC000C5FA234912E0012005B0BDE8304001F0EB
:104CD000E7BA6B78002BC0D11B4B1E491A681E48DF
:104CE00002EB820252001BF0A3FE1B491B4805B0D9
:104CF000BDE8304001F0C6BA194D1020296801F016
:104D0000F7FB0028A5D029684FF4805001F0F0FB94
:104D100001289ED105B0BDE8304001F0D9BA03208A
:104D200005B0BDE8304001F0BBBA0220CCE700BFBF
:104D3000249C00205C9B00209971020836420F00E1
:104D4000CDCCCCCC9999991948630020A09B002028
:104D500094360208303A020820610020DE870020E5
:104D6000209C002000000000F0B52DED028B504883
:104D7000504E85B01AF076FE3168012055EC104B8C
:104D800001F0B6FB002848D1494B1A783F2A26D0BB
:104D90003168012001F0ACFB002867D1294620468C
:104DA000FBF7F4FE08EE100AFBF7DEFB3EA3D3E9A7
:104DB000002304460D46FBF7B5FEF2EE047AB4EE8E
:104DC000E78A00283ED0F1EE10FA57D946DC0120E0
:104DD00005B0BDEC028BBDE8F04001F061BA5B7834
:104DE000002BD5D1344C354A402192ED000A2046A3
:104DF000012200F073FF2046FBF7F4F9304B021953
:104E0000198821529B782F489370214605B0BDEC3C
:104E1000028BBDE8F04001F035BA2B4F1020396805
:104E200001F066FB0028AFD039684FF4805001F0E4
:104E30005FFB0128A8D105B0BDEC028BBDE8F040B6
:104E400001F046BAF1EE10FA08DC17A3D3E900230B
:104E500020462946FBF752FE0028B8D0022005B0B4
:104E6000BDEC028BBDE8F04001F01ABA032005B09A
:104E7000BDEC028BBDE8F04001F012BA0F4C00947B
:104E800004234FF47A72CDE90132A02101230822D4
:104E90000E4884ED008A06F02BFA322004F0D6F991
:104EA0000B490848B2E700BF9A9999999999B93F77
:104EB0005C9B0020249C0020206100204063002097
:104EC00040380208DE870020209C0020A09B0020A4
:104ED0009436020870B5AD4C84B02168012001F011
:104EE00007FB002840F09F80A94D2B783F2B00F056
:104EF0008180A849A648FBF76BF9002840D1A64D50
:104F00002B783F2B00F0C1802168012001F0F0FADE
:104F1000002840F09D802B78A04AD25C510702D433
:104F20002D2B40F0A0809C481AF09CFD51EC100BFA
:104F3000FBF72CFE9FED9A7A07EE900AF4EEC77A03
:104F4000F1EE10FA00F191809FED967AF4EEC77AB7
:104F5000F1EE10FA00F3898004234FF47A72924C38
:104F600092480094CDE9013201230C22A021C4ED26
:104F7000007A06F0BDF9322004F068F98C494CE063
:104F80008C498348FBF724F9002840F09780824D34
:104F90002B783F2B62D02168012001F0A9FA00286C
:104FA00056D12B787D4AD25C520701D42D2B5AD191
:104FB00079481AF057FD51EC100BFBF7E7FD9FED18
:104FC000787A07EE900AF4EEC77AF1EE10FA4CD434
:104FD0009FED747AF4EEC77AF1EE10FA45DC042303
:104FE0004FF47A72744C71480094CDE90132012378
:104FF0001022BBE76B78002B7FF47BAF6F4C4FF434
:105000000070216801F074FA002830D06C4A6D4BB2
:105010001068127918601A716A496B4804B0BDE8CB
:10502000704001F02FB9654D1020296801F060FA39
:1050300000283FF459AF29684FF4805001F058FA26
:1050400001287FF451AF04B0BDE8704001F040B9D1
:10505000032004B0BDE8704001F022B96B78002B4A
:1050600099D1554A16E00120F3E70220F1E72168C3
:105070004FF4007001F03CFA0028CDD1534A514B57
:105080001068928818609A80C6E76B78002B7FF4CE
:105090003BAF454A4B4C92ED000A40210622204688
:1050A00000F01CFE2046FBF79DF8494B02191988B9
:1050B0009B782152444893702146AFE72168012034
:1050C00001F016FA0028C3D12B784F2B24D02B786F
:1050D0004F2B3CD02B78432BC5D16B784C2BC2D1B6
:1050E0003C4B1A78522ABED15D78002DBBD13A4B89
:1050F0002A4693E8030001F01DFE04202946234AB6
:1051000001F0FCF92168042001F0F2F9002830D008
:10511000324B00221A7031E76B784E2BD7D12D4BD2
:105120001E78002ED3D12C4B324693E8030001F0B9
:1051300001FE3146154A042001F0E0F91F4A012121
:105140004FF4007001F0DAF901F0E2F916E76B783C
:10515000462BBFD11F4B1A78462ABBD1597800295C
:10516000B8D1164A4FF4007001F0C8F901F0D0F937
:1051700004E7124B4FF40070196801F0B9F90028E8
:10518000C6D0164B01221A70F8E600BF249C0020FE
:105190005C9B0020D83802083C9B002099710208D3
:1051A000000096C400009644F4600020A09B0020FC
:1051B00094360208E038020800000020209C0020FD
:1051C000A436020820610020DE870020AC360208E9
:1051D000403802085E9B0020286902081561002003
:1051E00070B53448344C84B01AF03FFC2168054651
:1051F000012001F07DF900283DD12E4B1A783F2A7D
:1052000029D02168012001F073F900284CD16B1ED0
:10521000632B43D8012D294C274A256014BF014632
:1052200029464FF4806001F069F94FF47A72042343
:10523000CDE90132A021012346220094204806F046
:1052400057F8322004F002F81E491F4804B0BDE8A8
:10525000704001F017B85B78002BD2D1174B1B4977
:105260001A681B481BF0E4FB1949174804B0BDE855
:10527000704001F007B8174E1020316801F038F97E
:105280000028BAD031684FF4805001F031F901287C
:10529000B3D104B0BDE8704001F01AB8022004B0E8
:1052A000BDE8704000F0FCBF032004B0BDE87040D2
:1052B00000F0F6BF5C9B0020249C0020446300208B
:1052C000A09B002094360208DE870020303A0208B6
:1052D00020610020209C002080B54FF4FA600FF080
:1052E00077FE544B93E8030001F038FD002847D1C6
:1052F000514904465148FAF76BFF514A002800F023
:1053000093802146802001F0F9F84E4A01214FF4A4
:10531000003001F0F3F84C4A01214FF4805001F0C5
:10532000EDF8494A0021102001F0E8F8464A002132
:10533000202001F0E3F8444A0021802001F0DEF84B
:10534000414A00214FF4807001F0D8F83E4A002114
:105350004FF4007001F0D2F83C483D4B384A4FF012
:105360007E54012104604FF48060196001F0C6F89A
:10537000384A394B1188927819809A70FCF77CFC76
:105380002F4DDFF8DC80354E2E4FDFF8ACA0DFF874
:10539000AC9014E00021402001F0B0F8294A01212E
:1053A0004FF4807001F0AAF839682A4669B30121E8
:1053B000022001F0A3F84FF4FA700FF009FE2968FB
:1053C000012001F095F8044680B9D8F800306BB19F
:1053D0000822514648461BF0BEFB2A46C8B90121A7
:1053E000802001F08BF80023C8F8003096E8030015
:1053F00001F0B4FC2A460028CCD10121402001F064
:105400007DF839682A460029D1D1022001F076F8CA
:10541000D1E72146802001F071F80A4A01214FF4BA
:10542000003001F06BF8DEE70121802001F066F822
:1054300071E700BF20690208CC610020D461002020
:10544000249C0020289C0020209C002040630020F9
:10545000446300209C3602085C9B00201869020807
:10546000349C0020000000002DE9F0472DED028B58
:105470008CB0002207A93E48DFF80C81DFF80CA1B0
:105480003C4C9FED3D8ADFED3D8A394D07F054FAE3
:105490003748002201A907F08BFA33A7D7E9006744
:1054A0004FF00009204603F08FFF4FF0FF312046F8
:1054B00004F00EF8204604F063F807EE900AF8EEC8
:1054C000677A17EE900AFBF74FF832463B46FBF738
:1054D000A3F800222A4BFAF7E7FEFBF757FB034637
:1054E0004FF47A70C8F800300FF072FD002202A964
:1054F000284607F021FA002201A9284607F058FAA9
:105500009DF81CC09DF808309DF81DE01D4AA3EBD6
:105510000C039DF809C0C3EB0313ACEB0E0C0CEBB2
:10552000830300214FF40060CAF80030B9F1000F86
:1055300001D11E2BB6DDD8ED007AF4EEC87AF1EE7B
:1055400010FA04D4F4EEE87AF1EE10FA04DD00F07B
:10555000D5FF4FF00109A5E70A4A01214FF4006089
:1055600000F0CCFFF5E700BF08AC1C5A643BAF3F2E
:10557000489C00209006002000005C42000082420F
:1055800000004940249C00201000002050630020AF
:105590000B4C08B5206800210EF014FF4FF0E026F8
:1055A0004FF080554FF0FF3120680EF00BFF00F0F8
:1055B000AFFEC6F8045DBFF34F8FBFF36F8FF1E707
:1055C0001C9C002080B5144D144F2868144C154EB7
:1055D00084B000210EF0F6FE28684FF0FF310EF087
:1055E000F1FE97ED000A002307221021684600F023
:1055F00075FB6846FAF7F6FD03460DEB000EB4F8AE
:1056000000C0A2782DF803C0694630468EF802200B
:1056100000F038FEE0E700BF109C0020F86000209A
:1056200040380208DE8700202DE9F04FB54EB6481D
:10563000B64DB74CB74FDFF8E882DFF824B3DFF898
:105640002493A3B0402220211BF0AFFA3068002140
:105650000EF0B8FE4FF0FF3130680EF0B3FE95F853
:1056600000A021684FF4805000F042FF5FFA8AFAF0
:10567000216888BB102000F03BFF0028EAD098F892
:105680000020A548032AA54A0AF1FF3A12684FF400
:10569000B4630AF00F0A03FB0A714FF001030360C1
:1056A0004FEAC2020CBF9E48484600F045FD8BF809
:1056B00000000028CED0964A0021102000F01EFFE6
:1056C000984A01214FF4803000F018FF002389F838
:1056D000003088F80030BDE74FF4805000F008FF3C
:1056E0000128B7D12B78013B4FF4B46A03F00F03C4
:1056F0000AFB037393ED010A07220023202109A866
:1057000000F0ECFA09AB00932B788749013B03F0DA
:105710000F030AFB03F311A8FA582B78013B03F09F
:105720000F030AFB037322F07F42DB781BF080F942
:105730002168042000F0DCFE0128824600F0B480DD
:105740002168022000F0D4FE0128824600F09780F4
:10575000764B4FF40070196800F0CAFE002872D131
:1057600011A8FAF73FFD11AB824603447048216847
:1057700002880DF1440C2CF80A2082789A701020CF
:105780000AF10203039300F0B3FE002842D121681E
:10579000202000F0ADFE00283FF45CAF039B11A970
:1057A00003F0030242F2200321F80A30C2F104029E
:1057B000554911A81BF010FA11A8FAF713FD5D4B1B
:1057C000821E824611A840F60D211B6881525A4A5A
:1057D0001068002B7DD0012B00F08A80B0F57C6F23
:1057E0007FF638AF534A83F001031360524A002317
:1057F0001360524A194610681A460EF05BFB4FF0D0
:10580000E0234FF08052C3F8042DBFF34F8FBFF356
:105810006F8F1FE7039A012311A9484600F08CFC03
:105820008BF800000028B2D0394A0021102000F087
:1058300065FE3C4A01214FF4803000F05FFE0023FA
:1058400089F80030A3E72168082000F051FE012804
:10585000824685D111A8FAF7C5FC394B93ED000AB1
:10586000384B11A91B880B52524605A80023102162
:1058700000F034FA05A911A81BF09FF970E711A8F0
:10588000FAF7B0FC304B93ED000A2E4B11A91B88A0
:105890000B52524605A80023102100F01FFA05A95B
:1058A00011A81BF08AF953E711A8FAF79BFC274BC4
:1058B00093ED000A234B11A91B880B52524605A8F1
:1058C0000023102100F00AFA05A911A81BF075F9B0
:1058D00036E703931E4B5246184411A91BF097FA62
:1058E0001C4B186850441860134B1860039B75E7F5
:1058F0000393194B5246184411A91BF088FA174B11
:10590000EFE700BF149C002014000020E46000209A
:10591000209C0020D80600204C630020DC60002082
:10592000DD870020289C0020E8380208249C002005
:10593000403802086C630020686300200C9C002043
:1059400010000020F4380208080000200C0000209D
:105950007073002064630020706300206063002087
:10596000DC870020DE8700202DE98048DFF8F88002
:10597000374FD8F80000374CDFF8F090364EDFF89C
:10598000F0B0364DDFF8ECA083B000210EF01AFD28
:1059900016E052460021202000F0B0FD304A0121DF
:1059A000042000F0ABFD28460DF090FC307078BB71
:1059B0002C4A0021102000F0A1FD236800221A606B
:1059C0004FF0FF31D8F800000EF0FCFC00F07AFA3E
:1059D0002368D9F800101A6828463B460DF0B6FA3D
:1059E000014630700028D4D123683A681868904284
:1059F00014D05246202000F081FD194A01212020B8
:105A000000F07CFD28460DF061FC30700028CFD0FE
:105A1000134A0121102000F071FDC9E7DBF80020D6
:105A2000092A03D80132CBF80020C7E72846CBF873
:105A3000001001910DF0CEFB019930700028BCD010
:105A40005246202000F05AFD054A01210820A8E70F
:105A5000546300205863002070830020748300206A
:105A6000289C0020249C00200C9C00205C630020CB
:105A7000E0870020209C002010B582B000240F4B4E
:105A80000194196B41F4800119631B6B03F48003CB
:105A90002246062101933B20019B03F02FFE3B2071
:105AA00003F068FE22460621452003F027FE45202C
:105AB00002B0BDE8104003F05DBE00BF00380240F8
:105AC0000F4A104BD2F8FC1021F08071C2F8FC1084
:105AD000D2F8FC1041F08071C2F8FC101A6822F074
:105AE00001021A601A68002042F001021A60586030
:105AF00000BF00BF00BF5868B0FA80F0400970478F
:105B000000ED00E0001000E030B5002483B0012576
:105B10000AF050F819F08EFCCDE9005423463B49B9
:105B20003B484FF480720EF093FFCDE900542346BA
:105B3000384939484FF480720EF08AFF0223CDE9CC
:105B400000343649364823464FF400720EF080FF89
:105B5000344B35493548CDE900534FF4C0722346E4
:105B60000EF076FFCDE900542346314931484FF419
:105B700020720EF06DFF0323CDE900340425234687
:105B80002D492E484FF4A0620EF062FFCDE900547B
:105B900023462B492B484FF4A0620EF059FFCDE964
:105BA000005423460625284928484FF400720EF079
:105BB0004FFF2346CDE90054254926484FF4F062B3
:105BC0000EF046FF0723CDE900342349234823463E
:105BD0004FF400620EF03CFF0823CDE90034204969
:105BE000204823464FF400620EF032FFCDE9005406
:105BF0001D491E4823464FF400720EF029FF20462F
:105C000003B0BDE830400EF053BF00BFF8380208C3
:105C1000F1730008003902086954000810390208BD
:105C2000D9520008009C002020390208B57A0008EB
:105C30002C3902089D6F000834390208915500087C
:105C400040390208695900084C390208C555000856
:105C50005C390208295600086C390208ED8B0008EF
:105C60007839020871850008843902082D8A0008F5
:105C7000704700BF014B586A704700BF000C0040DE
:105C8000704700BF704700BFFEE700BFFEE700BFE0
:105C9000044B10B40360044C0C6080235DF8044B8B
:105CA00013607047E4890020E487002010B5094C98
:105CB0000FCC88B00DF1040CACE80F0094E807009D
:105CC0008CE80700002101A80DF078FD024B186058
:105CD00008B010BDE03502088C8A0020072AB5EE16
:105CE000C00AF0B5174628BF0727F1EE10FA4CBFDF
:105CF000F1EE407AF0EE407ABDEEE77A8BB0F8EE46
:105D0000C76A064677EEE67A0D461C46002A6BD037
:105D10004FF0000C01220CF1010C5FFA8CFE02EB3B
:105D2000820277454FEA4202F5D806EE902AF8EE55
:105D3000666A67EEA67AF6EE006A77EEA67AFCEE61
:105D4000E77A17EE903A934205D317EE103A0133F3
:105D500007EE103A0023B5EEC00AF1EE10FA0097F4
:105D600002AF4CBF224A234A0193202117EE103A7A
:105D700038461AF027FE84422CD9012D9DF80830B0
:105D800024D9721E1444A919241A02394FF0200C88
:105D900001E08A4204D0104602F801CFA242F8D1B5
:105DA000C6F102020244B11803B3501C85421DD94A
:105DB000013A324402E0A94207D2084602F8013F04
:105DC00017F8013F411C002BF5D106440023337026
:105DD0000BB0F0BD013D2A46394630461AF021FF8E
:105DE000002373550BB0F0BD0122A4E70E46EDE78A
:105DF000A0390208AC390208274B284A1B68D2EDAB
:105E0000007A1B05F8EE677A21D52549254A264BED
:105E100092ED006AD3ED006A91ED007A2349244B9C
:105E2000244AB8EE477A27EE866A67EEA66A26EE1F
:105E3000076A66EE876A91ED007AC3ED006A27EE85
:105E4000877A1D4B82ED006A83ED007A70471B4B09
:105E50001B78ABB1124B1549D3ED006A91ED007A76
:105E6000134B144AF8EE666A27EE877A66EEA76A45
:105E7000C3ED006A104BC2ED006A83ED007A7047F3
:105E80000B4B0C4AC3ED007A9FED0D7A0A4BC2ED25
:105E9000007A83ED007A7047209C002004000020E7
:105EA0004463002068610020646100206C61002070
:105EB000E8600020EC600020F060002060610020BD
:105EC00000000000094B1B6833B90949094B0A4817
:105ED0000A4A08601A607047012B00D070470449D5
:105EE000044B0748074A08601A6070476C6300203B
:105EF0005C63002058630020706300206063002012
:105F0000707300206463002070B5154E8EB00D468E
:105F1000044609A90022304606F00EFD08A9002219
:105F2000304606F045FD0F4A9DF8261006929DF872
:105F300025200D4BCDE904219DF824109DF8222049
:105F4000CDE902219DF821109DF823202046CDE9BE
:105F50000021064A29461AF035FD0EB070BD00BF7B
:105F6000489C0020D839020888610020B83902080E
:105F70002DE9F041474E484C484F494D82B03146DB
:105F80000022204606F0D8FC2046464C3946002226
:105F900006F00EFD4FF00008434A444985F80080A2
:105FA00020461AF045FD214628461AF006FEBB7829
:105FB00000937B78FA783E4920461AF039FD214655
:105FC00028461AF0FAFDB37800937378327839498D
:105FD00020461AF02DFD2846FAF704F921462844F8
:105FE0001AF032FE3449024608681060334890EDDA
:105FF000000A888889799080434691712046012261
:106000004FF48051FFF76AFE2046FAF7EBF82C4A6E
:1060100003461E191068E0509388B3802146284635
:106020001AF0CBFD274B28491A6820461AF000FDCC
:10603000214628461AF0C1FD244B25491A681B68E1
:10604000C2F34002C3F3800320461AF0F1FC21465C
:1060500028461AF0B2FD1F4B186820609B88A38069
:106060002846FAF7BFF8214628441AF0EDFD421BF6
:1060700002F003021849C2F1080228461AF0ACFDEA
:106080002846FAF7AFF8023840F60D232B5202B03B
:10609000BDE8F0816C9C0020489C0020689C00209A
:1060A000706300207073002088610020DC390208D2
:1060B000E8390208003A0208183A02084063002052
:1060C000203A020844630020283A0208209C00205D
:1060D000383A0208483A020814000020074B4FF4EF
:1060E000FA601B68B0FBF3F0B42804D8B3F5FA6F7C
:1060F00088BF01207047B420704700BF0400002013
:106100009FED0B7AC7EE007A10B50A4C2368002287
:106110005A622046FCEEE77A17EE903A013BE360C4
:1061200007F0C6FF2046BDE8104007F0B1BD00BF34
:10613000A037A04CB89E00202DE9F043484F1D46E3
:106140003B6883B00446164653B3DFF83081C8F885
:1061500000102378012B2CD02378022B43D02378F6
:10616000032B62D02378042B34D005B925703B680B
:1061700083B9D8F800303B493B4833445A1AB2F54A
:10618000606F88BF0B460260C8F80030002003B083
:10619000BDE8F083002000233B6003B0BDE8F0833E
:1061A000DFF8D880D8F800001AF031FE2378012BF0
:1061B000D2D1D8F80000B1B219F062FA05B9257051
:1061C0003B682BB90028D4D0C0B203B0BDE8F0833F
:1061D000C0B2E0E7D8F800102448B2B208F0DAF80C
:1061E000002DEDD1EBE7DFF89890D8F80020009271
:1061F0000023D9F8000001961A4669460DF05AFEB0
:106200000128B2D0642003F021F8D9F80000002161
:106210000DF04CFD164B93F82D305A071AD505B9E1
:1062200025703B68D3B90120B1E7124BD8F80020A4
:106230001868009200231A46694601960DF03AFE4E
:10624000012892D0642003F001F8094B93F82D3017
:106250005B07E4D4084B01221A60E0E701209AE7CB
:106260004C630020DC8A0020908A0020609F002080
:1062700064A00020FC9B0020988A0020540000208D
:10628000089C002070B5054608460C46F9F7AAFFA1
:106290002146024600232846BDE87040FFF74CBF68
:1062A00010B5084C0849024620461AF0C1FB2046AA
:1062B000F9F798FF21460246BDE810400348002345
:1062C000FFF73ABF20610020503A0208DE87002025
:1062D0000B480C49036810B50B4C23F01003036006
:1062E000042220461AF0A4FB2046F9F77BFF214642
:1062F0000246BDE8104005480023FFF71DBF00BF60
:10630000209C0020503A020820610020DE870020F7
:10631000F0B583B0424D434B434A4449444800954D
:106320001AF0A8FB02283ED0032829D001280BD15F
:10633000404A41493C481AF09DFB4049404A0023ED
:1063400001280B70137040D03E4B1B68D80706D550
:106350003D4B1A68D10402D51A68D20652D43B4983
:106360003B4800221AF064FB3948F9F73BFF3849F3
:1063700002463848002303B0BDE8F040FFF7DCBE1A
:106380002C4A2D4928481AF075FB2C4A2A49044604
:1063900024481AF06FFB0128294A2F49284639D092
:1063A0001AF068FBD0E7234A23491F481AF062FB22
:1063B000224A214904461B481AF05CFB204B00226C
:1063C00001281A70C0D1012CBED1244F3968002990
:1063D000BAD0184E3D46002404E055F8141F01348D
:1063E0000029B1D03046F9F7F3FE0028F5D104EBCF
:1063F000840407EB84071A4A7B68136003B0BDE886
:10640000F04018471C681149114824F01004042278
:106410001C60A7E71AF02EFB012895D1D3E700BF37
:10642000DC9A0020FC9A00201C9B00205C3A0208A9
:106430009C8A00207C9B0020743A02085C9B002010
:106440003C9B0020249C0020209C0020503A020805
:1064500020610020DE870020783A020858000020E2
:10646000F49B0020F0B5A5B0014601A80CF062FF36
:10647000002832D11B4F1C4D1C4E0EA901A80DF057
:1064800001F8044618BB9DF84E4004B32E2CF4D0FE
:106490009DF84030DB06F0D40DF14E023946284617
:1064A0001AF0C6FA2846F9F79DFE0123024629464E
:1064B0003046FFF741FE0028F4D1142002F0C6FE5A
:1064C0000EA901A80CF0DEFF04460028DBD001A8CD
:1064D0000CF0AAFF204625B0F0BD0446204625B0AA
:1064E000F0BD00BF3037020820610020DE870020A9
:1064F000014214BF01200020704700BF136819B982
:1065000023EA00031360704703431360704700BF22
:1065100000B585B0094B00934FF47A710422CDE9A0
:10652000012101230022A021054804F0E1FE3220D0
:1065300005B05DF804EB02F089BE00BF209C00208E
:10654000A09B00202DE9F041744C754B84B04FF4B2
:106550007A750426CDE90165009300220123A0216C
:10656000204604F061FF6F4A0092CDE901650123E6
:106570000822A021204604F057FF6B4A0092CDE983
:10658000016501231022A021204604F04DFF674A37
:106590000092CDE9016501230C22A021204604F0E0
:1065A00043FF634A0092CDE9016501231C22A0212B
:1065B000204604F039FF5F4A0092CDE901650123CE
:1065C0002822A021204604F02FFF5B4A0092CDE94B
:1065D000016501234622A021204604F025FF574AE9
:1065E0000092CDE9016501234A22A021204604F052
:1065F0001BFF534A0092CDE9016501235022A021DF
:10660000204604F011FF4F4A0092CDE901650123B5
:106610006022A021204604F007FF10274A4B009378
:106620003A46CDE901750123A221204604F0FCFE83
:106630004FF02008454B00934246CDE901850123E8
:10664000A221204604F0F0FE414B00930823019361
:10665000029501237022A221204604F0E5FE3D4B65
:106660000093CDE9018501234022A221204604F0B8
:10667000DBFE394B0093CDE9017501238022A22175
:10668000204604F0D1FE354B0093CDE9017501237E
:106690008022B021204604F0C7FE314A0092CDE9A5
:1066A000016501233022A021204604F0BDFE2D4AC1
:1066B0000092CDE9016501233422A021204604F097
:1066C000B3FE294A0092CDE9016501233822A021B9
:1066D000204604F0A9FE254B00930622CDE90125B2
:1066E00001234022A021204604F09EFE0126204BDB
:1066F0000093CDE901653346FF22A021204604F036
:1067000093FE1C4B0093CDE90165FE223346A02188
:10671000204604F089FE04B0BDE8F081A09B002073
:10672000209C00204063002000000020F460002036
:10673000486300206C6100204463002068610020F1
:10674000646100207403002088610020DC61002067
:10675000CC610020A86100207061002098610020B9
:1067600054A0002050A000204CA00020C8A0002071
:1067700081610020806100202DE9F043AF4BB04CD7
:10678000DFF82C8385B04FF47A7504270022CDE919
:1067900001750093A0211A602046012304F0A8FD92
:1067A000322002F053FDA74BA74A0093CDE90175B3
:1067B000A0211A6020460123082204F099FD32200E
:1067C00002F044FDA14BA24A0093CDE90175A0213E
:1067D0001A6020460123102204F08AFD322002F0C4
:1067E00035FD9C4B9C4A0093CDE90175A0211A60B0
:1067F000204601230C2204F07BFD322002F026FD0E
:10680000964B00936422CDE90175A0211A602046C1
:1068100001231C2204F06CFD322002F017FD904B86
:1068200000930022CDE90175A0211A6020460123C2
:10683000282204F05DFD322002F008FD894B009310
:106840000126CDE9017546221E60A021334620466F
:1068500004F04EFD322002F0F9FC834B0093CDE9A9
:1068600001754A22C3F80080A0213346204604F077
:106870003FFD322002F0EAFC7C4BCDE9017550224D
:10688000C3F80080A02100932046334604F030FD79
:10689000322002F0DBFC764B764A0093CDE901759D
:1068A000A0211A6020463346302204F021FD322018
:1068B00002F0CCFC704B00936FF07F42CDE9017584
:1068C000A0211A6020463346342204F011FD322004
:1068D00002F0BCFC694B6A4A0093CDE90175A02126
:1068E0001A6020463346382204F002FD322002F0BE
:1068F000ADFC644B029506220192634A00931A6034
:1069000040F205529A80A02133464022204604F0EE
:10691000EFFC322002F09AFC5C4B019742F21272BB
:1069200002950093A0211A6020463346602204F0AD
:10693000DFFC322002F08AFC554A564B10689188E1
:10694000927902954FF010080093534F1860CDF8DC
:106950000480204699809A71A2213346424604F071
:10696000C7FC322002F072FC0FCFDFF848C1CDF82F
:1069700000C04FF020090295CDF80490CCF80C30FF
:106980003B78CCF80000CCF80410CCF808208CF848
:1069900010304A463346A221204604F0A9FC32209A
:1069A00002F054FC3D4A3E4B106812790295009368
:1069B00018601A710823019370223346A2212046E1
:1069C000384F04F095FC322002F040FC0FCFDFF886
:1069D000E8C0CDF800C0CDE90195CCF80C303B887B
:1069E000ACF81030BB78CCF80000CCF80410CCF830
:1069F00008208CF8123040223346A221204604F0B1
:106A000077FC322002F022FC274A029503CA274D68
:106A1000CDF80480009569601188298191782860FB
:106A2000A972334680222046A22104F061FC322064
:106A300005B0BDE8F04302F009BC00BF209C002077
:106A4000A09B0020406300200000204100000020A7
:106A500000009644F4600020000096C448630020C3
:106A60006C610020446300206861002064610020A4
:106A700054A00020C0A8000A50A000204CA0002074
:106A8000C0A80001C8A0002000125E01740300200D
:106A9000803A020888610020883A02089C3A02087D
:106AA000CC610020A43A0208B83A020870610020C4
:106AB00000401C46DC610020A86100200A4A0B4B04
:106AC00003CA70B40A4D0B4C2860696003CB0A4EB0
:106AD0001B882381336812782A722060616043F436
:106AE0000063336070BC7047C43A0208D03A0208B1
:106AF0000C620020FC610020209C00202DE9F04F5A
:106B000000248FB0CDE90844CDE90A44764B0094C7
:106B10000C941A6BDFF8DC81744EDFF8DCA1744F43
:106B2000DFF8D8B1DFF8D89142F010021A631A6B7F
:106B300002F010020092009A01941A6B42F00402D3
:106B40001A631A6B02F004020192019A02941A6B02
:106B500042F020021A631A6B02F020020292029A9B
:106B600003941A6B42F080021A631A6B02F08002DF
:106B70000392039A04941A6B42F001021A631A6B8F
:106B800002F001020492049A05941A6B42F0020288
:106B90001A631A6B02F002020592059A06941A6BA8
:106BA00042F040021A631A6B02F040020692069A03
:106BB00007941A6B42F008021A631B6B03F0080378
:106BC0000793404601227C21079B04F035F82246BA
:106BD0003046402104F030F850460122102104F0E4
:106BE0002BF822463846012104F026F82246584662
:106BF000112104F021F8224640464FF2807104F042
:106C00001BF8224648464CF2B30104F015F8012562
:106C10004FF2FC7308A94046CDE90835CDE90A4496
:106C200003F02EFE30464023022608A90893CDE942
:106C300009540B9603F024FE082208A950464FF48D
:106C40000413CDE908230A9403F01AFE10235046DA
:106C500008A90893CDE909540B9603F011FE08A981
:106C60003846CDE90855CDE90A4603F009FE02226F
:106C700008A938464FF44413CDE908230A9603F0D7
:106C8000FFFD5846112308A90893CDE909560B9634
:106C900003F0F6FD404608A940F603020023CDE9C3
:106CA00008230A9403F0ECFD4FF40042384608A98B
:106CB0000023CDE908230A9403F0E2FD4CF2B3036C
:106CC00008A948460893CDE909540B9403F0D8FD70
:106CD0000822002308A94846CDE908230A9403F0B6
:106CE000CFFD0FB0BDE8F08F003802400014024025
:106CF0000004024000100240000002400018024060
:106D0000000C0240022800D0704708B5074B4FF432
:106D100080501968FFF7ECFB012803D0044B0022D8
:106D20001A6008BDBDE80840FAF712BC209C00209C
:106D30001C61002082B002AB03E90300BDF804101F
:106D400002B003F079BF00BF82B002AB03E90300D9
:106D5000BDF8041002B003F073BF00BF82B002ABF5
:106D600003E90300BDF8041002B003F05FBF00BFE9
:106D700010B50C480C4A0D4C0023C0E900424FF4FA
:106D800080418022C0E90233C0E90413C0E9063320
:106D9000026204F0E5F900B910BDBDE8104000F052
:106DA000B5BD00BFA09B0020801A06000054004023
:106DB00030B5174B026889B000249A42CDE90244ED
:106DC000CDE90444069401D009B030BD114D0094C2
:106DD0002B6B114843F002032B632B6B03F0020370
:106DE00000934FF4C0721223CDE9022302A90423B9
:106DF0000693009A03F044FD01942B6C43F40013B6
:106E00002B642B6C03F400130193019B09B030BD7C
:106E100000540040003802400004024038B5134CD2
:106E2000134D2368134823F44013236000220121EB
:106E300003F002FF01222021284603F0FDFE01227B
:106E40008021284603F0F8FE00228021284603F026
:106E5000F3FE06484FF4806103F0E8FE236843F434
:106E6000801323600028DCD138BD00BF0010024031
:106E7000000C02400014024070B51D4C002220217D
:106E800006461C4803F0D8FE656805F06FFC1A4BF7
:106E9000A3FB0032920C63685B1B9342FBD3154D3E
:106EA00080210122284603F0C7FE144A4FF0F06308
:106EB00093613309DB019361B3039BB2C6F381068F
:106EC0000F4AAA611E43AE61646805F04FFC0A4B8D
:106ED0000749A3FB0032920C4B681B1B9342FBD368
:106EE000BDE8704003480022802103F0A5BE00BF2A
:106EF000001000E0000C024083DE1B430010024043
:106F0000000003C010B50446FFF788FF04480022C4
:106F1000012103F091FE2046BDE81040FFF7ACBF11
:106F20000014024010B501EB810100EBC10000F03C
:106F30007F04FFF773FF05480022012103F07CFE68
:106F400044F08000BDE81040FFF796BF00140240F7
:106F500010B50446FFF762FF01220448114603F012
:106F60006BFE2046BDE81040FFF786BF00140240CC
:106F700070B504787CB1084E0546FFF74FFF01223B
:106F80001146304603F058FE2046FFF775FF15F80E
:106F9000014F002CF1D170BD001402402DE9804852
:106FA00091B0B94BB948BA4EDFF818A3DFF818838F
:106FB000DFF818B3B74F002502951A6B42F00802AC
:106FC0001A631A6B02F008020292029A03951A6B76
:106FD00042F010021A631A6B02F010020392039A35
:106FE00004951A6B42F020021A631B6B03F0200316
:106FF0000493A0220123CDE90A230AA90022049BBD
:1070000000230124CDE90C2303F03AFCA2480A94A2
:107010000AA903F035FC4FF4F063A0480A930AA9CB
:1070200003F02EFC4CF2030398480A930AA903F0DC
:1070300027FC214698482A4603F0FEFD2A462021D7
:10704000924803F0F9FD322002F000F93820FFF7F2
:1070500013FF204602F0FAF83820FFF70DFF204614
:1070600002F0F4F80C20FFF707FF032002F0EEF81F
:107070002046FFF701FF032002F0E8F80620FFF7A3
:10708000FBFE032002F0E2F82046FFF73BFF8020E2
:10709000FFF738FF8020FFF735FF8148FFF768FFD3
:1070A000A820FFF72FFF7F48FFF762FF4FF4FA6039
:1070B00002F0CCF82046FFF725FF8020FFF722FFE3
:1070C0008020FFF71FFF7848734CFFF751FFA8207F
:1070D000FFF718FF7549764A0AA819F0A9FC0AA813
:1070E000FFF746FF4FF4FA6002F0B0F831684FF452
:1070F0008050FFF7FDF9002840F08E809AE80300E9
:107100000A908DF82C100AAB3A46112105A819F007
:1071100059FCFFF783FE00220121204603F08CFD7D
:107120008020FFF7A9FE9DF814507DB10DF11409E0
:10713000FFF774FE01221146204603F07DFD28462C
:10714000FFF79AFE19F8015F002DF1D1594B5A4A09
:10715000112105A819F036FCFFF760FE002201217D
:10716000204603F069FD8620FFF786FE9DF8145047
:107170007DB10DF11409FFF751FE012211462046A1
:1071800003F05AFD2846FFF777FE19F8015F002D3E
:10719000F1D1D8F800100120FFF7AAF90546002820
:1071A00041D031684FF48050FFF7A2F981460028A2
:1071B00040F09080DFF818C1BCE80F0005AD0FC5A6
:1071C000DCF800302B70FFF729FE4A4601212046EB
:1071D00003F032FDA820FFF74FFE9DF814507DB15B
:1071E0000DF11409FFF71AFE01221146204603F0A3
:1071F00023FD2846FFF740FE19F8015F002DF1D16D
:107200004FF47A700DF0E4FE31684FF48050FFF7D0
:107210006FF900283FF472AF284B93E803000A90FF
:107220008DF82C106FE7DBF800202549130E019331
:10723000C2F30743009305A8C2F30723D2B219F0A3
:10724000F7FBFFF7EBFD2A460121204603F0F4FC93
:10725000A820FFF711FE9DF81450002DD0D00DF19D
:107260001409FFF7DBFD01221146204603F0E4FC80
:107270002846FFF701FE19F8015F002DF1D14FF408
:107280007A700DF0A5FEBFE700380240000C024006
:10729000209C0020343B02080014024000100240F1
:1072A000DC3A0208F03A0208043B0208183B0208E4
:1072B0001C37020888610020403B02082C3B020872
:1072C000503B0208243B0208249C002060A00020C0
:1072D0006C3B02081A4B112193ED000A07220D2383
:1072E00005A8FEF7FBFC05A8F8F77CFF154A034646
:1072F000106805AAD050FFF791FD00220121204619
:1073000003F09AFCA820FFF7B7FD9DF81450002D5C
:107310003FF476AF0DF11409FFF780FD012211460D
:10732000204603F089FC2846FFF7A6FD19F8015F07
:10733000002DF1D14FF47A700DF04AFE64E700BFE2
:10734000F86000204C3B020810B588B0224B234C5B
:10735000002201921A6B42F008021A631B6B03F0C1
:107360000803019308220123CDE9022302A9002288
:1073700020460023CDE90423019B03F081FA10236A
:1073800002A92046029303F07BFA202302A920469B
:10739000029303F075FA402302A92046029303F0FA
:1073A0006FFA0F4B012293E80300FFF7C3FC0D4B6C
:1073B000012293E80300FFF7BDFC0B4B012293E889
:1073C0000300FFF7B7FC094B012293E80300FFF726
:1073D000B1FC08B010BD00BF0038024000100240F0
:1073E0006069020858690208506902084869020881
:1073F0002DE9F047514F524E3B78DFF85081514C08
:10740000514DDFF84CA1DFF84C9147E095E80300BF
:10741000FFF790FC64200DF0DBFDD9F800203B78ED
:10742000002A6CD0FF2B14BFD6E90001D8E9000177
:107430000122FFF77FFC21684020FFF759F8002860
:1074400057D021688020FFF753F800284BD095E8EB
:1074500003000122FFF76EFC21680120FFF748F8C6
:1074600002469AE80300002A65D00122FFF762FC79
:1074700021681020FFF73CF83B780246002851D0E5
:10748000FF2B14BFD8E90001D6E900010122FFF764
:1074900051FC4FF448700DF09BFD3B78D9F800206B
:1074A000002A35D0FF2B14BFD6E90001D8E900012E
:1074B0000022FFF73FFC21684020FFF719F8024641
:1074C0000028A3D021688020FFF712F828B921688E
:1074D0004020FFF70DF800289CD095E8030001221A
:1074E000FFF728FC96E721684020FFF701F8002805
:1074F000B2D095E803000022FFF71CFCACE7FF2B9D
:1075000014BFD6E90001D8E90001FFF713FC92E7A8
:10751000FF2B14BFD6E90001D8E900010122FFF7D3
:1075200009FCC8E7FF2B14BFD8E90001D6E9000128
:10753000FFF700FCADE7FFF7FDFB99E78161002055
:1075400058690208249C00206069020850690208FA
:1075500048690208289C002030B5002395B0CDE989
:107560000B33CDE90333CDE90533234901930D9363
:107570000793086C214A40F080500864096C01F0C0
:107580008051019101990293136843F48043136081
:10759000136803F48043029302244FF48003052010
:1075A0004FF480310822CDE90E434FF4A873CDE9A2
:1075B0000801CDE91023029801210222072308A81F
:1075C000CDE912230A9104F01DFE08B172B6FEE760
:1075D0000F220346CDE903244FF4A0554FF4805207
:1075E00003A80521CDE90535079205F021F808B17A
:1075F00072B6FEE715B030BD0038024000700040A2
:1076000080B501F0F7FDFFF7A7FFFFF777FAFEF768
:1076100033FA08F04BF9FFF797FEFEF751FAFFF740
:10762000A7FBFEF78FFFFFF749FAFAF7BDF901F064
:10763000C7FB8548854C864D864E874FDFF83882DC
:10764000DFF83892F9F7CCFD01F082FB8348F9F7B7
:10765000C7FD01F099FB82498248012206F0B6FE7F
:1076600000F052FC00F0BAFDF9F7F6FE01F0D8F890
:1076700001F09CF8002204217B4803F0DDFA02208F
:1076800001F0E4FD78480122042103F0D5FA00223C
:107690000321092002F032F80322002101200CF01E
:1076A0009FFB032203460021012023600CF098FB7E
:1076B00003220021286001200CF092FB032230609D
:1076C000002101200CF08CFB0322386000210120F6
:1076D0000CF086FB0322C8F80000002101200CF00A
:1076E0007FFB0322C9F80000002101200CF078FB89
:1076F00023685E4C2060002B5ED02A68002A52D09E
:107700003268002A6AD03A68002A70D0D8F800207F
:10771000002A5AD0D9F80020002A7AD000286FD049
:10772000184600231A4619460CF0C4FB00231A46DB
:10773000194628680CF0BEFB00231A46194630682B
:107740000CF0B8FB00231A46194638680CF0B2FB5F
:1077500000231A461946D8F800000CF0ABFB0023B2
:107760001A461946D9F800000CF0A4FB00231A466B
:10777000194620680CF09EFB0022082107200CF01F
:107780002FFB3B4B186000284CD00022082107201B
:107790000CF026FB374A106000284CD0FEF786FA22
:1077A0000BF0F6FFFEE74FF0300383F31188BFF3D1
:1077B0006F8FBFF34F8FFEE74FF0300383F31188D5
:1077C000BFF36F8FBFF34F8FFEE74FF0300383F3AC
:1077D0001188BFF36F8FBFF34F8FFEE74FF0300379
:1077E00083F31188BFF36F8FBFF34F8FFEE74FF026
:1077F000300383F31188BFF36F8FBFF34F8FFEE722
:107800004FF0300383F31188BFF36F8FBFF34F8FB7
:10781000FEE74FF0300383F31188BFF36F8FBFF3A0
:107820004F8FFEE74FF0300383F31188BFF36F8F64
:10783000BFF34F8FFEE74FF0300383F31188BFF3A0
:107840006F8FBFF34F8FFEE7189F00201C9C002016
:10785000189C0020149C00200C9C0020A89F002055
:10786000F89F0020609F002000100240F89B00203D
:10787000089C0020FC9B0020109C0020049C002001
:1078800038B50368B3F1804F03D01C4A934216D039
:1078900038BD1B4D044629684FF48050FEF728FE82
:1078A000012829684FF480700DD0FEF721FEF8B949
:1078B000144A236800211160104A9342E8D1BDE8C0
:1078C000384001F0B1BCFEF713FE48B10E4B012267
:1078D00093E80300FFF72EFAF9F73AFE2368D4E79E
:1078E00029684FF40050FEF703FE0028EED1F3E7BD
:1078F000054B93E80300FFF727FAD9E70010004093
:10790000209C00201C6100203869020872B6FEE746
:1079100030B583B0BE2308220DF1070105468DF86E
:107920000730F9F783FC0A4C2378DA07FCD40949BD
:1079300048222846F9F792FC2378DB07FCD409217A
:107940000448F9F7B3FCB0FA80F0400903B030BD49
:10795000880600203C9C002070B582B006460023BB
:1079600008460D468DF80730F9F746FCB0B1BEB1B8
:10797000552308220DF1070128468DF80730F9F745
:1079800055FC0F4C2378D907FCD4402231462846B9
:10799000F9F74CFC2378DA07FCD4012002B070BD63
:1079A000CC2308220DF1070128468DF80730F9F79E
:1079B0003DFC034C2378DB07FCD40120EEE700BF3D
:1079C0008806002010B50C46FFF7C6FF00B910BDB1
:1079D0002046BDE81040FFF79BBF00BF30B589B01F
:1079E0000C46FFF7B9FF08B909B030BD482308229B
:1079F0000DF1070120468DF80730F9F717FC154AFD
:107A00001378DB07FCD401234FF480720024002597
:107A100002A91148CDE90223CDE9044502F030FF67
:107A200001224FF480710C4803F006F932200DF06A
:107A3000CFFA4FF480721223CDE9022306480723C0
:107A400002A9CDE90445069302F01AFF012009B00E
:107A500030BD00BF88060020000C024030B583B066
:107A60000D46FFF779FF08B903B030BD4E23082259
:107A70000DF1070128468DF80730F9F7D7FB0A4CBE
:107A80002378DA07FCD4094A094912880A807F233F
:107A9000284618228B70F9F7C9FB2378DB07FCD442
:107AA000012003B030BD00BF88060020C86100205F
:107AB000389C00202DE9F04F754B764EDFF8109280
:107AC000DFF810B2DFF81082734F2DED028B0FCB71
:107AD0008DB003AC002584E80F008DF80A506F4C80
:107AE0006F4D9FED708A07E08BED008AD8F800009B
:107AF00041F288310CF066FC29684FF48050FEF7A3
:107B0000F7FC30B129680420FEF7F2FC002840F0B1
:107B1000B78031680120FEF7EBFC00BB3846F9F76F
:107B20006BFB002800F0A280D9F80030002B00F099
:107B3000D5804FF0000A39465046C9F800A0FFF73B
:107B40008DFF002800F08E8050463946FFF746FF33
:107B5000002800F0878054495448FEF793FB2968B9
:107B60004FF48050FEF7C4FC28B931680120FEF7BD
:107B7000BFFC0028BAD14E48F9F73EFB0028B3D02D
:107B800000234B488DF80B30F9F736FB00285DD009
:107B9000CC2347488DF80B3008220DF10B01F9F783
:107BA00045FB2378D907C3F3000AFAD44048FFF70E
:107BB000AFFE00284AD03F4B3D488DF80BA093F80C
:107BC00004A0F9F719FB002840D0CC2338488DF8E1
:107BD0000B3008220DF10B01F9F728FB2378DA07A7
:107BE000FCD4442332488DF80A3008220DF10A01F2
:107BF000F9F71CFB237813F00103FBD101222E4877
:107C0000019307A9CDE90933CDE9072202F038FE37
:107C100001221146284803F00FF84FF47A700DF056
:107C2000D7F90122019B079212222348089207A943
:107C30000822CDE909330B9202F022FE019B1C4978
:107C40001846FFF7BFFE002840F0EB801B4A136880
:107C50000133092B13603FF647AF194B1B68CBF874
:107C6000003043E70920FEF71BFB78E7154B164A67
:107C700018605860154B83ED008A012313606EE78E
:107C800031680120FEF734FC00283FF442AF45E79D
:107C9000FC350208249C0020189F00208806002044
:107CA000209C0020003C1CC694360208DE87002081
:107CB000A89F00203C9C0020000002402C9C00203B
:107CC00064030020D4610020349C00200C000020BC
:107CD0008461002008000020049C00203323082237
:107CE0000DF10A0138468DF80A30F9F79FFA23782A
:107CF00013F00103FBD1764A7649136038464022DF
:107D0000F9F7ACFA94F800A01AF0010AFAD1714818
:107D10000721F9F7CBFA002879D16D4A8DF80B00CD
:107D2000012338461360F9F767FA002860D0CC23A6
:107D300008220DF10B0138468DF80B30F9F776FA71
:107D40002378DA07C3F3000AFAD43846FFF7E0FDD8
:107D500000284DD0604B8DF80BA0384693F804A056
:107D6000F9F74AFA002843D0CC2308220DF10B0181
:107D700038468DF80B30F9F759FA2378DB07FCD435
:107D8000442308220DF10A0138468DF80A30F9F72C
:107D90004DFA237813F00103FBD10122CDE9093319
:107DA0004E48019307A94FF48073CDE9073202F0E2
:107DB00067FD01224FF48071484802F03DFF4FF407
:107DC0007A700DF005F94FF4807307931222019B2E
:107DD0004248089207A90722CDE909330B9202F025
:107DE0004FFD019B3E491846FFF7ECFD002844D1AA
:107DF0003C4A13680133092B13600ED83A4B3B4AB7
:107E00001B681360344B3A4A5B881380A7E6314BFA
:107E1000C3F800A0C3F804A0A1E6344B83ED008AA8
:107E2000F0E73448F9F7E8F90CAACAF3411302EB7A
:107E3000830353F8240C284B1B881840F8F782FB67
:107E40002D4B0022F8F7E8FBF8F7A0FE9FED2B7A08
:107E5000CBF8000007EE900AF4EEC77AF1EE10FAC4
:107E600003DD274B1B68CBF80030254ADBF80030D8
:107E70001360244A0023136038E61948F9F7BCF967
:107E80000CAACAF3411302EB830353F8240C124BE0
:107E90001B881840F8F756FB0022174BF8F7BCFB7D
:107EA000F8F774FE9FED157A104A07EE900AF4EE8B
:107EB000C77AF1EE10FA106002DD0B4B1B681360FD
:107EC0000A4B094A1B681360064A0023136099E7AE
:107ED000349C0020D46100203C9C0020000C024017
:107EE000189F0020309C0020680300200C00002018
:107EF000C8610020A89F00200000B03F0000A04201
:107F0000640300202C9C002000B52848284987B035
:107F10007F2200238260FF22CDE90133CDE90333C4
:107F2000C0E90013C0E90323C0E9053305930093BA
:107F300004F0B6FD68BB1D48012104F067FF43F261
:107F4000F223984202D107B05DF804FB00221748E3
:107F5000ADF8042001A9CDE904228DF8062004F033
:107F6000E9FDC8B9134B114800930022694604F09B
:107F70005FFEB8B900220D48114604F0CFFE70B97B
:107F80000A4843F2F222012104F03AFF07B05DF8FB
:107F900004FBFFF7BBFCCEE7FFF7B8FCE2E7FFF717
:107FA000B5FCEDE7FFF7B2FCE4E700BF489C00201A
:107FB000002800400202181A00B50F4A016885B077
:107FC00000239142CDE9013302D005B05DF804FBF6
:107FD00002224FF4807368460092039304F00EFC73
:107FE00030B9064B0122C3F83C2E05B05DF804FB06
:107FF000FFF78CFCF5E700BF002800400000474277
:10800000054B064800220121C3E90002C3E9022210
:10801000C3E9042299617047409D0020002C014073
:108020002DE9F041524B02688AB000249A42CDE912
:108030000444CDE90644089402D00AB0BDE8F081BA
:1080400003F5863301945A6C42F400625A645A6C08
:1080500002F400620192019A02941A6B42F0040247
:108060001A631A6B02F004020292029A03941A6BCA
:1080700042F008021A631B6B03F008034FF4F85236
:10808000039303270C26022304A905463948CDE9AA
:108090000423CDE90776039B4FF0040802F0F0FBC0
:1080A00002233548089604A9344ECDE90483CDE96E
:1080B000064702F0E5FB4FF480534FF480614FF424
:1080C0008040C6E904132023C6E906034FF40002EA
:1080D0004FF44033C6E90A723362294AC6F8248055
:1080E0004FF40013336330464FF00063C6E9024497
:1080F000C6E9002301F07EFBA0BB224C224B23608B
:108100004FF000614023C4E9011300224FF4806363
:10811000C4E903234FF480514FF48043C4E90513AD
:1081200020224FF44033C4E9072304210323C4E988
:1081300009134FF400024FF400132E642046C4E9E3
:108140000B23B56301F056FB78B900220521EC63DF
:108150003120A56301F0D2FA312001F00BFB0AB007
:10816000BDE8F081FFF7D2FBC7E7FFF7CFFBECE7F5
:10817000002C014000080240000C0240E09C00205E
:1081800058640240809C0020A06402400F4B0268AB
:108190009A4200D070470E4A536C10B523F4006326
:1081A000044653640B484FF4F85102F085FC042157
:1081B000094802F081FC206C01F0B0FBE06B01F09B
:1081C000ADFBBDE81040312001F0E2BA002C0140C7
:1081D0000038024000080240000C024010B511496E
:1081E000114C4FF482720023C4E9001201204FF4B5
:1081F0000072C4E904300821A26120460A22C4E9C1
:108200000233C4E90713C4E90933E26205F02CFC28
:1082100028B92268136843F04003136010BDFFF7CC
:1082200075FBF6E700300140C89D002030B5294BB2
:1082300002688BB000249A42CDE90444CDE906449B
:10824000089401D00BB030BD03F5843301945A6C0F
:10825000214842F480525A645A6C02F480520192CE
:10826000019A02941A6B42F001021A631A6B02F02F
:1082700001020292029A03941A6B42F002021A63FC
:108280001B6B03F00203039360220223CDE9042356
:108290000525022204A90323CDE906230895039BA3
:1082A00002F0EEFA20220223CDE9042304A90323DD
:1082B00000220A480895CDE9062302F0E1FA224699
:1082C0002946232001F01AFA232001F053FA0BB0BB
:1082D00030BD00BF003001400000024000040240F9
:1082E00082B00E4B00220092596C41F480415964D7
:1082F000586C00F48040009000980192186C40F097
:10830000805018641B6C03F080530193019B0F2174
:108310006FF0010002B001F0F1B900BF0038024077
:1083200070B588B0234B002202921A6C42F0100202
:108330001A641B6C03F010030293054601A903A8FD
:10834000029B04F039FA069BD3B904F015FA0346F0
:10835000194A1A4C1A49A2FB03239B0C013B002229
:10836000C4E90013204640F2E7332261A260A26113
:10837000E36005F09DFE064630B1304608B070BDA2
:1083800004F0FAF94300E3E7204605F081FC0646D5
:108390000028F2D1362001F0EDF90F2D01D9012688
:1083A000EBE732462946362001F0A8F9054B1D605F
:1083B000E3E700BF0038024083DE1B43209E00201D
:1083C000001000407C030020FEE700BFFEE700BF76
:1083D000FEE700BFFEE700BFFEE700BF704700BF3B
:1083E000014805F059BD00BFB89E0020014805F0C6
:1083F0009FBB00BFC89D0020014806F07FB800BFAA
:10840000609F002010B5044C2046F8F773FF20460B
:10841000BDE8104006F072B8189F0020014805F032
:10842000F9B900BF409D002010B5044C2046F8F774
:1084300061FF2046BDE8104006F060B8A89F00200C
:10844000014805F029BD00BF209E0020014801F031
:108450003BBB00BFE09C0020014802F0A5B800BF74
:1084600028A10020014803F0B3B900BFAC76012079
:10847000014801F029BB00BF809C0020014B988877
:1084800002F0E8BB40690208014804F09FBC00BF4D
:10849000489C0020704700BF704700BF0120704714
:1084A000024B16221A604FF0FF307047CC7C01203F
:1084B000014B16221A60FEE7CC7C012070B5161E17
:1084C00007DD0C468D19AFF3008004F8010BA542BF
:1084D000F9D1304670BD00BF70B5161E07DD0C46E1
:1084E0008D1914F8010BAFF30080A542F9D1304685
:1084F00070BD00BF4FF0FF30704700BF4FF4005316
:108500004B600020704700BF01207047002070477B
:108510000D490E4A0B6810B40D4C121B83B1184460
:10852000904204D808605DF8044B18467047094B28
:108530005DF8044B0C221A604FF0FF331846704769
:10854000054B0B60EBE700BF689E00200000022097
:1085500000040000CC7C0120E07C0120034AD2F81A
:10856000883043F47003C2F88830704700ED00E0B3
:108570002DE9F04F9BB00023DFF820827F4FDFF81A
:1085800020B2DFF82092DFF820A205931E461D4698
:108590000022114610200DF0C7FB04460028F7D03A
:1085A00042F2117200210DF03FFC40B9FF2120463C
:1085B0000DF096FC05A920460DF0B6FC18B120463A
:1085C0000DF012FCE4E7039020460DF029FE204652
:1085D0000DF00AFC059C6A4B62681868518B039B7E
:1085E00041F040015183674904324FF00A0C0A60A0
:1085F000C4F81CC01A4619460BF05CFC059806A985
:108600000DF0FCFC002836D00A30C0F293805E4B9F
:108610001A68002A40F089805C4B1968002940F0F4
:10862000A0800F24D9F800000A2208A90BF010FE40
:10863000012803460AD1DDE90812059800960DF0DD
:10864000E1FD002840F08480013CEBD101200CF0DA
:10865000BFFCD3E798F80030022B16D0059800969F
:108660000123042251460DF0CDFD002506980FF0A0
:10867000C5F8002851DB06980DF1120207A90FF08A
:108680008BF898F80030002BE4D1BDF812100223CB
:1086900088F800300029E9D0002402E00134A1422A
:1086A000E4D9079B1B5D05F168020DEB0200FA5C43
:1086B00002F00302022A04BF203BDBB20D2B05F1BE
:1086C000010500F8403C14D03F2DE7D951460598EC
:1086D0000096012304220DF095FDDBF80010012027
:1086E000FDF706FF98B988F80060BDF81210002564
:1086F000D4E70AA900F8406C254818F080FB25490A
:10870000002308681A4619460BF0D4FBEDE7224A0D
:1087100000211020FDF7F2FEE5E706980EF0CCFFF1
:10872000194B1A68002A3FF477AF0123174A1360E8
:10873000154B1E60DBF800100120FDF7D9FE90B943
:1087400005980DF06DFD05980DF04EFB05961FE7A1
:10875000114A00211020FDF7D1FE01200CF038FC59
:108760004CE71346E2E70C4B4FF480501968FDF7D5
:10877000BFFE0028E4D1F9F76FF9E1E7997102082B
:10878000F89B002070030020988A0020948A002023
:108790009C8A00201C9C0020209C0020DE8700205A
:1087A000249C0020089C00207C3E020800B51A484A
:1087B0004FF0804287B00260184A0023CDE90233AF
:1087C000CDE90433CDE90033C0E90133C0E9032327
:1087D000836105F06DFC98B94FF480530E48029305
:1087E00002A905F0A7FA98B9102200230A486946A1
:1087F000CDE9002305F08AFC28B907B05DF804FB39
:10880000FFF784F8E8E7FFF781F807B05DF804FBAD
:10881000FFF77CF8E8E700BFB89E00207F2C8000BF
:1088200000B51A481A4A87B00260532200234260FA
:108830004FF0FF32CDE90233CDE90433CDE9003307
:10884000C0E902320361836105F032FC98B94FF44C
:1088500080530E48029302A905F06CFA98B90022E1
:1088600000230A486946CDE9002305F04FFC28B9EA
:1088700007B05DF804FBFFF749F8E8E7FFF746F8B3
:1088800007B05DF804FBFFF741F8E8E7709E0020B1
:10889000000C004000B50368B3F1804F83B014D0E2
:1088A000154A934202D003B05DF804FB134B00223B
:1088B00001921A6C42F008021A641B6C03F0080360
:1088C0000193019B03B05DF804FB03F50E33002216
:1088D0000092196C41F0010119641B6C03F0010353
:1088E000009303211C20009B00F008FF1C2003B014
:1088F0005DF804EB00F03EBF000C00400038024081
:1089000070B53F4C034607CC3E4C186020789873F6
:108910006078D873A078596018743B49E07858742F
:1089200020799A606479394A9874312508789D8154
:10893000DC744D788C781875C87835499C75D87575
:10894000147850785D751C7658760C784E7891F8CE
:1089500003E0907891F808C0987604F00F0404EBD7
:10896000061483F830400C798879D278DA760EF0E4
:108970000F0E0EEB041483F83140CC79497A254A66
:10898000254D0CF00F0C0CEB011100F00F0000EB6B
:10899000041083F83310214983F8320010780978E5
:1089A00083F834001E4883F82B101E490078D962E2
:1089B000697883F82A0059772878E978AC781877AD
:1089C000D97719489C77002141F227151D6258621A
:1089D00019859178507883F836101179D47883F816
:1089E000350083F8381050799179D27983F837407F
:1089F00083F8390083F83A1083F83B2070BD00BF3C
:108A0000843E0208C8A0002054A0002050A00020EE
:108A1000A8610020886100204CA000208161002016
:108A20008061002033303031B16B00B52DE9F04F5B
:108A3000624C634D8BB00022114620200DF074F97A
:108A400020600028F7D047F2FF7229460DF0ECF9BC
:108A50000028F0D15B4D5C4FDFF88881DFF888910A
:108A6000206829460DF0CAFA0028F9D10DF112024A
:108A700005A928680EF090FE0EF012FE3860D0B105
:108A80003C210EF02BFE064690B1BDF812A0BAF1C3
:108A90000B0F0DD9DDF814B00C224146584618F0E2
:108AA000AEF8B0B10C224946584618F0A8F830B1DB
:108AB00038680EF001FE28680EF0FEFDD0E7BAF12E
:108AC0001F0F06D9414906220BF10C0018F043F89C
:108AD00050B13046FFF714FF3D4A3968206847F22D
:108AE000FF730DF0E9FAE3E7DBF81200DBF816108C
:108AF000DBF81A20BBF81EC00DF11A03009306AB79
:108B000007C34FF0040B4FF47A7AA3F800C0302269
:108B10000123A021CDE901BA2E4802F0E9FB322061
:108B200000F094FB0DF11E033422A021CDE901BA1F
:108B300000932848012302F0DBFB322000F086FB83
:108B40000DF122033822A021CDE901BA009321487A
:108B5000012302F0CDFB322000F078FB1E4B0120F8
:108B60001968FDF7C5FC83460028B2D10121FEF744
:108B7000D9F91A48FEF7FCF901215846FEF7D2F957
:108B80001748FEF7F5F94FF4967000F05FFB2E20C2
:108B9000FEF7DEF94FF4967000F058FB2E20FEF73A
:108BA000D7F94FF4967000F051FB2E20FEF7D0F964
:108BB000504600F04BFB00F0FDFD8AE7089F0020C7
:108BC0004C6F0208049F0020009F0020C8A00020D6
:108BD000486F0208A09B0020249C0020B43E02089D
:108BE000C43E0208943E0208A43E02082DE9F04F5C
:108BF0004B4C4C4DDFF848B1DFF848A1DFF8488115
:108C0000DFF8489185B00022114620200DF08CF845
:108C100020600EF045FD226828609AB1D8B1104658
:108C2000494642F211720DF0FFF8C0B128680EF00B
:108C300043FDD8F8000000210BF038F820680DF053
:108C4000D3F8E0E718B10EF037FD22681AB96420B6
:108C50000CF0BEF9D7E710460DF0C6F8F7E7324B37
:108C6000C82118680BF0AEFB0128DFD1BBF800204B
:108C7000DAF8001020680DF005F92C4B2C491B6820
:108C8000032207460A70F3B901932A4B1B68002B95
:108C900044D10F26D8F800000A2202A90BF0D8FA16
:108CA000012809D1BDF80C20029928680EF046FD74
:108CB00008B35FBB013EEDD101200CF089F91B4BDD
:108CC0001B68002BE1D001231A4A1360174B0022C6
:108CD0001A60194B01201968FDF70AFC0028A5D07D
:108CE000164B4FF480501968FDF702FC00289DD107
:108CF000F8F7B2FE9AE7BBF80030DAF800202968EE
:108D000020680DF0D9F90746002FD3D00B4A002177
:108D10001020FDF7F3FBF8F79FFECDE7019BD3E7AB
:108D2000109F00200C9F0020F89B0020988A0020B4
:108D3000DD870020948A0020249C0020209C0020B5
:108D40007403002070030020FC9B00204C6F02087D
:108D500010B50B480B4C00234FF4E1310C22C0E955
:108D60000041C0E90233C0E90432C0E9063305F02E
:108D7000D9FA00B910BDBDE81040FEF7C7BD00BF6D
:108D8000A89F0020004C004010B50B480B4C00235E
:108D90004FF4E1310C22C0E90041C0E90233C0E9DF
:108DA0000432C0E9063305F08BFA00B910BDBDE806
:108DB0001040FEF7ABBD00BF609F002000100140D7
:108DC00010B50B480B4C00234FF4E1310C22C0E9E5
:108DD0000041C0E90233C0E90432C0E9063305F0BE
:108DE000A1FA00B910BDBDE81040FEF78FBD00BF6D
:108DF000189F00200048004030B50368564A8FB0E5
:108E000000249342CDE90844CDE90A440C9407D0EC
:108E1000524A93422DD0524A934269D00FB030BD8E
:108E2000504B01941A6C504842F400221A641A6C98
:108E300002F400220192019A02941A6B42F001029C
:108E40001A631B6B9FED407B03F00103029308A99B
:108E500008238DED087B0C93029A01F011FD224648
:108E60000621342000F04AFC342000F083FC0FB0CF
:108E700030BD3C4B03945A6C3B4842F010025A649C
:108E80005A6C02F010020392039A04941A6B42F097
:108E900001021A631A6B02F001020492049A05940B
:108EA0001A6B42F002021A631B6B03F00203059374
:108EB0004FF48062072508A90223CDE908230C9509
:108EC000059B01F0DDFC0223402208A927480C95F0
:108ED000CDE90823CDE90A4401F0D2FC2246052160
:108EE000252000F00BFC252000F044FC0FB030BD25
:108EF0001C4B06941A6C1E4842F480221A641A6CA9
:108F000002F480220692069A07941A6B42F0080235
:108F10001A631B6B9FED0E7B03F00803079308A9F0
:108F200007238DED087B0C93079A01F0A9FC2246DC
:108F30000621272000F0E2FB272000F01BFC0FB0E9
:108F400030BD00BFAFF30080010000001200000040
:108F50000001000012000000004C00400010014021
:108F60000048004000380240000002400004024077
:108F7000000C024070B52E4B02689A4282B03ED07F
:108F80002C4C237813B12378042B1FD12A4B2B4A66
:108F90001B782B4DD25C02F00302022A08BF203B53
:108FA0004FF0040108BFDBB22A68217025490D2B60
:108FB0008B542AD001323F2A11DC2A601E492248F4
:108FC000012202B0BDE8704005F000BA1C4B1F49F9
:108FD0001D48002405221C6005F0DCF9EEE71B4962
:108FE0001948002605222E6005F0D4F9184B0120FF
:108FF0001968FDF77DFAA0B900232370DEE7154953
:109000001548012205F0E2F9BAE7002313488B5412
:109010002B6017F0F4FE124B01A918680BF0C2F890
:10902000CCE7104A31461020FDF768FAE4E700BFAC
:1090300000480040DE870020F89F00209971020858
:10904000F49F0020FC9F0020609F002080690208A0
:10905000249C0020F09F0020189F00209C8A002064
:109060001C9C0020209C0020DFF834D0FFF776FA0B
:109070000C480D490D4A002302E0D458C450043373
:10908000C4188C42F9D30A4A0A4C002301E0136049
:109090000432A242FBD317F08BFEFEF7B1FA704701
:1090A000000002200000002060060020A8730208D3
:1090B00060060020DC7C0120EFF3058000BEFEE7A7
:1090C00080B1CB6873B18A6862B130B40C6964B1A5
:1090D000D1E90051C0E90423C0E9025184610020B4
:1090E00030BC70474FF0FF3070474FF0FF30F7E76C
:1090F00070B5446882B0002301931CB1002630464D
:1091000002B070BD8368054603B1984720232B60E9
:10911000002607E0019B03F01F03A34215D0013492
:10912000202C0BD06B6901AA1221204698470028F9
:10913000F0DA0134202C6FF00406F3D12B681F2BDA
:1091400007D81EB1304602B070BD2C6001236B60A1
:10915000D4E76FF00206D2E730B583B0002543694B
:109160000195044601AA006801219847A8423DDB09
:109170006369206801AA01219847002836DB019B1A
:109180005B072AD56369206801AA29469847002809
:109190002CDB019BDD0414D56369206801AA1F2123
:1091A0009847002822DB019BDA041DD503F01C033D
:1091B000182B17D0082B13D0142B0BD1042003B07D
:1091C00030BD03F40452B2F5045F0BD0980407D409
:1091D000D905F3D4052003B030BD012003B030BD64
:1091E0000320F8E70220F6E70620F4E76FF004001A
:1091F000F1E700BF08B50B4B1A6842F400721A6021
:109200001A6842F480621A601A6842F480721A6026
:10921000032000F061FA0F20FFF782F8FFF760F8F3
:10922000002008BD003C0240034A044B11681B7833
:109230000B441360704700BF3CA00020780300205F
:10924000014B1868704700BF3CA0002038B50446A9
:10925000FFF7F6FF631C054602D0044B1B781C4445
:10926000FFF7EEFF401BA042FAD338BD7803002081
:10927000002800F09E8038B5056C04463DB1236C93
:10928000DB060CD5002384F83C30012038BDF8F70C
:1092900027F96564236C84F83C50DB06F2D4236C18
:1092A000474A23F4885323F0020343F00203236464
:1092B0005168236821F4403151605168606801436E
:1092C00051605A682069A16822F480725A605A6815
:1092D00042EA00225A605A68E06822F040725A60FE
:1092E0005A680A435A609A68A16A22F400629A6036
:1092F0009A6802439A60334A91429A6851D022F0A8
:109300007062E06A9A609A68114399609A6822F0E4
:1093100040529A609A6802439A609A6822F0020268
:109320009A609A68217E42EA41029A6094F820206D
:10933000002A40D05A68616A42F400625A605A6852
:1093400022F460425A605A68013942EA41325A6056
:10935000DA6AE16922F47002DA62DA6A013942EA11
:109360000152DA629A68616922F400729A609A681E
:1093700094F8300042EA40229A609A6822F48062AF
:109380009A609A68002042EA81229A606064236CA5
:1093900023F0030343F001032364002384F83C30EB
:1093A00038BD22F070629A609A6822F040529A604A
:1093B000B3E7012070475A6822F400625A60C7E799
:1093C000002301400100000F10B490F83C3083B03E
:1093D0000022012B019268D00123026880F83C3002
:1093E0009368DB0714D4354B354C1B689168A4FB9C
:1093F00003439B0C03EB430341F001019160019394
:10940000019B2BB1019B013B0193019B002BF9D1E7
:10941000936813F0010F036C37D023F4E06323F05B
:10942000010343F48073036453685C0505D5036C42
:1094300023F4405343F480530364036C13F48053C8
:109440001CBF436C23F0060343646FF022011D4BE5
:10945000002480F83C4011605968C80621D11A499F
:109460008A4209D001F580718A4223D017498A4285
:1094700012D15B68DB060FD4936813F0405F0BD109
:10948000936843F08043936006E043F01003036465
:10949000436C43F001034364002003B05DF8044BC8
:1094A0007047094B9A42F7D1E6E7022003B05DF816
:1094B000044B70475B68D906DED0EDE76C030020F3
:1094C00083DE1B43002301400020014000220140B5
:1094D00003689A6870B50D465105044602D59B682D
:1094E000DA0544D4FFF7ACFE2268064613689907F4
:1094F00004D46B1C23D113689807FCD56FF01203BA
:109500001360236C43F400732364936813F0405F8B
:1095100013D1237E8BB9D36A13F4700F02D09368F2
:109520005A050AD4236C23F480732364236CDB0470
:1095300003D4236C43F001032364002070BD5DB9A4
:10954000136813F00203D1D1226C84F83C3042F04E
:1095500004022264032070BDFFF772FE801BA84244
:109560002268C3D9136813F00203BFD1ECE7036C80
:10957000002243F0200380F83C200364012070BDEA
:109580000368D86C704700BF70B590F83C3082B06B
:109590000246012B4FF00000019000F09380012360
:1095A00082F83C300D6813688C68092DA8B228D861
:1095B0001E6905EB450E4FF0070C0CFA0EFC26EA6F
:1095C0000C061E611E6904FA0EF434431C614C68DB
:1095D000062C04EB84012AD85C6B05394FF01F0C74
:1095E00088400CFA01F124EA01015963596B0843E0
:1095F000586336498B422BD0002082F83C0002B0E1
:1096000070BD00EB400CDE68ACF11E0C4FF0070E95
:1096100004FA0CF40EFA0CFC26EA0C06DE60DE6896
:109620003443DC604C68062C04EB8401D4D90C2C48
:1096300034D81C6B23391F26884006FA01F124EA2E
:1096400001011963196B0843204918638B42D3D178
:10965000122D30D0A5F11003012BCDD81C494B6839
:10966000102D43F400034B60C6D11A4B01F1467133
:109670001B6801F52E3101F28331A1FB03139B0C12
:1096800003EB83035B000193019B002BB4D0019B90
:10969000013B0193019B002BF9D1ADE7DC6A413915
:1096A0001F26884006FA01F124EA0101D962D96A2D
:1096B0000843D8629DE7D1F8043343F48003C1F82E
:1096C000043399E7022002B070BD00BF00200140C2
:1096D000002301406C0300200749CA6803024FF6CB
:1096E000FF0003F4E0630240134343F0BF6343F41D
:1096F0000033CB60704700BF00ED00E01B4BDB6820
:10970000C3F3022300B5C3F1070EBEF1040F03F14A
:10971000040C28BF4FF0040EBCF1060F1CD9A3F1B6
:10972000030C4FF0FF3303FA0CF322EA03024FF06D
:10973000FF3303FA0EF321EA030303FA0CF3134396
:109740001B010028DBB20ADB00F1604000F561403C
:1097500080F800335DF804FB00229446E7E7044AF2
:1097600000F00F00024413765DF804FB00ED00E00A
:10977000FCEC00E0002807DB044A4109012300F06B
:109780001F00834042F82130704700BF00E100E035
:1097900000280CDB4309064900F01F00203301229A
:1097A000824041F82320BFF34F8FBFF36F8F704784
:1097B00000E100E0BFF34F8F0549064BCA6802F491
:1097C000E0621343CB60BFF34F8F00BFFDE700BFE4
:1097D00000ED00E00400FA05002808DB4309044915
:1097E00000F01F0001226033824041F823207047BF
:1097F00000E100E038B50446FFF722FD002C6BD0F5
:1098000023680022022184F8351084F834201A6875
:1098100022F0010205461A6005E0FFF711FD431B27
:10982000052B37D823681A68D107F6D4D4E901206C
:10983000E16802430A43D4E90451A0692A430A4378
:10984000E1691D6802430A4331492940256A2A43D8
:109850000A43616A042924D01A605A6922F0070277
:109860001143D8B22B4A59611038A2FB0052120999
:1098700029496FF30903895CE1655F2888BF0433D8
:109880003F228A40A36500209A600123606584F826
:10989000353038BD03232022626584F83530184600
:1098A00038BDD4E90B512943114319605969A26AA3
:1098B00021F00701114341F00401002DD1D068B916
:1098C000012A21D032F00202CBD1EA01C9D54022CF
:1098D0000123626584F83530012038BDB0F5005FA2
:1098E00004D0022AF3D9032AEFD0BAE7032AB8D862
:1098F00001A050F822F000BFCF980008CB980008D4
:10990000CF98000809990008B5F1C07FA9D1DEE71A
:109910003F8010F0ABAAAAAA88690208002835D0B7
:1099200090F83520022A0346D0B22ED01A68184982
:10993000D0B2103830B4A1FB004109091468154DAC
:1099400024F001046D5C146000211160516091608D
:10995000D1601161212151615F286FF3090288BF35
:1099600004323F240021AC40DD65C3E90F11C3E997
:109970001111C3E913119A659460596583F8341085
:1099800083F83510084630BC704770470120704797
:10999000ABAAAAAA8869020870B490F83440856D11
:1099A000012C0AD090F835404FF0010C644580F846
:1099B00034C005D0002380F83430022070BC7047DA
:1099C000022680F83560046800264665266826F47D
:1099D0008026266063608368402B0EBFA260A16072
:1099E000E260C26D08BFE1603F239340AB60236833
:1099F000026C43F0160323601AB1236843F0080396
:109A00002360236843F001030020236070BC70478B
:109A100070B50446866DFFF713FC94F83530022BC1
:109A200006D080236365002384F83430012070BDA4
:109A300023681A6822F016021A605A6922F080021E
:109A40005A61226C054642B31A6822F008021A6075
:109A50001A6822F001021A6005E0FFF7F1FB431BD0
:109A6000052B10D823681B6813F00103F5D1E16DB5
:109A70003F228A40184601210023B26084F8351045
:109A800084F8343070BD032320226265184684F8C0
:109A90003530002384F8343070BDA26C002AD3D155
:109AA000D6E700BF90F83530022B03D08023436502
:109AB000012070470268052380F83530136823F0D1
:109AC0000103002013607047F0B583B0674A876DCB
:109AD000166800230193C36D3D6808229A402A420C
:109AE000044603D001680868400778D401229A40F0
:109AF0002A4203D02168496908066AD404229A40A0
:109B00002A4203D02168096889075CD410229A4050
:109B10002A4203D021680868000741D420229A40D5
:109B20002A4214D021680868C00610D5BA6094F89B
:109B30003520052A63D00B6813F4802F0B687ED084
:109B4000190340F18980E36B0BB120469847636DA0
:109B500023B3636DDA071AD522684549052384F8D3
:109B600035301368A1FB061623F00103B60A136013
:109B700002E01368DB0704D5019B0133B342019374
:109B8000F7D90122002384F8352084F83430E36CBF
:109B900023B1204603B0BDE8F040184703B0F0BD44
:109BA000BA600A6812F4802F0A6822D1D20503D461
:109BB0000A6822F008020A60226C002AAED0204611
:109BC0009047E36DAAE7BA60626D42F004026265F5
:109BD0009CE7BA60626D42F0020262658EE7086837
:109BE00020F004000860BA60626D42F00102626514
:109BF0007CE71103E0D5A26C002AE0D18EE70A6869
:109C000022F016020A604A6922F080024A61226C40
:109C10003AB30A6822F008020A603F2202FA03F30C
:109C2000216DBB600122002384F8352084F8343094
:109C30000029B3D0204603B0BDE8F040084713F434
:109C4000807380D10A6822F010020A60012284F831
:109C5000352084F8343076E7636C002B7FF475AFE1
:109C600075E7A26C002AD4D1D7E700BF6C030020AF
:109C7000B5814E1B406D70472DE9F043876A8E68B1
:109C800000EB870CDCF818301C68002C7CDBDCF85F
:109C90002C40002C78D134689C605C6875686FF348
:109CA0000C042C430D685C609146EA0706D51C68DD
:109CB00024F4400E4C694EEA04041C60AC0605D541
:109CC0000C69196821F04061214319606A0703D5C6
:109CD000196841F0800119601968B46841F0805139
:109CE0001960002C7DD0DFF804E13D4601262AE012
:109CF00041F0804119606B1C032B94BF1D46033D4E
:109D000000EB85018B69D3F80080B8F1000F26DBEA
:109D1000C96A21BB1968D4F80080626821F08051BB
:109D20001960C3F80880596801EA0E0111435960AF
:109D3000BFF35F8F1968A46841F0004106F1010884
:109D4000196024B34646196821F00051196019685A
:109D5000B9F1000FCCD121F080411960CBE7DCF8DC
:109D600018208EB10021BFF35F8F13687C1C032C79
:109D700023F000438CBF033F27461360013100EB03
:109D80008703B1429A69EED10220BDE8F083DCF886
:109D900018101A68B9F1000F1FD042F080421A6003
:109DA0001A6842F000521A60BFF35F8F0B68C26BF3
:109DB00043F000430B6000EB8503DA628562EFF34A
:109DC0001082012383F31088036C0133334403644E
:109DD00082F310880020BDE8F08322F080421A60F0
:109DE000DEE73D4626461946D3E700BF00E0FFFF09
:109DF00070B58B680C46D1E905120B43616A1343B9
:109E0000A27B05460B43E07F217F43EA426343EA9E
:109E1000004343EA013321792A6843EA8123E17B45
:109E2000106843EAC11394F8281043EA01132B4940
:109E300001400B43217CB1FA81F1490943EAC15346
:109E4000617CB1FA81F1490943EA8153A17FB1FAFA
:109E500081F1490943EA413394F82010B1FA81F1C4
:109E6000490943EA4123136001201668FFF7EEF920
:109E70002968A26C236D0E60886943EA024394F856
:109E80004C204FF6417C00EA0C00B2FA82F25209F3
:109E9000034343EAC21394F8552094F85600A2F104
:109EA0000102B2FA82F2520943EAC20394F8542042
:109EB000A0F10100B0FA80F0A2F101024009B2FA6B
:109EC00082F243EA8003520943EA42038B61012094
:109ED0008C69FFF7BBF92B689C6170BD0F8120FD79
:109EE00070B54B6902680C46096A0B43617B43EA13
:109EF0004163A17B43EA4153217F43EAC113A17F20
:109F000002F5805243EA811394F82410054643EA8F
:109F1000810390691A4901400B43217BB1FA81F119
:109F2000490943EA8163617FB1FA81F1490943EA52
:109F30000153936101209669FFF788F92A68A368A5
:109F4000A169A06A02F580520B43966194F825102E
:109F500043EAC11321690B4321680B43217943EA8A
:109F6000800343EA416343F4000313600120146853
:109F7000FFF76CF92B6803F580531C6070BD00BFC0
:109F8000233FDEF82DE9F041D0E91A7882B007F1DD
:109F90001203002250F82340204E01920546B8F1EA
:109FA000000F18D0236A83B3AA6D6B694ABB334391
:109FB000636023687A1C032A43F000438CBF033F8D
:109FC0001746236007F1120308F1FF3855F82340C4
:109FD000B8F1000FE6D1EB6E43450FD0BFF35F8FB2
:109FE0002A682969FB1C03F0030303EB830302F5D2
:109FF000805201EBC3019160C5E91A7802B0BDE857
:10A00000F08143F480436360D3E701A806F01EF9B2
:10A01000019B002BDFD02362A360C5E700400080D6
:10A02000002800F016812DE9F041D0F88430A6B068
:10A030000546002B00F00781874AA868002301939A
:10A04000516C864B41F480415164526C02F4804261
:10A050000192019A5A6822F400025A6059682A68EB
:10A06000014302F5805259605B68136843F00103B5
:10A070001360FFF7E5F8064606E0FFF7E1F8801BFE
:10A08000B0F5FA7F00F2D5802B6803F580531C6889
:10A0900014F00104F1D14FF480430126704A129369
:10A0A0000DA94FF400632846ADF852608DF8386072
:10A0B000CDF8422013930F948DF850408DF8544002
:10A0C00016948DF85C401F948DF8804021948DF893
:10A0D0008A40ADF88840FFF78BFE4FF48072ADF8F0
:10A0E00024204FF480014FF4803240F20113049297
:10A0F00008914FF4005202A92846ADF814308DF8AB
:10A1000016608DF80C600692ADF82C3007948DF82F
:10A1100026400A940C940294FFF7E2FEEA68146069
:10A1200054609460D46011682E46134641F4801147
:10A1300046F8182F02F1A00743F8281B1146CB6000
:10A14000086840F4400008601C605C609C60DC6053
:10A1500046F8043F186840F48010194643F8280B6D
:10A160009F42ECD1C2F88420D5E904172E68936F82
:10A1700006F5805E43F4400347F480474FF0004CFF
:10A180009367AC62CEF810200C604C608C60CC60A1
:10A19000C1F800C04F604B68C1E908442C4623F069
:10A1A00000434B6044F8481F01F1280305F15408AF
:10A1B00008460022C3601A605A609A60DA60C3F8E9
:10A1C00000C05F60586820F000405860C3E9082272
:10A1D00044F8043FA045184603F12803EAD1C1F82A
:10A1E0008410C5E91722C5E91A22AA65CEF80C1019
:10A1F00069681C4B8888186409685964F36B43F4D8
:10A200000273F363D6F80C3143F4003343F0600378
:10A21000C6F80C31D6F81031102143F40313002096
:10A22000C6F81031C5F88820C5F8841026B0BDE8FE
:10A23000F0810422E0230120C5F88820C5F884308D
:10A2400026B0BDE8F0812023C0F8843005F024FF5B
:10A25000F2E60120704700BF00380240003801409C
:10A260000100010100800240D0F88430102B01D0A1
:10A270000120704770B5202204460126042382B0D5
:10A28000C0F884208665C366FFF77CFE23683046ED
:10A290001D68FEF7DBFF226802F5805315609A699E
:10A2A00042F400529A619A69002542F002029A61D2
:10A2B00001959A6942F480129A619B690193304634
:10A2C000FEF7C4FF2368019903F58052304691617F
:10A2D0001A6842F008021A601E68FEF7B7FF23688A
:10A2E0001E601A6803F5805142F004021A60CB69BF
:10A2F00043F4D0332846402243F0C103CB61C4F875
:10A30000842002B070BD00BFD0F88430402B01D053
:10A310000120704730B50168202201F5805383B0D9
:10A32000C0F88420DA6922F4D03222F0C102DA6166
:10A330009A6922F400529A619A6922F002029A61A3
:10A340000B68044623F004030B6001200D68FEF740
:10A350007DFF236800221D6003F5805301929A69F6
:10A3600042F480129A619B6901930120FEF76EFF0F
:10A370002368019903F58052012091611A6822F047
:10A3800008021A601D68FEF761FF224604F15400BE
:10A3900052F8443B1D6052F8041F4B68824243F060
:10A3A00000434B60F7D100201023A065C4F884302F
:10A3B00003B030BD10B5044631B3D0F88420402A34
:10A3C00001D0012010BD4B6BC3630122FFF754FC89
:10A3D00098B9BFF34F8FA36A5A1C032A88BFDA1EAD
:10A3E0002368A26203F580535A69520703D50421FA
:10A3F000002259615A60002010BDD4F8883043F023
:10A400000203C4F88830DCE7D0F8883043F0010359
:10A41000C0F88830D5E700BF2DE9F04F054685B07C
:10A42000002975D0D0F88430402B5BD1C76DC36E46
:10A4300007F11202C3F1040A50F822402268002AF0
:10A4400074DBBAF1000F73D000F180034FF0000805
:10A45000019300F17C030293C146039103E0C245DE
:10A4600039D0002E48D12368D90503D5E369AB67FD
:10A47000A3696B6723689A0501D4EE6FEEB1236878
:10A480009B0548BFC5E918992368266816F48076AD
:10A49000C3F30D4B02D022682A670126A26822620C
:10A4A000DDE901105B4605F0F5FE2A6E01322A66F1
:10A4B0006A6E5A446A66C4F820907B1C032B8CBFDA
:10A4C000033F1F4607F1120308F1010855F8234026
:10A4D0002368002BC3DAEB6E03994344EB662BB978
:10A4E000EF657EB9012005B0BDE8F08F28460191E7
:10A4F000FFF748FD0199F3E7EB6E03994344EB66E0
:10A500006BB9EF65EA6F0A6000231846EB67EAE76C
:10A51000D0F8883043F00103C0F88830E2E72846DD
:10A520000191FFF72FFD0199EF65EBE7002BD9D0E3
:10A530002846FFF727FDEF65D4E700BF2DE9F0417E
:10A54000D0E9105475B106464FF0000806EB8407B9
:10A55000A300F86A2344013D38B1F26852F8333061
:10A56000002B0BDA0020BDE8F081631C032B13D90C
:10A57000033C002DEAD10020BDE8F08105F0A6FEE5
:10A58000631C032B8CBF033C1C46C7F82C80C6E918
:10A590001054002DDAD1EEE71C46002DD6D1EAE7A3
:10A5A000704700BF704700BF026802F580532DE975
:10A5B000F041D2F838805D69304ADE695769690632
:10A5C000044601D5720647D4E90701D5F20739D40C
:10A5D0002B0401D5300406D418F0080F1BD13B031F
:10A5E00027D4BDE8F081D4F8883043F00803C4F8DC
:10A5F0008830236803F58053A9045A6931D448F29E
:10A6000080610A40C4F88C205961204605F034FC72
:10A6100018F0080FE3D02368DB6A03F06003C4F886
:10A6200094302046FFF7BCFF0023C4F894303B036E
:10A63000D7D5124B4FF400225A612046FFF7B2FFE4
:10A64000BDE8F081236803F580534FF001125A6191
:10A65000204605F00BFCBBE7094A5A6105F000FCF7
:10A66000B2E708490A40C4F88C20DA6922F4C03203
:10A67000DA61E023C4F88430C7E700BF003C014042
:10A680004000010000207E0070B5044600681D46B1
:10A690000369920103F01C0302F4F862C9021A4331
:10A6A00089B2114341F001010161FEF7C9FD06467F
:10A6B00004E021680A6912F0010207D0FEF7C0FD2C
:10A6C000801BB0F5803FF4D3012070BD4B699BB275
:10A6D00010462B6070BD00BF38B5044600689DB2BF
:10A6E00003694561920103F01C0302F4F862C90298
:10A6F0001A4389B2114341F003010161FEF7A0FD45
:10A70000054604E023681B6913F0010307D0FEF738
:10A7100097FD401BB0F5803FF4D3012038BD1846AB
:10A7200038BD00BF002964D003681A68C2F3001264
:10A7300010B481F828201C681A6882F40072C2F3F1
:10A74000402281F820201A68C2F30042CA771A68B2
:10A7500082F40052C2F340328A771A68C2F30032A0
:10A760000A7704F060044C621C681A6804F4006400
:10A7700002F48042C1E905241A6882F48002C2F31F
:10A7800080524A741A6882F40002C2F3C0520A74FA
:10A790001A68C2F3C012CA731C681A68C2F3802216
:10A7A0000A711A68C2F340628A739A6904F46024D9
:10A7B000C2F340028C6081F854209A6982F08002D2
:10A7C000C2F3C01281F84C209C699A69120C8A6409
:10A7D0009A69C2F3800281F856209B6904F0300424
:10A7E000C3F3C00300200C6581F855305DF8044BBD
:10A7F00070470120704700BF31B108B5D0F88430F0
:10A80000102B03D0012008BD01207047FFF7F0FA9C
:10A81000002008BD38B5036805461C6901F0A6FF95
:10A820000F4B984224F01C0404D844F008042B6811
:10A830001C6138BD0B4B984204D22B6844F00C04C9
:10A840001C6138BD084B9842F1D9084B98422B68DF
:10A8500094BF44F0040444F010041C6138BD00BFF0
:10A86000BF0E160200879303FFE0F5057FD1F008C5
:10A87000D0F88800704700BFD0F88C00704700BF48
:10A880002DE9F04F00230C68DFF814A285B04FF0DB
:10A89000010B894603E00133102B00F092800BFA84
:10A8A00003F202EA0408A243F5D1D9F8041001F03A
:10A8B000030C5A0003250CF1FF369540012E6FEA78
:10A8C000050540F28180BCF1030F40F0D980066895
:10A8D0000CFA02F235402A4311F4403F0260DAD00C
:10A8E00000220392DAF8442042F48042CAF844205D
:10A8F000DAF8442002F480420392039A23F0030220
:10A9000002F1804203F003060F2702F59C32B600E5
:10A9100007FA06FC5F4F9568B84225EA0C0527D078
:10A9200007F58067B84200F087805B4FB84200F0BF
:10A930008980DFF870C1604500F08A80DFF868C167
:10A94000604500F08B80DFF864C1604500F08C80CA
:10A95000DFF85CC1604500F08D80DFF858C16045CC
:10A960000CBF4FF0070C4FF0080C0CFA06F63543FD
:10A9700095604A4A9268CE026FEA0805474E54BF76
:10A980002A4048EA0202B260F268444E8F0254BF85
:10A990002A4048EA0202F26072688E033F4E54BFBA
:10A9A0002A4048EA020272603268C90303F10103D7
:10A9B0003A4954BF2A4048EA0202102B0A607FF449
:10A9C0006EAF05B0BDE8F08F866806EA050ED9F8CF
:10A9D0000C60964046EA0E068660466826EA080E37
:10A9E000C1F300169E4046EA0E064660C66806EAB7
:10A9F000050ED9F80860964046EA0E06BCF1020F33
:10AA0000C6607FF464AFDE0800EB86060196376A05
:10AA1000D9F81060009703F0070E4FEA8E0E0F274B
:10AA200006FA0EF607FA0EFE009F27EA0E0E019FA9
:10AA300046EA0E063E624AE74FF0010C0CFA06F6B3
:10AA4000354395E74FF0020C0CFA06F635438FE7D5
:10AA50004FF0030C0CFA06F6354389E74FF0040C6F
:10AA60000CFA06F6354383E74FF0050C0CFA06F6B0
:10AA700035437DE74FF0060C0CFA06F6354377E7D1
:10AA8000C66806EA050ED9F80860964046EA0E0642
:10AA9000C6601CE70000024000080240003C014084
:10AAA00000380240000C0240001002400014024036
:10AAB00000180240001C02402DE9F04F0023534FC4
:10AAC00083B001264FF00F094FF0030A02E0013373
:10AAD000102B76D006FA03F232EA010402EA010CE6
:10AAE000F5D123F0030505F1804503F00304A4002C
:10AAF00005F59C3509FA04F80194454CD5F808E0B1
:10AB0000A04208EA0E0E20D004F58064A0425BD07B
:10AB1000404CA0425CD0404CA0425FD03F4CA04291
:10AB200062D0DFF8FCB0584564D0DFF8F8B0584583
:10AB300066D0DFF8F4B0019C58450CBF4FF0070B0E
:10AB40004FF0080B0BFA04F400E00024A64513D1E3
:10AB50003C6824EA0C043C607C6824EA0C047C60B9
:10AB6000FC6824EA0C04FC60BC6824EA0C04BC60A9
:10AB7000AC6824EA0804AC6004685D000AFA05F5D4
:10AB80004FEAD30C24EA050400EB8C0C046003F0BC
:10AB90000704DCF820E0A40009FA04F42EEA040417
:10ABA000CCF82040C46824EA0504C460446824EA60
:10ABB000020242608268013322EA0502102B8260A1
:10ABC00088D103B0BDE8F08F019C06FA04F4BDE71C
:10ABD000019C4FF0020B0BFA04F4B7E7019C4FF015
:10ABE000030B0BFA04F4B1E7019C4FF0040B0BFAD2
:10ABF00004F4ABE7019C4FF0050B0BFA04F4A5E756
:10AC0000019C4FF0060B0BFA04F49FE7003C014057
:10AC10000000024000080240000C02400010024008
:10AC20000014024000180240001C0240036919424F
:10AC300014BF01200020704702B9090481617047E8
:10AC4000436901EA030221EA030141EA0241816109
:10AC5000704700BF044A5169014200D1704708B5EE
:10AC60005061FCF74FF808BD003C01402DE9F84366
:10AC70000D46804616461F464FEA1149B9F1010FAD
:10AC8000D8F8003002D111E07A1C19D19C6925EA6C
:10AC9000040C1FFA8CFCBCFA8CFC4FEA5C1C664569
:10ACA000F2D00020BDE8F883791C09D15C6925EA5F
:10ACB0000404A4B2B4FA84F46409A642F4D0F0E720
:10ACC000FEF7BEFA089BC01AB84220D9D8F8003067
:10ACD000B9F1010F0CBF5B699B6925EA03039BB2C5
:10ACE000B3FA83F35B09B342C8D100222023C8F82A
:10ACF000302088F83D3088F83E20D8F8403088F879
:10AD00003C2043F02003C8F840300120CAE7002F60
:10AD1000B4D1DBE72DE9F843046880460E461746B8
:10AD2000994604E065696A0509D47B1C21D16069F4
:10AD300026EA000080B20028F4D1BDE8F883236839
:10AD400043F400732360002220236FF4806161616B
:10AD5000C8F8302088F83D3088F83E20D8F84030D8
:10AD600043F00403C8F84030002388F83C30012049
:10AD7000E3E7FEF765FAA0EB0900B842D8F8004017
:10AD800001D8002FD3D1636926EA03039BB2002BBD
:10AD9000CDD000232022C8F8303088F83D2088F834
:10ADA0003E30D8F840301343C8F84030DCE700BFED
:10ADB000F8B5036806465869400624D40D46174680
:10ADC0000DE0FEF73DFAC01BA842336800D81DB95C
:10ADD0005C6914F0400418D05A69520613D45A69B9
:10ADE000D106EED500226FF01000202158613263A9
:10ADF00086F83D1086F83E20336C3364002386F8D5
:10AE00003C300120F8BD0020F8BD2023346386F8D3
:10AE10003D3086F83E40336C43F020033364EDE769
:10AE2000F8B5046805460E46174601E0731C1AD1B2
:10AE3000636913F0800314D160694205F6D56FF49D
:10AE40008061202261612B6385F83D2085F83E30CA
:10AE50002B6C43F004032B64002385F83C30012065
:10AE6000F8BD0020F8BDFEF7EBF9C01BB0422C681E
:10AE700001D8002EDCD1636913F08003D8D12022E1
:10AE80002B6385F83D2085F83E302B6C13432B64F3
:10AE9000E2E700BFF8B5046805460E46174601E034
:10AEA000731C1AD1636913F0040314D1606942055D
:10AEB000F6D56FF48061202261612B6385F83D2017
:10AEC00085F83E302B6C43F004032B64002385F897
:10AED0003C300120F8BD0020F8BDFEF7B1F9C01BE1
:10AEE000B0422C6801D8002EDCD1636913F0040352
:10AEF000D8D120222B6385F83D2085F83E302B6C7D
:10AF000013432B64E2E700BF2DE9F04F056883B0DF
:10AF10009B462B68DDF83080DDF834A043F4807365
:10AF200006460F4691462B606B69DB0705D4B8F1E6
:10AF3000FF3F0ED16C69E007FCD507F0FE073249F0
:10AF40002F61534642463046FFF7E4FE00B301242A
:10AF50001AE0FEF775F9A0EB0A008045356830D29B
:10AF60006B69D907E0D400222023326386F83D3094
:10AF700086F83E20336C86F83C2043F0200333648F
:10AF80002B68DA0524D40324204603B0BDE8F08FF3
:10AF900033680190596901919B690193524641467A
:10AFA0003046019BFFF73CFF044618BBBBF1010F85
:10AFB000336811D15FFA89F220461A6103B0BDE807
:10AFC000F08FB8F1000FAFD16B69D907ACD4CAE7E5
:10AFD0004FF400733364D6E74FEA192018615246E4
:10AFE00041463046FFF71CFF20B932685FFA89F30B
:10AFF0001361C9E7336C042BA9D13268136843F499
:10B0000000731360A3E700BF020001002DE9F04FB9
:10B0100005689B462B6843F4806385B02B602B68E2
:10B02000DDF83880DDF83CA043F4807306460F4617
:10B0300091462B606B69DA0705D4B8F1FF3F4AD11E
:10B040006C69E407FCD507F0FE032B6143495346C6
:10B0500042463046FFB2FFF75DFE002869D13368F3
:10B060000390596903919B690393524641463046C8
:10B07000039BFFF7D5FE002853D1BBF1010F3368C6
:10B0800059D15FFA89F21A61524641463046FFF7BC
:10B09000C7FE002845D102463068016841F480713E
:10B0A00001604346CDF800A04FF001113046FFF794
:10B0B000DDFD336800284DD147F001071F612749A6
:10B0C000534642463046FFF725FE003818BF0120A0
:10B0D00005B0BDE8F08FFEF7B3F8A0EB0A0080459D
:10B0E000356817D26B69D807A4D4002220233263B5
:10B0F00086F83D3086F83E20336C86F83C2043F0DD
:10B10000200333642B68D90502D54FF400733364F0
:10B110000320DDE7B8F1000F8CD16B69D80789D423
:10B12000E3E7336C042B04D13268136843F40073F3
:10B1300013600120CCE74FEA19221A6141465246BA
:10B140003046FFF76DFE0028EBD132685FFA89F3D5
:10B15000136199E71B68DB05DAD5D6E70200010029
:10B16000002800F0B88070B590F83D30044603F038
:10B17000FF02002B00F098802368242284F83D20F1
:10B180001A6822F001021A601A6842F400421A603A
:10B190001A6822F400421A6001F0EEFA4F4B65681B
:10B1A0009D424FD84E4B98427CD94E4B6A00A3FB30
:10B1B0000035431EB3FBF2F32268516821F03F01D2
:10B1C00041EA95415160116A4FEA954C0CF1010C2E
:10B1D00021F03F0141EA0C011162D16940F6FC7097
:10B1E000013321F44F41034221F0FF0161D10423D7
:10B1F0000B43D361D4E907301168034321F0C00148
:10B200000B4313609168D4E9030321F40341034322
:10B2100021F0FF010B439360D4E90530D16803436B
:10B2200021F0FF010B43D3601168002341F00101BD
:10B2300020201160236484F83D00236384F83E30AD
:10B24000184670BD284B98422CD92268254B274EB2
:10B25000A3FB003C431E506820F03F0040EA9C40A6
:10B2600050604FEA9C414FF4967000FB01F1A6FB41
:10B270000161106A890920F03F0001310143116228
:10B28000D169A06821F44F4121F0FF01A0B905EB7D
:10B290004505B3FBF5F30133C3F30B03CBB143F423
:10B2A0000043A5E7012070BD80F83C20FBF780FD3E
:10B2B00062E7C3F30B039BE705EB850505EB85050B
:10B2C000B3FBF5F30133C3F30B0313B143F4404372
:10B2D0008EE701238CE70120704700BFA0860100A4
:10B2E0007F841E0083DE1B43FF083D00D34D6210A8
:10B2F0002DE9F047044682B09946BDF82CA00C9E7B
:10B300000F469046FDF79CFF94F83D30202B03D06C
:10B31000022002B0BDE8F08705460090404919239D
:10B3200001222046FFF7A2FC0028F1D194F83C301E
:10B33000012BEDD00123206884F83C300368DA0744
:10B340005ED53946076827F4006707600A9860628F
:10B350002120CDE9006584F83D00402084F83E00BE
:10B3600000202064A4F82AA0608D20852D48E0628A
:10B370004B4642462046FFF7C7FD00284DD1238D9E
:10B38000002B2AD02A4631462046FFF749FD0028E7
:10B390003BD1676A2068B4F828C03A460CF1FF3107
:10B3A00012F8013B0361638D013B9BB263854369E6
:10B3B000626289B25B0721850DD571B17A7802612D
:10B3C000628DACF1020C013A1FFA8CF1023792B295
:10B3D0006762218562850029D4D12A4631462046FC
:10B3E000FFF758FD88B922681368202143F40073E1
:10B3F000136084F83D1084F83C0084F83E0088E730
:10B40000036843F0010303609BE7236C042B04D122
:10B410002268136843F400731360012079E700BFCA
:10B42000020010000000FFFF2DE9F047044686B03F
:10B430009946BDF83CA0109E0F469046FDF700FFD0
:10B4400094F83D30202B05D04FF00208404606B05E
:10B45000BDE8F08705460090934919230122204654
:10B46000FFF704FC0028EFD194F83C30012BEBD01F
:10B470000123206884F83C300368D90739D5394660
:10B48000076827F4006707600E9860622220CDE904
:10B49000006584F83D00402084F83E0000202064D0
:10B4A000A4F82AA0608D20858048E06242464B4681
:10B4B0002046FFF7ABFD8046A8B9238D2268EBB983
:10B4C00002905369029393690293029B136843F4B9
:10B4D000007313600023202284F83D2084F83C3060
:10B4E00084F83E30B2E74FF00108404606B0BDE8B0
:10B4F000F087036843F001030360C0E7012B00F00D
:10B50000C480022B00F08A800590516905919269F0
:10B510000592059A664F032B4ED8012B00F0A880A8
:10B52000022B009533464FF000023946204600F0CA
:10B530008480FFF79BFB02460028D4D1236819685A
:10B5400021F4806119601969636A1970616A638DF9
:10B5500001316162013B218D9BB263854B1E2385C6
:10B560003946009533462046FFF780FB0028BAD1C4
:10B570002368616A1A6842F400721A601B690B70D2
:10B58000638D626A2168013B9BB26385531C096924
:10B590006362238D013B23855170238D628D616A27
:10B5A000013B013A01319BB292B26162238562850F
:10B5B000002B8FD0032BB0D92A4631462046FFF707
:10B5C000F7FB00288FD12268636A12691A70628DB6
:10B5D0002168238D606A013A92B262854A69013B13
:10B5E0009BB200F1010C52072385C4F824C0DFD5BB
:10B5F000032B03D10B6823F480630B600B6943704A
:10B60000628D238D013A92B26285626A013B9BB2E0
:10B61000013223856262002BCCD15BE7116821F4F3
:10B6200080611160116841F40061116004905169FA
:10B63000049192690492049A6CE7FFF717FB0028C3
:10B640007FF451AF2368616A1A6842F400721A608D
:10B650001B690B70638D626A013B9BB26385238D0E
:10B66000013B23852368511C1B6961625370C7E746
:10B670002A4631462046FFF79BFB00287FF433AF74
:10B6800023681A69636A1A70BAE7116821F4806145
:10B6900011600390516903919169039103991168B5
:10B6A00041F40071116035E7020010000000FFFF57
:10B6B0000400010070B582B000B390F895340568BD
:10B6C000044603F0FF02002B5AD028460323B5F1AD
:10B6D000A04F84F8953404BF0023A37103F042FC0B
:10B6E000237C8DF80030251D95E80E00206803F0BE
:10B6F0006FFB014630B1022384F8953401252846BA
:10B7000002B070BD206803F035FC01460028F2D17C
:10B71000267906B3234622464FF0010C1175D185D8
:10B720000131B142C2E9070082F815C0107642F833
:10B73000240FF3D100210A4683F854120131B1429B
:10B74000C3E9972283F8552283F85822C3F864226C
:10B7500003F12403F0D1207C95E80E008DF8000061
:10B76000206803F08DFC05460028C4D101236074D5
:10B77000206884F8953404F01FF8284602B070BDA4
:10B7800080F8942414F01CF820689FE710B590F816
:10B790009434012B0446006817D0012384F89434B4
:10B7A000C3685B0602D5637B012B09D003F0D2FB93
:10B7B000206803F0F1FF002384F89434184610BD8C
:10B7C000836B43F480338363F0E7022010BD00BF36
:10B7D0002DE9F04F066889B00446304604F02AF897
:10B7E00010B109B0BDE8F08F0546206803F0F4FF02
:10B7F0000028F6D0D6F808382068C3F30D23C4F823
:10B80000D43406F50063039303F0E6FF10F0020F53
:10B8100020681EBF436903F00203436103F0DCFFAD
:10B8200010F0100F206814D0836923F01003836197
:10B83000376A07F4F013B3F5802F07F00F0800F014
:10B84000BB82B3F5402F00F06282836943F010039E
:10B85000836103F0C1FF10F4002F206840F0F681EF
:10B8600003F0BAFF470300F15181206803F0B4FFF1
:10B870000028C0F2C280206803F0AEFF02057ED42B
:10B88000206803F0A9FFC70400F1E180206803F0FD
:10B89000A3FF10F4005F206840F0C28003F09CFF1B
:10B8A000000700F12A81206803F096FF01061DD5EC
:10B8B000B36923F08003B3612379012B16D927469E
:10B8C000012504E00135AB4207F124070ED997F8B2
:10B8D0007B22012AF6D105EBC50104EB810120682A
:10B8E00001F5157103F06AFE2379EBE7206803F098
:10B8F00073FFC20241D52379012B20D906F51268C6
:10B900002746012506E00135AB4208F1200807F182
:10B91000240714D997F83C20D8F80010012AF2D156
:10B920000029F0DA242305F00F0103FB0141206810
:10B9300087F83B20143103F041FE2379E3E72068C8
:10B94000436903F48013436103F046FF830221D46B
:10B95000206803F041FF400000F1C680206803F03A
:10B960003BFF41077FF53DAF23685D686A0700F143
:10B9700044825A682A435A6033E72068E4E7039B0D
:10B980009B68DB0700F135822068436903F400639C
:10B99000436176E794F804C0BCF1010F27D906F59E
:10B9A00032622346012103E0614503F124031ED0E6
:10B9B00093F87C021568012801F1010102F12002CF
:10B9C000F2D1002DF0DAD4F8D47487EA1547FF07D6
:10B9D000EAD483F87B02B06940F08000B0617069FE
:10B9E0000506E1D4039A536843F40073536020685A
:10B9F000436903F400134361ABE7039A536823F0F0
:10BA00000103536094F8CC34012B00F07981204677
:10BA100013F062FF2068436903F0004343612BE7A2
:10BA200003F00CFF206803F005FCE071256800F0CE
:10BA30009DFEE2790146284603F012FA204613F0F3
:10BA40001DFF2068436903F40053436126E7039A0E
:10BA50002068536823F001035360102103F0C2FAF9
:10BA60002079D8B106F510634FF67F3199601A68D6
:10BA700022F400121A60C3F80812D3F8002222F44C
:10BA80000012C3F80022D3F80022013542F0006210
:10BA90008542C3F8002203F12003E7D1039AD3695A
:10BAA00043F00113D361E37B002B40F01D81039A27
:10BAB000536943F4005343F02B035361136943F07C
:10BAC0000B031361D6F80038206823F4FE63C6F830
:10BAD0000038A17904F29C4203F0C0FE206843695B
:10BAE00003F480534361D2E6204613F001FF20683F
:10BAF000436903F08043436131E7204613F0BAFE07
:10BB00002068436903F008034361CDE6206803F031
:10BB10006FFE81462068B9F1000F3FF4A7AECDE972
:10BB2000046506F51067A0464FF0000A064609E0D6
:10BB30005FEA59090AF1010A08F1240807F1200710
:10BB400000F0F88019F0010FF2D05FFA8AFB594635
:10BB5000304603F05FFEC107054612D50398012168
:10BB6000436B0AF00F0201FA02F223EA0203436375
:10BB7000B960A179012900F045815946204613F0AA
:10BB80006FFE2A0744BF0823BB60EB0644BF1023A7
:10BB9000BB606E0644BF4023BB60A80700F1018173
:10BBA00029062668C4D5D8E90953AB42C0D806F5A2
:10BBB0001061D8F81C00079601EB4A11A5EB030CA5
:10BBC00084458A6928BF84461FFA82FE0CF1030C63
:10BBD000BEEB9C0FC0F04D81CDF818A08A4621E045
:10BBE000D8F81C30D8F820109D4228BF1D46A379F4
:10BBF00000935A46ABB2304603F02AFDD8F8203005
:10BC0000DAF818202B44C8F82030D8F8283092B23F
:10BC10002B440335B2EB950FC8F82830C0F02481CF
:10BC2000D8F824509D42A5EB0305D9D8DDF818A01B
:10BC30002668079B0AF00F0503F500610122D3F87F
:10BC40003438AA4023EA02034B6371E703F0C8FDCE
:10BC500007462068002F3FF403AE049506F53068D0
:10BC6000A3464FF0000A254607E07F080AF1010AC3
:10BC700008F120080BF1240B60D0FC07F5D55FFA22
:10BC80008AF4214603F0BCFD10F0010F814669D112
:10BC900019F0080F55D119F0100F1CBF1022C8F869
:10BCA000082019F0020F0FD07269100604D5039B0B
:10BCB0005A6842F480625A609BF85722012A00F0C9
:10BCC000DC800223C8F8083019F0200F1CBF2023A5
:10BCD000C8F8083019F4005F18BF4FF40053286803
:10BCE00018BFC8F80830C0E7039AD2F8843043F090
:10BCF0000B03C2F88430536C43F00B035364E1E64A
:10BD0000002184F8CC14204600F07AFA82E608225A
:10BD100004F29C41304608EBC80803F0AFFC04EB8A
:10BD20008802C7F30A13D2F8681220680B44C2F8DD
:10BD300068328AE53046059D049E97E52C46049DB1
:10BD40008EE529680822C8F80820086C01F53062E1
:10BD50006B4902EB4A128842936866D8284613F072
:10BD60006FFD98E728680122C8F80820A979D0F863
:10BD700040E000F5306202EB4A120129936866D078
:10BD800060498E4500F08180BAF1000F04D1D5F8EA
:10BD90006422002A00F0A7802146284613F056FDB1
:10BDA00076E70498514603F01DF998F81730012BF7
:10BDB00072D00223BB60F3E647F6F0731F423FF4F4
:10BDC00044AD08EBC80804EB8808C7F30A12D8F89A
:10BDD00060123046174603F051FCD8F860322068F4
:10BDE0003B44C8F86032D8F868323B44C8F868323F
:10BDF0002BE5204613F058FDC6E5204613F07CFDE8
:10BE00002368B6E5D8E907231344C8F82030BAF10F
:10BE1000000F7FF4B2AE636A002B7FF4AEAE2068F1
:10BE200004F29C4203F01AFDA7E61B0444BF4FF442
:10BE300000419160284613F003FDA97901297FF4A0
:10BE40002AAF286805F29C4203F008FD23E7190792
:10BE50002AD52B498E457FF61BAF18047FF518AF06
:10BE60004FF40041916013E7DDF818A0D8F8245092
:10BE70002668AB42FFF45CAEDBE6002221468BF87D
:10BE80005722284613F02CFD1BE71804E8D4990626
:10BE900082D5202191607FE7002388F8173059462A
:10BEA000204613F021FD84E7990602D520219160F8
:10BEB000EEE613498E4501D91B04D1D41169DBF894
:10BEC0007422C1F31201521ACBF86822BAF1000FA2
:10BED0007FF462AFD5F8641259B1D5F860121144FD
:10BEE000C5F8601258E705F29C42514603F0B6FCD3
:10BEF00052E705F29C42012103F0B0FC4CE700BF81
:10BF00000A30544F0A31544F90F89424012A0DD02E
:10BF100010B504460122006884F89424617403F08B
:10BF20002BFC002384F89434184610BD022070477F
:10BF300010B501F00F0E0EEBCE0C090604464FEAC9
:10BF40008C0C27D40CF5157101440EEBCE0004EBDC
:10BF500080004FF0000C80F855C2C2F30A028A60DC
:10BF60004A7881F800E00B710AB1A1F81AE0022BBF
:10BF700004BF00234B7194F89434012B16D0012395
:10BF800084F89434206803F061F9002384F8943431
:10BF9000184610BD0CF1140101440EEBCE0004EB69
:10BFA00080004FF0010C80F815C0D6E7022010BDCC
:10BFB00001F00F0301F00F0210B503EBC3030446B9
:10BFC000090602EBC2004FEA830304EB800016D49B
:10BFD00003F51573E1184FF0000C80F855C20A7094
:10BFE00094F89434012B15D0012384F894342068FC
:10BFF00003F074F9002384F89434184610BD143308
:10C00000E1184FF0010C80F815C00A7094F89434D0
:10C01000012BE9D1022010BD10B501F00F0E0EEB7F
:10C02000CE0C00EB8C0C1446CCF8643200238CF858
:10C0300054E2CCF86022CCF868328CF85532827920
:10C04000242101FB0E01012A01F5157108BFCCF86E
:10C050007042006803F0A4F9002010BD01F00F0148
:10C0600001EBC10100EB8100D0F86802704700BF0E
:10C0700010B501F00F0E0EEBCE0C00EB8C0C14463D
:10C08000CCF824300023CCF8283001238CF814E0BD
:10C09000CCF820208CF815308279242101FB0E0188
:10C0A0009A4201F1140108BFCCF83040006803F057
:10C0B00077F9002010BD00BF38B5037901F00F05F6
:10C0C000AB4232D30B0604461CD401EBC10324223D
:10C0D00002FB010100EB830301F51571002283F8D7
:10C0E000552201238B700D7094F894249A421AD033
:10C0F000206884F8943403F0E5FAC5B1002084F890
:10C10000940438BD05EBC503242101FB050100EBB8
:10C110008303012214315A7501238B700D7094F83A
:10C1200094249A42E4D1022038BD012038BDA1797F
:10C13000206804F29C4203F091FBDFE738B50379F5
:10C1400001F00F0293422ED3044602EBC20302EB2E
:10C15000C20009064FEA830304EB800016D403F5FE
:10C160001573E118002580F8555200258D700A706E
:10C1700094F89434012B14D00123206884F894346B
:10C1800003F0CEFA84F89454284638BD1433E118ED
:10C190000125457500258D700A7094F89434012BA3
:10C1A000EAD1022038BD012038BD00BF10B40468B8
:10C1B0001204636A29B91A43A26200205DF8044B95
:10C1C0007047A06A013903EB104C0AD0002303F139
:10C1D000400004EB80000133406899420CEB104CA6
:10C1E000F5D1403104EB810442EA0C026260002088
:10C1F0005DF8044B704700BF036800205962704728
:10C20000704700BF002800F0D8812DE9F041036895
:10C21000DD0782B004462FD59D498A6802F00C02E2
:10C22000042A00F0EC808A6802F00C02082A00F070
:10C23000E2806368B3F5803F00F0EB80B3F5A02F98
:10C2400000F07381924D2A6822F480322A602A68B5
:10C2500022F480222A60002B40F0E080FCF7F0FFFF
:10C26000064605E0FCF7ECFF801B642800F2008125
:10C270002B689F03F6D423689D0728D5844A9168CC
:10C2800011F00C0F00F09B80916801F00C0108295F
:10C2900000F09180E368002B00F00C817D4B7C4E18
:10C2A00001221A60FCF7CCFF054605E0FCF7C8FF49
:10C2B000401B022800F2DC8033689F07F6D5336804
:10C2C000226923F0F80343EAC203336023681A07A4
:10C2D0005CD45D073AD56E4A136C13F0805340F07E
:10C2E00088800193136C43F080531364136C03F044
:10C2F00080530193019B0125674E3368D80540F1B7
:10C30000A780A368012B00F0B780052B00F01D81EA
:10C310005F4E326F22F001023267326F22F0040268
:10C320003267002B40F0AD80FCF78AFF41F288387D
:10C33000074605E0FCF784FFC01B404500F29880EB
:10C34000336F9B07F6D4002D40F0F980A369CBB181
:10C350004F4DAA6802F00C02082A00F0BC80022BA4
:10C360004C4B4FF000021A6600F0F980FCF768FFB2
:10C37000044604E0FCF764FF001B022878D82B6811
:10C380009B01F7D4002002B0BDE8F0816369FBB1E6
:10C39000404B3F4E0122C3F8802EFCF751FF05466B
:10C3A00004E0FCF74DFF401B022861D8736F9B0728
:10C3B000F7D523688DE7526851023FF56BAF344AD9
:10C3C0001268920738D5E268012A35D00120DAE7F1
:10C3D000304A2F4EC2F8803EFCF732FF054604E09B
:10C3E000FCF72EFF401B022842D8736F9F07F7D43B
:10C3F000DFE7002580E74A6851027FF51AAF244A3B
:10C40000126892037FF538AF6268002A7FF434AF78
:10C41000DCE71F4A136843F480331360FCF710FF16
:10C420001B4E054604E0FCF70BFF401B64281FD899
:10C4300033689B03F7D51EE7154920690A6822F087
:10C44000F80242EAC0020A601A077FF542AF9DE790
:10C45000336843F480733360FCF7F2FE07463368B9
:10C46000D9053FF54EAFFCF7EBFEC01B0228F6D90D
:10C47000032002B0BDE8F081054A136F43F00103C9
:10C480001367FCF7DDFE024F064641F288380AE0EA
:10C49000003802400000474200700040FCF7D0FE28
:10C4A000801B4045E4D83B6F9A07F7D5002D3FF439
:10C4B0004DAF44E0424A434E1360FCF7C1FE0546CF
:10C4C00004E0FCF7BDFE401B0228D1D83368990771
:10C4D000F7D42368FBE6012B3FF478AF6B68E26981
:10C4E00003F4800191427FF471AF226A03F03F01AF
:10C4F00091427FF46BAF616A47F6C0721A40B2EBAB
:10C50000811F7FF463AFA26A520803F44031013AFD
:10C51000B1EB024F7FF45AAFE26A03F07063B3EB02
:10C52000026F14BF012000202DE7264B1A6842F449
:10C5300080221A601A6842F480321A606EE7214A3B
:10C54000136C23F08053136400E71E4B1A6F42F004
:10C5500004021A671A6F42F001021A6791E7FCF7AA
:10C560006FFE064605E0FCF76BFE801B02283FF6D7
:10C570007FAF2B689901F6D4D4E90731626A0B4387
:10C5800043EA8213D4E90A2052080D4943EA0063C2
:10C59000013A43EA024301226B600A66FCF750FE4F
:10C5A000084D044605E0FCF74BFE001B02283FF651
:10C5B0005FAF2B689A01F6D5E4E60120704700BF13
:10C5C0000000474200380240164908B58B6803F066
:10C5D0000C03042B1BD0082B01D0134808BD4A685C
:10C5E0004B68496813F4800302F03F0211D10E48F2
:10C5F000C1F38811A1FB0001F4F726FC094B5B682D
:10C60000C3F3014301335B00B0FBF3F008BD0748FF
:10C6100008BD0648C1F388110023A1FB0001F4F70F
:10C6200013FCEBE7003802400024F40000127A000B
:10C63000002800F08780484A136803F007038B4204
:10C640002DE9F0410D46044609D2CBB213701368B0
:10C6500003F007038B4202D00120BDE8F08123687C
:10C66000980714D5590704D53C498A6842F4E0522A
:10C670008A601A0704D539498A6842F460428A60A0
:10C680003649A0688A6822F0F00202438A60DF0718
:10C6900021D56268012A57D0931E012B2F4B1B68AE
:10C6A0004DD99907D8D52D4EB36823F00303134312
:10C6B000B360FCF7C5FD41F28838074604E0FCF79B
:10C6C000BFFDC01B404544D8B368626803F00C034B
:10C6D000B3EB820FF3D1204A136803F00703AB4298
:10C6E00006D9EBB21370136803F00703AB42B3D162
:10C6F00023685A0706D51949E0688A6822F4E0528F
:10C7000002438A601B0707D5144A2169936823F402
:10C71000604343EAC1039360FFF756FF0F4A104C92
:10C7200092681049C2F303120346A25C0E48D3403C
:10C7300000680B60FBF7F4FD0020BDE8F081980174
:10C74000B1D489E701207047044B1B689E03AAD42B
:10C7500082E7032081E700BF003C0240003802402E
:10C76000706902086C0300207C030020014B1868EC
:10C77000704700BF6C030020044B05499B68054AC5
:10C780000868C3F38223D35CD84070470038024066
:10C790006C03002068690208044B05499B68054A40
:10C7A0000868C3F34233D35CD84070470038024076
:10C7B0006C030020686902080E4B0F2210B402605F
:10C7C0009A680D4C02F0030242609A6802F0F0028F
:10C7D00082609A6802F4E052C2609B68DB0803F44E
:10C7E000E053036123685DF8044B03F007030B601B
:10C7F000704700BF00380240003C0240F0B50368BB
:10C8000013F0050F83B0044604D198073BD40020F1
:10C8100003B0F0BD454B464E00229A66FCF710FD72
:10C82000054604E0FCF70CFD431B022B28D83368B7
:10C830001B01F7D4D4E901131B0743EA81133B4AD8
:10C84000C6F8843001239366FCF7FAFC384E05469F
:10C8500004E0FCF7F5FC431B022B11D833681F01E1
:10C86000F7D52368D1E7FCF7EBFC41F288370646A1
:10C870002B6F9B073CD4FCF7E3FC801BB842F7D935
:10C88000032003B0F0BD2A4B2A4D002201921A6CFE
:10C8900042F080521A641B6C03F080530193019B99
:10C8A0002B6843F480732B60FCF7CAFC064604E057
:10C8B000FCF7C6FC831B022BE2D82B68D905F7D501
:10C8C0001B4DE3682A6F12F4407203F4407112D0DA
:10C8D0008A4210D02B6F154A0121C2F8401E23F462
:10C8E00040730021C2F8401E2B672B6FDA07BAD4C1
:10C8F000E36803F44071B1F5407F0BD00C498A68BE
:10C9000022F4F8128A600A4A116FC3F30B030B4337
:10C9100013677CE70648826823F0704121F4407178
:10C9200022F4F8120A438260EDE700BF000047429C
:10C930000038024000700040036830B59C6A1869F6
:10C940001B68C0F30E00C1E90140C3F30544002099
:10C95000C3F3062E64F3070003F07F0C6EF30F2081
:10C96000C3F306456CF31740C3F3805363F31F60B2
:10C970000860DAB94FEA1E1303EB83030EF00F0EC3
:10C980000EEB430E24094FEA1C1304EB840405F05C
:10C990000F0503EB83030CF00F0C05EB44050CEBC8
:10C9A000430C0D7081F801E081F802C0002030BD19
:10C9B00003685B6810B50020C3F3423E6EF30700C6
:10C9C000C3F3042EC3F3074CC3F307246EF30F2005
:10C9D00003F03F0363F317406CF31F600860D2B9A4
:10C9E0001A0902EB820203F00F0303EB42034FEA42
:10C9F0001E1E8B704FEA1C130EEB8E0E04F00F04FC
:10CA000003EB83030CF00F0C04EB4E040CEB430C14
:10CA10004C7081F803C0002010BD00BF38B503681A
:10CA2000DA68520601D5002038BDDA6842F080028B
:10CA3000DA600446FCF704FC05462368DB685B0605
:10CA4000F1D4FCF7FDFB431BB3F57A7FF5D92368DE
:10CA500004226277DB68012038BD00BF38B5036867
:10CA6000DA6822F08002DA609A68920601D5002026
:10CA700038BD0A4ADA600446FCF7E2FB0546236843
:10CA8000DB689B06F3D4FCF7DBFB431BB3F57A7F33
:10CA9000F5D904236377012038BD00BF5F7F010013
:10CAA000002845D038B5437F044603F0FF024BB160
:10CAB000022223686277DA68D20607D501236377FA
:10CAC000002038BD0277FBF777FAF1E7CA2153223D
:10CAD000596220465A62FFF7A1FF236810B1FF2276
:10CAE0005A6238BD99686268256921F4E00121F035
:10CAF00040019960616998682A430A430243E168EA
:10CB00009A6019611A69A16842EA01421A612046D5
:10CB1000FFF7A4FF23680028E1D11A6CA06922F472
:10CB200080221A641A6CFF2102431A645962C5E715
:10CB300001207047037F012B78D070B50E4601218C
:10CB400002230177016843778B680546002A37D1B5
:10CB500013F0400C18BF96F803C033780CBF86F86A
:10CB600003C04FEA8C5C092B09D900200A3BDBB2D9
:10CB7000092B00F10100F9D843EA0013DBB21C04D1
:10CB80007378092B09D900200A3BDBB2092B00F18D
:10CB90000100F9D843EA0013DBB2B07809284FEA64
:10CBA000032308D90A38C0B2092802F10102F9D8D2
:10CBB00040EA0210C0B244EA0C041C4304430FE0F4
:10CBC0007478327813F040034FEA042414BFF378EA
:10CBD000F37044EA0244B27818BF9B0514431C4327
:10CBE000CA234B6253234B622846FFF717FF28B135
:10CBF0002A68FF21002351622B7770BD2B683069B2
:10CC0000F26804F07F3424F0FE441C60996821F43B
:10CC100080219960996802430A4328469A60FFF789
:10CC20001DFF0028E4D101236B77E1E70220704764
:10CC300038B5037F012B6FD00546022301202877EA
:10CC40006B7791F800E0CB78487891F802C04FEA12
:10CC50004E3EAAB14EEA034444EA0C0444EA0024DE
:10CC60002B68CA215322596228465A62FFF7D6FE22
:10CC7000002840D02A68FF21002351622B7738BD5D
:10CC8000C40646D520F010000A30C0B2092B487007
:10CC900098BF1C040DD900210A3BDBB2092B01F11E
:10CCA0000101F9D843EA0113DBB209284FEA034432
:10CCB00009D900230A38C0B2092803F10103F9D8C1
:10CCC00040EA0313D8B2BCF1090F4FEA00200CD997
:10CCD000ACF10A0C5FFA8CFCBCF1090F02F1010205
:10CCE000F6D84CEA02125FFA82FC44EA0E040443CE
:10CCF00044EA0C04B4E72B6824F07F4424F0C00419
:10CD00005C602846FFF7AAFE0028B3D101236B77A9
:10CD1000B0E7092BBFD8C8E7022038BDF8B5037FBC
:10CD2000012B50D016460122027703680222427777
:10CD3000CA225A6253225A629A68044650050D4626
:10CD40000DD5FCF77DFA074605E0FCF779FAC01B24
:10CD5000B0F57A7F2ED82368DA685107F5D49A683F
:10CD600022F480629A60DA68D2B262F49062DA6089
:10CD7000FCF766FA074605E0FCF762FAC31BB3F559
:10CD80007A7F17D82368DA685207F5D59A6822F0B7
:10CD900007029A609A6832439A605D619A6842F429
:10CDA00080629A600021FF20012258626277217719
:10CDB0000846F8BD2268FF210323516263770023F0
:10CDC00023770320F8BD0220F8BD00BF0B4A03689B
:10CDD0004FF4800110B55161DA685205044602D45F
:10CDE0000123637710BDDA68D2B262F49062DA6030
:10CDF000FBF750FB0123637710BD00BF003C0140EF
:10CE00000368503343F82120704700BF0368503354
:10CE100053F82100704700BF836B1A68D36B43F44B
:10CE20008073D363704700BFF0B589B005460F46E5
:10CE3000FCF706FA00220023064608212868CDE9FF
:10CE4000002301F02BFE044610B1204609B0F0BDCE
:10CE5000296D2868090401F081FE04460028F4D1F8
:10CE60004FF0FF320823CDE9022330220223CDE91F
:10CE7000042302A9002201232868CDE9062301F03A
:10CE800007FD286801F086FE044640B1DDE7436BEC
:10CE90009B0415D5FCF7D4F9831B013327D02868F0
:10CEA000436B13F02A0F0BD1436B9A02EFD501F0BD
:10CEB000D5FC08AB03EB8403013443F8200CE9E70D
:10CEC000436B190719D4436B9A0516D4436B9B0720
:10CED00010D4446B14F0200412D1DDE9003240F28A
:10CEE0003A5112BA1BBA8163C7E90023ADE74FF08C
:10CEF0000044AAE702248463A7E708248463A4E724
:10CF000020248463A1E700BF80B110B50446032349
:10CF1000006884F8343001F0AFFC2046FBF736F9A6
:10CF20000023A36384F83430184610BD01207047F5
:10CF30002DE9F043044687B000297FD090F83400F3
:10CF400001285FFA80F866D11E46E36D1746324429
:10CF500000259A42A56308D9A36B43F00073A3632D
:10CF60000125284607B0BDE8F0830A462168206CF9
:10CF7000DFF8ECC0032384F83430CD62CB6B43F48C
:10CF80004A7343F00203CB63056585600568314B46
:10CF9000C3632B68C0F84CC023F0C0034FEA462996
:10CFA0002B6080314FEA9903FCF7F6FC0546002818
:10CFB00036D1294B2068C3F88C85636CCDF804907A
:10CFC000012B4FF090024FF00203CDE902234FF006
:10CFD00000014FF00103CDE904134FF0FF33694620
:10CFE00018BF7F02009301F053FC012E2BD982233E
:10CFF00020682363394601F06BFD0028B1D0236817
:10D00000164A9A63A36B012103430022A36384F8A9
:10D0100034102263A4E70225284607B0BDE8F08358
:10D0200023680E49DA6B22F49572DA639963A36B75
:10D0300043F08043A36384F8348091E7836B43F02B
:10D04000006383638CE7812320682363394601F002
:10D0500031FDD2E795D1000800802542FF05400050
:10D0600065D700082DE9F041044686B000296DD04F
:10D070001D4690F83430012B30D1C36D0E4600218F
:10D080008163501998422ED820683D4F032384F8BD
:10D090003430C162C36B43F4067343F00203C363CD
:10D0A000E36B1965616CDF63012918BF5202354FCC
:10D0B000DF64012D11464ED9A023236301F022FD28
:10D0C00007462268C7B1304B9363A36B01213B43F2
:10D0D0000022A36384F83410226308E0022630465D
:10D0E00006B0BDE8F081A36B43F00073A363012693
:10D0F000304606B0BDE8F081E06B244B31464FF07E
:10D1000001080668C3F88C85336823F0C00343F038
:10D1100040034FF0400C6D02C0F808C0803233600D
:10D12000AB08FCF739FC0646D8B12268D36B23F470
:10D13000067323F00203D363134B9363A36B43F093
:10D140008043A36384F834802763D0E7836B43F084
:10D1500000638363CBE79023236301F0C7FC07469A
:10D16000AFE790230293206801954FF0FF336946A3
:10D17000CDE90377CDF81480009301F089FBAEE789
:10D1800019CE000865D70008FF0540000080254241
:10D19000704700BF10B5846B236B2068822B0FD0C3
:10D1A000C36A23F00803C36240F23A51012200230C
:10D1B000816384F834202046236302F0BDFB10BD58
:10D1C00001F0AEFC034608B92068E9E7A26B1343FF
:10D1D0002046A363FFF7DCFFF6E700BF426E10B402
:10D1E0000346940FC2F383600C704870C2F301646D
:10D1F000C2F307408C70C870C2F30720D2B2087126
:10D200004A719A6E140DCC80C2F303440C72C2F3BF
:10D21000C0344C72C2F380348C72C2F34034CC728E
:10D220000020C2F300340C734873586C00286FD18F
:10D23000D86E40F6FC7404EA820242EA9072C0F3AF
:10D24000C2640A610C75C0F34252C0F302644C75AB
:10D250008A75C0F38244C0F3C232CC750A760C6979
:10D260000A7E02F007020232013494405C6591F8B4
:10D2700008C001220CF00F0C02FA0CF29A65520A57
:10D2800004FB02F2DA65C0F380324FF400741C66CE
:10D290004A76C0F3C61200F07F008A76C8761B6F0C
:10D2A000DC0FC3F341720C774A77C3F38264C3F394
:10D2B00083528C770020CA77C3F34054C3F30042F3
:10D2C00081F8204081F82100C3F3C03481F8222086
:10D2D000C3F3803281F8234081F82420C3F3403423
:10D2E000C3F3003281F8254081F82620C3F381245E
:10D2F000C3F3012281F82740C3F3460381F82820B5
:10D30000012281F8293081F82A205DF8044B70470A
:10D3100001280FD1D86E120402F47C1242EA1042A6
:10D320000A610A69013292024FF40074C3E916429D
:10D330005A65A8E71A68064991639A6B012142F081
:10D3400080529A6383F8341008465DF8044B7047A6
:10D35000FF054000F0B5002299B07623CDE90A23FD
:10D360000024099409AB054693E807008DE80700FF
:10D37000CDE906440894824E286806AB0ECB01F036
:10D3800051FA01272868C6F8A04001F071FA02207E
:10D39000C6F8A070FBF75AFF2868059401F08EFAD2
:10D3A000044648B1012385F83430AB6B2343AB63AB
:10D3B0000124204619B0F0BD286801F0CDFC0028FA
:10D3C00040F0C880AF642868002101F0C7FB08BBAB
:10D3D000059B4FF6FE76B3421FD86A4F0DE02146FB
:10D3E000286801F051FA059B01330593059BB34270
:10D3F00004464FEAD07210D87AB90021286801F0AB
:10D40000ADFB394604460028CCD1286801F07AFAF1
:10D410000028E4D04FF08054C4E7059A4FF6FE731D
:10D420009A4200F2A980C4F38074012328686C64D6
:10D43000ADF8123001F024FA002800F095806B6CF2
:10D440002868032B1CD1042101F01EFA000DE864AA
:10D450000DA92846FFF7C2FE0446002840F0878049
:10D460002A6D28681204234601F06AFB0146002851
:10D4700053D0012385F83430AB6B0B43AB6397E794
:10D4800001F0D0FB01460028F3D1286801F0FCF937
:10D49000034604216B67286801F0F6F9034608216A
:10D4A000AB67286801F0F0F90346EB6728680C21A8
:10D4B00001F0EAF96B6CC5F88000032B2868C2D034
:10D4C0000DF1120101F00CFC01460028D1D16B6C6A
:10D4D0002868032BB7D0BDF812102965090401F0A4
:10D4E000ADFB01460028C4D1286801F0CDF9034600
:10D4F00004216B66286801F0C7F903460821AB6672
:10D50000286801F0C1F90346EB6628680C2101F098
:10D51000BBF903462B67286895E72A462B1D52F86E
:10D52000106B07CA8DE8070030460ECB01F07AF980
:10D5300028684FF4007101F0B1FA00283FF439AFC8
:10D540002B68114A9A63AB6B01220343AB6385F8E6
:10D5500034202DE72868AC6401F0B0F950B9AB6C09
:10D56000012B7FF435AF2EE74FF0806181E74FF05C
:10D5700080517EE7044615E74FF0807412E700BF44
:10D5800000802542000010C1FF054000C8B110B561
:10D5900090F83430044603F0FF0273B1032384F89B
:10D5A00034302046FFF7D6FE28B90123A06320635C
:10D5B00084F8343010BD012010BD0277FAF730FD39
:10D5C000ECE70120704700BFF0B4D0E911C7D0E903
:10D5D0001365D0E91542D0E91730C1E900C7C1E9A8
:10D5E0000265C1E90442C861F0BC00208B6170474C
:10D5F00070B5426C0323032A8AB0044680F83430A5
:10D600000E46036825D0B1F5805F22D0B1F5006FDA
:10D6100061D000293DD0826B42F000628263A56B2D
:10D62000F5B9D4E90512CDE90812D4E90112CDE922
:10D630000412E268079606920AAA12E907008DE82A
:10D64000070004AE184696E80E0001F0EBF82368D8
:10D650000CE0A26B42F08052A263A56B002DE0D0DB
:10D66000012235499963154684F834204FF400713E
:10D67000184601F013FA30B123682F4A9A63A36B5E
:10D6800003430125A3630123284684F834300AB0FC
:10D6900070BD002218460023CDE9042301F0F4F800
:10D6A000820139D404A92046FFF7BEFB014668B9C0
:10D6B000059BDB0335D5216D2068090401F04EFA86
:10D6C000014618B9206801F057FA0146A26B236899
:10D6D0000A43A263C1E79FED167B184600218DED3A
:10D6E000047B01F0D1F8800119D404A92046FFF78A
:10D6F0009BFB60B9059B590316D5216D2068090471
:10D7000001F02CFA18B92068022101F035FAA26B59
:10D7100023680243A263A0E74FF40061D6E73046D6
:10D72000F5E74FF08061D1E74FF08060EFE700BF91
:10D730000000000000000000FF054000016D10B572
:10D7400009040446006801F035FA014620B1A36BD4
:10D750000B430020A36310BD206801F095F8C0F3CF
:10D76000432010BD10B5846BFCF784FA02280AD060
:10D77000D4E90F235B6D526D012B05D0012A03D034
:10D780002046FFF705FD10BD2368104A9A63DA6B47
:10D7900022F49D72DA63A36B43F080432046A363B7
:10D7A000FFF7CCFF0538012808D90122002384F8AF
:10D7B000342020462363FFF7EBFCE4E7206801F008
:10D7C000AFF9A36B0343A363EFE700BFFF0540007E
:10D7D00010B5846B236840F23A529A632046FFF7F3
:10D7E000ADFF012205380023904284F834202363E2
:10D7F00008D9A36B204613B902F096F810BDFFF7C5
:10D80000C7FC10BD206801F08BF9A36B0343A36331
:10D81000EFE700BF2DE9F04104460068256B436B3C
:10D820001A0482B01DD52B0700F1C080436BDB05C5
:10D830006BD54FF480738363C36B23F4434323F0AE
:10D840003A03C363C36A23F00103C362290605D503
:10D85000AA0600F1EC80AB0700F0BB8002B0BDE887
:10D86000F081436BDF0523D54FF480738363C36B73
:10D8700023F4434323F03A03C363C36A2E0723F020
:10D880000103C362E2D515F0220F40F0B08040F2F0
:10D890003A5383630122002384F834202046236313
:10D8A000AC0700F09F8002F047F802B0BDE8F081BD
:10D8B000436B5F042AD52E0728D5666A002ECDD08B
:10D8C000276A07F1040807F1240500E0206818F82A
:10D8D000043C019318F8032C43EA0223019318F83F
:10D8E000022C43EA0243019318F8012C01A943EAF0
:10D8F000026308F10408019300F0B4FF4545E5D147
:10D900002037203EC4E90876A8E7436B426B40F21B
:10D910003A231A42A2D0436B990703D5A36B43F075
:10D920000203A363436B1A0703D5A36B43F00803F9
:10D93000A363436B9B0603D5A36B43F02003A36350
:10D94000436BDF0603D5A36B43F01003A363436B64
:10D950009E0503D5A36B43F00803A36340F23A731B
:10D960008363C36B23F44E7323F00203C36301F09C
:10D97000D7F8A36B290743EA0003A3633DD42A0623
:10D980007FF56CAF15F0300F47D115F003055BD074
:10D99000206C324B0365FCF785F800283FF45EAF3E
:10D9A000206C02B0BDE8F041FFF712BFD4E90A577E
:10D9B000002F3FF453AF05F1200600E0206800F08F
:10D9C0004DFF45F8040BB542F8D1203FC4E90A5792
:10D9D00044E72268D36A012123F00803D36220467A
:10D9E00084F8341001F0A4FF02B0BDE8F08101F02A
:10D9F00097F8034650B9206849E70122002384F8CC
:10DA0000342020462363FFF7C3FB27E7A26B1343B1
:10DA10002046A363FFF7BCFBEDE7E06B104B03650B
:10DA2000FCF740F800283FF419AFE06BB9E701F0CC
:10DA300077F8034600283FF40EAFA26B134320464D
:10DA4000A363FFF7A5FB06E70123A563204684F83F
:10DA50003430256301F068FF00E700BF65DA000895
:10DA6000D1D70008FFF7B4BE00285CD070B50446DB
:10DA7000406A002847D00023C4E9043394F85130A9
:10DA80000022A26203F0FF01002B42D094462168DD
:10DA9000A568A269266A022384F851300B6823F036
:10DAA00040030B60636805F4044503F482732B4361
:10DAB000E56805F400652B43256905F002052B4355
:10DAC000656905F001052B43E56906F0800E02F457
:10DAD000007605F0380533432B43120C00F010009C
:10DAE00043EA0E0302F0040243EA0C0302430B6014
:10DAF0004A60CB69002023F400630122CB6160659A
:10DB000084F8512070BD6368B3F5827FB6D0E061C0
:10DB1000B4E7204684F85010FAF788FBD4E90903EB
:10DB200003F4005CB3E70120704700BF704700BFFB
:10DB300030B502685168936813F0400F85B0044611
:10DB4000C3F3801516D113F0010F53D198076AD58E
:10DB500008067CD4980613D4DB0568D58D0666D5F7
:10DB6000636D002043F0080363650390936803939B
:10DB7000039B18E0980742D5080668D4980640D55C
:10DB8000880654D5002D56D1606D40F001006065C7
:10DB90000020029090680290106820F04000106011
:10DBA0000298DB05DCD4636D002B40D05368012064
:10DBB00023F0E0038D07536084F8510059D0536877
:10DBC000E06C23F00303536040B12C4B0365FBF77B
:10DBD00069FF18B1636D43F040036365A06C30B317
:10DBE000264B0365FBF75EFF08B3636D43F040030C
:10DBF00063651CE011F0400FA8D0036C29E09D067E
:10DC000017D4880613D594F85100032817D0606DF7
:10DC100040F00400606500200090D068009090689B
:10DC200000900098BDE7980696D58806ACD405B05C
:10DC300030BD8D06FBD594F8510003280DD100238B
:10DC40000193D368019393680193019BEFE7636CA1
:10DC5000204605B0BDE830401847606D40F0040034
:10DC6000606500200090D068009090680090009857
:10DC70008AE72046FFF75AFFD9E700BF81DC00089A
:10DC800008B5806B0023C387C386FFF74FFF08BD2D
:10DC900090F83D30012B2FD103681849022280F8FB
:10DCA0003D20DA688B4242F00102DA6019D0B3F10C
:10DCB000804F16D0124A934213D002F580629342ED
:10DCC0000FD002F5806293420BD002F57842934266
:10DCD00007D002F57052934203D0A2F594329342DA
:10DCE00004D19A6802F00702062A03D01A6842F0AB
:10DCF00001021A60002070470120704700000140B7
:10DD0000000400400368DA6822F00102DA601A6A4F
:10DD100041F211110A4208D1196A40F244421142FB
:10DD200003D11A6822F001021A60012380F83D3005
:10DD30000020704790F83C20012A6ED0034602680C
:10DD400030B40120022483F83C0083F83D409468FD
:10DD500024F47F4424F0770494600C68602C76D01F
:10DD600011D8402C5BD02ED8202C04D000F2888013
:10DD700034F010011FD1916821F07001214341F06E
:10DD80000701916016E0B4F5805F13D0B4F5005F31
:10DD900033D0702C0FD1D1E9015094682843CD685D
:10DDA00024F47F4140EA052008439060916841F0E7
:10DDB0007701916000200121002283F83D1083F853
:10DDC0003C2030BC7047502CF5D14868CC68116AB3
:10DDD00021F00A010843116A21F0010111629169E1
:10DDE00021F0F00141EA041191611062916821F083
:10DDF000700141F057019160DCE7D1E9015094686E
:10DE00002843CD6824F47F4140EA05200843906010
:10DE1000916841F480419160CCE7022070474868E6
:10DE2000CC68116A21F00A010843116A21F001014E
:10DE30001162916921F0F00141EA041191611062CF
:10DE4000916821F0700141F047019160B2E74868A4
:10DE5000CC68116A21F0A00141EA0011106A20F09B
:10DE600010001062906920F4704040EA0430906124
:10DE70001162916821F0700141F06701916099E7AA
:10DE8000302C3FF478AF96E7704700BF704700BF73
:10DE9000704700BF704700BF036870B5DE681D693A
:10DEA000A907044601D5B20751D4690701D5720705
:10DEB0003AD42B0701D5300724D4EA0601D5F3065E
:10DEC00010D4E80701D5F10757D42A0601D5330647
:10DED0005BD4680601D571065FD4AA0601D5B306E6
:10DEE00042D470BD23686FF010021A6108222277B5
:10DEF000DB6913F4407F204663D0FFF7C7FF0023A0
:10DF00002377DEE723686FF008021A610422227784
:10DF1000DB699907204651D1FFF7B6FF2046FFF78E
:10DF2000B7FF00232377C8E723686FF004021A6164
:10DF3000022222779B6913F4407F20463BD1FFF7F2
:10DF4000A3FF2046FFF7A4FF00232377B1E76FF07C
:10DF500002021A61012202779B699B0725D0FFF715
:10DF600095FF00232377A0E723686FF02002204667
:10DF70001A61BDE8704000F009B923686FF0010232
:10DF80001A612046F9F77CFC9FE723686FF0800256
:10DF90001A61204600F0FCF89BE723686FF040020E
:10DFA0001A612046FFF776FF97E7FFF76DFF2046DF
:10DFB000FFF76EFFD5E7FFF769FFC5E7FFF766FFDD
:10DFC000AFE7FFF761FF2046FFF762FF97E700BF6B
:10DFD00070B4344E4A6903688D680C68B04245D00D
:10DFE000B0F1804F34D0A6F57C46B04230D006F573
:10DFF0008066B0422CD006F58066B04228D006F587
:10E000007846B04232D0284EB04225D006F5806620
:10E01000B04221D006F58066B0421DD0A6F59836F4
:10E02000B04233D006F58066B04215D006F5806662
:10E03000B04211D023F08003C5621A4384620368A2
:10E04000012143F00403036070BC4161026070472A
:10E050004E6823F070033343C968C56223F44073EC
:10E060000B4323F080031A438462E8E74E6823F0F1
:10E0700070033343CE68C56223F44073334323F007
:10E08000800384621A430B690363D8E7C96823F4E9
:10E0900040730B4323F080031A43044BDD629C6200
:10E0A000CDE700BF000001400040014000180040E3
:10E0B00050B310B590F83D30044603F0FF02F3B1C1
:10E0C0002146022384F83D3051F8040BFFF780FF0E
:10E0D000012384F8463084F83E3084F83F3084F8D9
:10E0E000403084F8413084F8423084F8433084F87A
:10E0F000443084F8453084F83D30002010BD80F86D
:10E100003C20FAF7C7FBDBE70120704790F83C2082
:10E11000012A37D003460268022030B483F83D005C
:10E1200050680D68946820F07000284350601648CD
:10E1300082421AD0B2F1804F17D0A0F57C408242C3
:10E1400013D000F5806082420FD000F580608242DB
:10E150000BD000F57840824207D000F57050824223
:10E1600003D0A0F59430824204D1496824F08004A1
:10E170000C4394600020012283F83D2083F83C008A
:10E1800030BC70470220704700000140704700BF5C
:10E19000704700BF026802F10C0353E8003F23F40C
:10E1A000907302F10C0C4CE800310029F3D102F11C
:10E1B000140353E8003F23F0010302F1140C4CE870
:10E1C00000310029F3D1036B012B05D0202200235D
:10E1D00080F842200363704702F10C0353E8003FCC
:10E1E00023F0100302F10C0C4CE800310029F3D1AC
:10E1F000ECE700BF0268116938B50446C068A3683F
:10E2000021F4405101432069116103436069D168E1
:10E210000343E06921F4164121F00C0103430B4351
:10E22000D3605369A069234923F4407303438A42AE
:10E23000536105D0204B9A4202D0FEF79DFA01E0CF
:10E24000FEF7AAFAE2691921B2F5004FD4E90053AA
:10E25000A0FB010113D09A009B0FF2F7F5FD174ABE
:10E26000A2FB00135B09642101FB130000013230A3
:10E27000A2FB00201B0103EB5013AB6038BDDA1882
:10E280004FF000035B41F2F7DFFD0C4AA2FB0031C7
:10E290004909642303FB1103DB003233A2FB032390
:10E2A000C3F342121B0902EB011203F4F873134487
:10E2B000AB6038BD00100140001401401F85EB51D8
:10E2C00070B310B590F84130044603F0FF0213B369
:10E2D0002268242384F84130D36823F40053204675
:10E2E000D360FFF787FF2368196921F49041196112
:10E2F000596921F02A015961D96800224FF0200C98
:10E3000041F40051D960626484F841C084F842C08D
:10E310001046626310BD80F84020FAF76DFDD7E724
:10E3200001207047002832D010B590F841300446E3
:10E3300003F0FF0233B32268242384F84130D3680A
:10E3400023F400532046D360FFF754FF2368196974
:10E3500021F490411961596921F0220159615969EB
:10E3600041F008015961D96800224FF0200C41F4B6
:10E370000051D960626484F841C084F842C01046FC
:10E38000626310BD80F84020FAF736FDD3E7012024
:10E39000704700BF90F84130202B15D101B10AB968
:10E3A0000120704710B40023046801622121C28457
:10E3B000436480F84110E168828441F08001E160AB
:10E3C00018465DF8044B70470220704790F84230C1
:10E3D000202B03D101B11AB90120704702207047E8
:10E3E00010B4046981620023222103638285C285FF
:10E3F0004364036880F842101CB1DA6842F480720A
:10E40000DA605A695DF8044B42F001025A61DA6839
:10E4100042F020020020DA60704700BF704700BF62
:10E42000704700BF08B5806B0023C385FFF7F8FF76
:10E4300008BD00BF704700BF90F84230222B57D173
:10E4400083680168826AB3F5805F44D0002B4BD1AA
:10E450000369002B48D14B68DBB21370826A01322A
:10E46000C38D8262013B9BB2C385002B40D100B5B6
:10E470000268D16821F0200183B0D160D16821F415
:10E480008071D16051694FF0200C21F00101516180
:10E4900080F842C04363016B01292AD1036302F172
:10E4A0000C0353E8003F23F0100302F10C0C4CE87E
:10E4B00000310029F3D11368DB0606D50023019350
:10E4C0001368019353680193019B818DFFF7B2FF9D
:10E4D00003B05DF804FB0369002BBCD14B68C3F3A8
:10E4E000080322F8023BBBE74B6803F07F03B4E765
:10E4F0007047FAF73FFD03B05DF804FB70B505689F
:10E500002B68EE68696913F00F0F82B004462A4643
:10E5100072D19D0602D5B10600F1C680216B01299A
:10E520000BD0180602D5310600F194805B0602D5A7
:10E53000750600F1AE8002B070BDD806F1D5F106C7
:10E54000EFD5002301931368019353680193019B56
:10E550005169A38D4D0640F10C81E06B016849685B
:10E5600089B2002900F04881994280F04581E18517
:10E57000C169B1F5807F36D002F10C0353E8003F4A
:10E5800023F4807302F10C0545E800310029F3D132
:10E5900002F1140353E8003F23F0010302F11405D4
:10E5A00045E800310029F3D102F1140353E8003F9C
:10E5B00023F0400302F1140545E800310029F3D1AE
:10E5C000202384F84230216302F10C0353E8003F1A
:10E5D00023F0100302F10C0545E800310029F3D1C6
:10E5E000FBF716FAA38D02226263E18D591A2046C9
:10E5F00089B2FFF71FFF9EE711F0010176D116F4F3
:10E60000907F8BD0DA070AD5F00540F1EC80626C80
:10E61000580742F0010262644FD500296AD1980779
:10E620005AD5190700F1A280626C002A83D09A069D
:10E6300002D5B30600F1DB806B69626C03F0400326
:10E6400002F0080253EA020620465CD1FFF7E8FE1A
:10E65000666470E794F84130212B7FF46CAFA168B9
:10E66000236AB1F5805F00F0D080591C21621B78CD
:10E670005360E38C013B9BB2E384002B7FF45BAFE0
:10E68000D36823F08003D360D36843F04003D360A2
:10E6900051E7D368202123F04003D360204684F85B
:10E6A0004110FFF7BBFE46E702B0BDE87040FFF740
:10E6B000C3BEF005ABD45A071CD498070CD500296B
:10E6C000AFD0626C42F0040262641A07ACD5626C8F
:10E6D00042F008026264A7E71807A5D506F02002F9
:10E6E0000A43F4D1636C002BA6D124E7DA07E0D407
:10E6F000580738D5626C990742F002026264E0D490
:10E700001A07E4D490E7FFF745FD6B695E0626D54E
:10E7100005F1140353E8003F23F0400305F1140111
:10E7200041E8003262B1226802F1140353E8003F6D
:10E7300023F0400302F1140040E800310029F3D136
:10E74000E06B60B1364B0365FBF7ACF900283FF492
:10E75000F2AEE06B036D02B0BDE870401847204692
:10E76000FFF75EFEE7E69907ABD4C9E7B206AED481
:10E77000B8E7E08DE18D89B280B200293FF4DBAECD
:10E780001B1A99B200293FF4D6AE02F10C0353E8EC
:10E79000003F23F4907302F10C0545E80030002897
:10E7A000F3D102F1140353E8003F23F0010302F117
:10E7B000140545E800300028F3D1202384F84230C6
:10E7C000206302F10C0353E8003F23F0100302F131
:10E7D0000C0545E800300028F3D10223636320468E
:10E7E000FFF728FEA7E65A073FF519AF65E7204671
:10E7F000FFF722FE25681FE799427FF49CAEC369AC
:10E80000B3F5807F7FF497AEE7E7216900297FF4B5
:10E810002CAF33F8021BC1F308015160236228E7D3
:10E8200025E4000884B010B40DF1080C8CE80E004B
:10E830000B46049913430B43DDE90541426823432A
:10E840000B4307995DF8044B22F4FD420B4322F081
:10E850007F021343436004B000207047D0F880006B
:10E86000704700BF0B68C0F880300020704700BFC1
:10E8700003230360002070470346002018607047A0
:10E88000006800F00300704714304058704700BF24
:10E8900010B4D1E900428B684462CC6882622343A1
:10E8A000D1E90441C26A234322F0F7020B43134328
:10E8B000C3625DF8044B0020704700BF00220F4B7D
:10E8C0008260C2680E491B686FF30B02A1FB031341
:10E8D00042F480625B0A41F28831C26001FB03F3BB
:10E8E00043B1426B120603F1FF33F9D5C5238363AD
:10E8F000002070474FF00040704700BF6C030020BD
:10E90000D34D621041F0004141F48011164B8160FB
:10E91000C26816491B686FF30B02A1FB031342F494
:10E920008D625B0A41F2883142F0010201FB03F380
:10E930008446C26043B1DCF8342012F0450F01D0A8
:10E94000120504D5013BF6D14FF000407047DCF8CA
:10E95000340010F0040015BF0420C523CCF83800A3
:10E96000CCF83830704700BF6C030020D34D6210E4
:10E97000474B10B41B68474CA4FB03435B0A03FBE3
:10E9800002F2531E4AB1426B12F0450F03F1FF33FE
:10E9900001D0120506D55C1CF5D14FF000405DF8A2
:10E9A000044B7047436B5B073CD4436BDC0707D4D5
:10E9B000C52383630369DBB2994204D00120EEE7EB
:10E9C00001238363FAE74369334818400028E6D0FF
:10E9D000002B2BDB5A002CD49C002CD4D9002CD437
:10E9E0001A012DD45C012ED4D9012FD41A0230D4AF
:10E9F0005C0231D499023BD4DA0236D45C0331D4C0
:10EA000099032CD4DA033FD41C043AD4590435D4E6
:10EA10009A0430D413F0080F0CBF4FF480304FF439
:10EA20000000BCE7042383631846B8E74FF000708A
:10EA3000B5E74020B3E78020B1E74FF48070AEE740
:10EA40004FF40070ABE74FF48060A8E74FF400602C
:10EA5000A5E74FF48050A2E74FF400509FE74FF432
:10EA600080209CE74FF4003099E74FF4004096E790
:10EA70004FF4804093E74FF4800090E74FF400108C
:10EA80008DE74FF480108AE74FF4002087E700BF3E
:10EA90006C030020D34D621008E0FFFD8160C16867
:10EAA0006FF30B0141F48A61C16041F28832102199
:10EAB000FFF75EBF8160C3686FF30B0343F48A63A3
:10EAC00043F0010341F28832C3601121FFF750BFC8
:10EAD0008160C3686FF30B0343F48A6343F002035E
:10EAE00041F28832C3601221FFF742BF8160C168E2
:10EAF0006FF30B0141F48B61C16041F28832182140
:10EB0000FFF736BF8160C3686FF30B0343F48B6379
:10EB100043F0010341F28832C3601921FFF728BF97
:10EB200000238360C368054A6FF30B0343F48963D2
:10EB300043F00403C3600C21FFF71ABF00E1F505A1
:10EB40008260C3686FF30B0343F4886343F00703E9
:10EB500041F28832C3600721FFF70ABF8160C368B2
:10EB60006FF30B0343F48E6343F0070341F28832E3
:10EB7000C3603721FFF7FCBE8160C3686FF30B03EE
:10EB800043F4886343F0060341F28832C3600621F0
:10EB9000FFF7EEBE00238360C3686FF30B0343F4FB
:10EBA0008E6343F0030341F28832C3603321FFF7E1
:10EBB000DFBE00BF8160C3686FF30B0343F489635A
:10EBC00043F0050341F28832C3600D21FFF7D0BE48
:10EBD000124B134A1B68A2FB032341F288315B0AE4
:10EBE00001FB03F301463BB14A6B12F0450F01D024
:10EBF000120504D5013BF7D14FF0004070474B6B35
:10EC00005B0707D4486B10F0010014BF0123C52334
:10EC10008B63704704208863704700BF6C0300203B
:10EC2000D34D621000238360C3686FF30B0343F47A
:10EC3000986343F00203C360FFF7CABF8160C368F3
:10EC40006FF30B0343F4996343F00103C360FFF7D1
:10EC5000BFBF00BF204B10B41B68204CA4FB034374
:10EC60005B0A41F2883404FB03F33BB1446B14F0BC
:10EC7000450F01D0240506D5013BF7D14FF00040E8
:10EC80005DF8044B7047436B5B071BD4436BDC0799
:10EC900005D40369DBB2994204D00120F0E70123D7
:10ECA0008363FAE7C5238363436913F4604010D09C
:10ECB0005A040BD413F4004F0CBF4FF480304FF4C0
:10ECC0008050DDE7042383631846D9E74FF40050F2
:10ECD000D6E71B0C1380D3E76C030020D34D6210E2
:10ECE00000238360C3686FF30B0343F4886343F02E
:10ECF00003030A46C3600321FFF7ACBF144B154A58
:10ED00001B68A2FB032341F288315B0A01FB03F37A
:10ED100001463BB14A6B12F0450F01D0100504D5F6
:10ED2000013BF7D14FF0004070474B6B5A070CD4B2
:10ED3000486B10F0010005D14B6B5B06F4D5402306
:10ED40008B63704701238B6370470420886370478F
:10ED50006C030020D34D62104FF4D5728260C268FC
:10ED60006FF30B0242F48962C260FFF7C7BF00BFB6
:10ED700082B00023019302E00369002B09DB019BB1
:10ED800001330193019BB3F1706FF5D9032002B0F9
:10ED900070470A230193019B2BB1019B013B019317
:10EDA000019B002BF9D1036943F00103036103E0E8
:10EDB000036913F0010307D0019B01330193019B09
:10EDC000B3F1706FF4D9E1E7184602B0704700BFA5
:10EDD00084B010B50DF10C0C8CE80E009DF81130CC
:10EDE000012B044624D1836B9DF8182023F4803333
:10EDF0008363C36823F4840323F04003C360C368C0
:10EE0000012A23F44013C36025D02046FFF7B0FF4A
:10EE10009DF80E30012B07D1A36843F00603A360D1
:10EE2000A36843F02003A360BDE8104004B070471E
:10EE3000C36843F04003C360FFF79AFF9DF81530A5
:10EE400023B9A36B43F48033A363E1E7A36B23F4FB
:10EE50008033A363DCE7C36843F48013C360D4E763
:10EE6000022A03460AD04FF41051DA6822F4705295
:10EE7000DA60DA680A430020DA607047264A2748D9
:10EE80000A44824232D9264A26480A44824230D96C
:10EE90002548A1F57402A2F5105282422CD92348CC
:10EEA000A1F18372A2F5E742824228D3204A214889
:10EEB0000A44824226D9204A20480A44824224D366
:10EEC0001F4A20480A448242CDD31F48A1F1B7729D
:10EED000A2F5585282421BD31C4A1D480A44824262
:10EEE0002CBF4FF4C0514FF4E051BEE74FF47051C6
:10EEF000BBE74FF46051B8E74FF45051B5E74FF41A
:10EF00004051B2E74FF43051AFE74FF42051ACE736
:10EF10004FF40051A9E700BF405327FFFF340C0016
:10EF2000401E1BFF3F420F007F4F120020D61300F0
:10EF300060B6E5FE5FE3160000D3CEFE40771B000F
:10EF4000C05BB3FEC091210020753800E05459FE2B
:10EF5000E09C4100034600209A6842F001029A605A
:10EF6000704700BF034600209A6822F001029A60B1
:10EF7000704700BF38B5C368012923F0C043054678
:10EF8000C36018D0A9B9C36843F080430C46C3607E
:10EF900001E0C82C0DD00A20FAF758F96B69DB079D
:10EFA00004F10A04F5D4A4F1C800B0FA80F04009D5
:10EFB00038BD012038BDC36843F000530024C3604E
:10EFC00001E0C82CF5D00A20FAF740F96B69DA079E
:10EFD00004F10A04F5D5A4F1C800B0FA80F04009A4
:10EFE000E6E700BF82B00023019302E00369002B33
:10EFF00009DB019B01330193019BB3F1706FF5D9DC
:10F00000032002B070478901002341F020010193E1
:10F01000016103E0036913F0200307D0019B013372
:10F020000193019BB3F1706FF4D9E9E7184602B080
:10F03000704700BF82B00023019302E00369002BF8
:10F0400009DB019B01330193019BB3F1706FF5D98B
:10F05000032002B07047002210230192036103E0F5
:10F06000036913F0100307D0019B01330193019B47
:10F07000B3F1706FF4D9EBE7184602B0704700BFE8
:10F0800084B0F8B507AC84E80E0000239DF81C504E
:10F090009DF826600446194603F1400204EB820203
:10F0A00001330F2B5160F7D104F50067002E40F0BB
:10F0B0009F807B6843F002037B60A36B43F40013E3
:10F0C000A363A36B23F40023A363A36B23F4802324
:10F0D000A3630023C4F8003E9DF82130012B00F00B
:10F0E0009780D4F8003843F00303C4F800381021A7
:10F0F0002046FFF777FF01462046FFF79BFF41EAD6
:10F10000000E5FFA8EFE0022BEF1000E3A6118BFBB
:10F110004FF0010E7A61FA6105B3D4F800190029A5
:10F1200004F5106315DB0021196000204FF67F31D4
:10F130000132AA421861996003F1200336D0D3F856
:10F1400000C0BCF1000FEEDA4FF0904CC3F800C0E5
:10F15000EEE74FF00061C4F80019E6E73B6923F4DD
:10F1600080733B6100229DF81E30A2616FF08042E7
:10F1700062611BB9A36943F01003A361A2692C4B20
:10F1800013439DF82220A3611AB1A36943F0080339
:10F19000A361012E05D1A36943F0804343F004032A
:10F1A000A3617046BDE8F84004B07047D4F8002B66
:10F1B000002A04F5306315DB0022002119604FF0AE
:10F1C000000C4FF67F300132AA42C3F810C098609D
:10F1D00003F12003C2D019680029EEDA4FF0904104
:10F1E0001960F0E74FF00062C4F8002B0022E6E758
:10F1F000A36B23F40013A363A36B43F40023A36363
:10F200000023C4F8003E9DF82130012B7FF469AF44
:10F210009DF81F3023B9D4F80038C4F8003866E7E9
:10F22000D4F8003843F00103C4F800385FE700BFAA
:10F2300000383C80D0F8083813F0060004D013F0F2
:10F24000020F14BF02200F20704700BF10B50A78CC
:10F25000012302F00F0E03FA0EF391F801E0BEF164
:10F26000010F00F5006C00EB42101AD0DCF81C20F6
:10F2700042EA0343CCF81C30D0F8003B1B040ED408
:10F280008B68D0F8004B0A79C3F30A03234343EA9F
:10F29000824343F0805343F40043C0F8003B002016
:10F2A00010BDDCF81C402343CCF81C30D0F80039EA
:10F2B0001C04F4D48B68D0F800490979C3F30A031D
:10F2C000234343EA814343EA825343F0805343F4A8
:10F2D0000043C0F80039002010BD00BF10B40A7808
:10F2E0004978012900EB42132CD0D3F8001B0029E8
:10F2F0001BDBD0F83C484FF4803102F00F0201FADA
:10F3000002F224EA0204C0F83C48D0F81C48224922
:10F3100024EA0202C0F81C28D3F8002B5DF8044B45
:10F3200011400020C3F8001B7047D3F8001B41F0C8
:10F330000061C3F8001BD3F8001B41F08041C3F803
:10F34000001BD6E7D3F8001900290BDAD3F800190F
:10F3500041F00061C3F80019D3F8001941F0804171
:10F36000C3F80019D0F83C1802F00F040122A240A3
:10F3700021EA0201C0F83C18D0F81C48074924EAE9
:10F380000202C0F81C28D3F800295DF8044B114094
:10F390000020C3F8001970470078F3EF007833ECD1
:10F3A0002DE9F0434C780E780D6991F804E0012CBA
:10F3B00000EB46135BD0D3F8104B6FF31204C3F885
:10F3C000104BD3F8104B6FF3DC44C3F8104B03F52C
:10F3D000306C8C6856BB05B10C610C62DCF81050C7
:10F3E000C4F312042C43CCF81040DCF81040012A7E
:10F3F00044F40024CCF8104033D0BEF1010F0CD1FE
:10F40000D0F8082812F4807FD3F8002B0CBF42F00C
:10F41000005242F08052C3F8002BD3F8002B42F088
:10F420000442C3F8002B0020BDE8F083002DD5D0A6
:10F43000614E2544013DB5FBF4F5ADB205FB04F486
:10F4400006EAC545DCF810600C623543CCF8105074
:10F45000DCF81050C4F312042C43012ACCF81040FD
:10F46000CBD1CA68002AC8D0CCF81420C5E703F570
:10F4700010648DB32769D1F808906FF312072761E4
:10F4800027696FF3DC472761002E4FD12769A94513
:10F4900047F400273CBFC1F810904D46276127690B
:10F4A000C5F312053D43012A256123D0D3F8004955
:10F4B000BEF1010F44F00444C3F800490C6958D070
:10F4C000002CB0D0D0F8342806F00F060123B3404A
:10F4D0001343C0F83438A6E725696FF3DC4525618E
:10F4E000256945F4002525612569012A6FF3120578
:10F4F0002561DBD1CA6902B16261BEF1010F0CD195
:10F50000D0F8082812F4807FD3F800290CBF42F00D
:10F51000005242F08052C3F80029D3F8002942F08B
:10F520000442C3F800290020BDE8F083224FD4F83C
:10F53000108009EB050C0CF1FF3CBCFBF9FC07EA61
:10F54000CC4747EA0807BEF1010F27611FFA8CFC80
:10F55000A5D14FEA4C7C0CF0C047D4F810C02CF079
:10F56000C04CC4F810C0D4F810C047EA0C0727619B
:10F5700095E7D0F8085815F4807FD3F800590CBFF0
:10F5800045F0005545F08055C3F80059002A7FF436
:10F590004AAFA3B203339B083FF445AFCA6800EB00
:10F5A000063606F5805602EB830352F8041B3160E1
:10F5B0009342FAD137E700BF0000F81F10B44A7831
:10F5C0000B7883B00021012A01914FEA431323D025
:10F5D00000F53060C218C158002904DB002003B0D8
:10F5E0005DF8044B7047C45844F00064C450C458DC
:10F5F00044F08044C45042F2107102E01368002BC2
:10F60000ECDA019B01330193019B8B42F6D9012077
:10F6100003B05DF8044B704700F51060C218C15884
:10F620000029DBDAC45844F00064C450C45844F0E4
:10F630008044C45042F2107102E01368002BCDDA0E
:10F64000019B01330193019B8B42F6D9DFE700BF99
:10F6500010B49DF8044064B903339B0809D001320B
:10F6600000EB023001EB830351F8042B02608B4264
:10F67000FAD100205DF8044B704700BF70B55FEA17
:10F68000920E054602F003061AD000F580548C460F
:10F690000023013322684CF8042B9E45F9D101EB7D
:10F6A0008E0066B105F5805506442968002321FACD
:10F6B00003F200F8012BB04203F10803F7D170BD4B
:10F6C0000846EEE74A780B78012A00EB43100CD08D
:10F6D000D0F8002B002A00DBD3B9D0F8003B43F46C
:10F6E0000013C0F8003B00207047D0F80029002A22
:10F6F00006DB2BB1D0F8003923F08043C0F8003985
:10F70000D0F8003943F40013C0F8003900207047E6
:10F71000D0F8003B23F08043C0F8003BDDE700BF9A
:10F720000B794A7891F800C0023B012A00EB4C109B
:10F73000DBB211D0D0F8002B012B22F40012C0F85C
:10F74000002B01D900207047D0F8003B43F08053D4
:10F75000C0F8003B00207047D0F80029012B22F4AC
:10F760000012C0F80029EDD8D0F8003943F08053DA
:10F77000C0F8003900207047D0F8003823F4FE6349
:10F78000C0F80038D0F80038090101F4FE611943CF
:10F79000C0F8001800207047D0F8002E034622F071
:10F7A0000302C3F8002ED3F8043800F5006123F0FB
:10F7B000020300204B607047D0F8002E034622F071
:10F7C0000302C3F8002ED3F8043800F5006143F0BB
:10F7D000020300204B607047426980691040704707
:10F7E000D0F8183800F50060C0691840000C704768
:10F7F000D0F8183800F50060C069184080B2704732
:10F8000000EB411100F50060D1F8082B4069104071
:10F81000704700BFD0F81028D0F8343800EB411002
:10F8200001F00F01CB40DB01D0F80809DBB2134334
:10F8300018407047406900F001007047D0F8002977
:10F8400003466FF30A02C3F80029D3F8043800F521
:10F85000006143F4807300204B60704730B4056C46
:10F86000114CA54200F5306303D9D0F8004B002CB1
:10F8700016DB00241C611C6944F400241C611C6913
:10F8800044F018041C611C69012944F0C0441C6147
:10F8900006D15A61D0F8003B43F08023C0F8003B0A
:10F8A000002030BC704700BF0A30544F08B50349F0
:10F8B000034803F0BBFE034B187008BD40A00020B6
:10F8C0009069020844A0002000207047844608B5D3
:10F8D000044813460A466146FDF72AFB003818BF64
:10F8E000012008BD409D0020844608B50448134609
:10F8F0000A466146FDF7B6FB003818BF012008BD77
:10F90000409D002008B50348FDF718FF043818BFD4
:10F91000012008BD409D002001460148FDF754BE6E
:10F92000409D0020704700BF08B5FFF7FBFF08BDF2
:10F9300008B500F02DF908BD08B500F031F908BD93
:10F9400000B583B001238DF8073000F021F808B925
:10F950008DF807009DF8070003B05DF804FB00BFB9
:10F9600008B5FFF7EDFF012801D0012008BD0748C9
:10F97000FDF70CFE0028F9D14FF400610348FDF7B4
:10F9800037FE003818BF012008BD00BF409D002091
:10F9900008B508210348FBF749F9B0FA80F040099F
:10F9A00008BD00BF000C024030B5164B187810F0AF
:10F9B000010489B006D11546032920D8DFE801F0FB
:10F9C000030F17060324204609B030BD6846FFF731
:10F9D000A3FF079B20465B0A2B6009B030BD684639
:10F9E000FFF79AFF069B2B60204609B030BD6846A2
:10F9F000FFF792FF079B2B80204609B030BD0424FF
:10FA0000E1E700BF800300202DE9F04184B00D46FE
:10FA100016461F4603F0CAFE47F22F58044602E07E
:10FA2000FFF770FF40B103F0C1FE001B4045F7D95E
:10FA3000012004B0BDE8F0813A4631462846FFF780
:10FA400053FF0028F4D10E4B47F23052196801A839
:10FA500004F00CF8019B102BEAD1029B022BE7D19A
:10FA600003F0A4FE47F22F55044603E0FFF74AFFD8
:10FA70000028DED003F09AFE031BAB42F6D9D7E78D
:10FA800048A0002070B5184C84B00125257003F003
:10FA900085FE10B9207804B070BDFFF761FFB8B1E2
:10FAA0002378012BF6D0114D2E68002EF2D1104B89
:10FAB0000FCBEC468CE80F003146604603F09AFF0E
:10FAC00028600028E6D1237843F001032370E1E7A2
:10FAD0002570FFF717FF18B9237803F0FE03237092
:10FAE0002378DBB22370DBE78003002048A00020EE
:10FAF0000C36020810B5064C01232370FFF702FFF5
:10FB000018B9237803F0FE032370207810BD00BFDE
:10FB1000800300202DE9F04184B00D4616461F46B3
:10FB200003F044FE47F22F58044602E0FFF7EAFED6
:10FB300040B103F03BFE001B4045F7D9012004B063
:10FB4000BDE8F0813A4631462846FFF7BFFE00285F
:10FB5000F4D10E4B47F23052196801A803F086FF2A
:10FB6000019B102BEAD1029B012BE7D103F01EFE73
:10FB700047F22F55044603E0FFF7C4FE0028DED00D
:10FB800003F014FE031BAB42F6D9D7E748A00020D0
:10FB9000024B00221868022103F03EBF48A000205B
:10FBA000024B00221868012103F036BF48A0002054
:10FBB000704700BF2DE9F047DFF8E0802C4F2D4E55
:10FBC0002D4D8CB000244FF47A7A4FF00409CDF813
:10FBD00008A0009701233C6034602C603022CDF8EF
:10FBE0000490A0214046FBF71FFCCDE9019A009646
:10FBF00001233422A0214046FBF716FC0095012387
:10FC00003822CDE9019A4046A021FBF70DFC2146A0
:10FC1000204607F0F7FE0094184A33681360184B2B
:10FC20002868184918603C68174D18480C60029005
:10FC300017480190284608F045FB284608F0E0FBED
:10FC4000144C284608F0E2FB2846134908F052FC01
:10FC50000FCC0DF1140CACE80F0094E807008CE811
:10FC60000700294605A803F0A9FD0CB0BDE8F08700
:10FC700054A0002050A000204CA000205CA0002038
:10FC800058A0002060A0002064A00020697901082D
:10FC900095FE00081C360208B1FB0008A09B00205E
:10FCA00000207047F8B590F82D305A0728D52E4D12
:10FCB0002E4E28680C464FF4FA6103F03DFE2C48A6
:10FCC000FAF73CFC30220021304610F06EFF14B3EE
:10FCD000D4E90023336063897360A2B106F10C0399
:10FCE0004FF0010C50685189126843F8043CC3E995
:10FCF00000010C3342B10CF1010CBCF1040FF1D145
:10FD00006FF00B00F8BD94460CEB4C0C06EB8C0C22
:10FD10000023CCF80830174F2389BE60144E7B6057
:10FD200020467C6308F06CFE39463046FAF742FB09
:10FD30000028E7D03046FAF79BFD83074FF4FA61BD
:10FD40000CD5286803F0F8FD3046FAF7F7FB394682
:10FD50003046FAF72FFB0028D4D0EBE7204608F016
:10FD6000D1FC6FF00B00CDE7D8A1002098A00020B7
:10FD700028A10020F0A00020F9F762BA844608B557
:10FD8000054813460A466146FAF77EFC003818BF5C
:10FD90000120404208BD00BF28A1002008B502484C
:10FDA000FAF738FD002008BD28A10020844608B5D8
:10FDB000054813460A466146FAF78EFC003818BF1C
:10FDC0000120404208BD00BF28A1002008B501461F
:10FDD000074808F0ABF9074B1A78012A00D008BD94
:10FDE000054900221A70BDE80840086803F0D0BD3C
:10FDF000DC69020820A30020DCA100202DE9F043EB
:10FE0000144CDFF85480DFF8549083B00646002786
:10FE100020684FF0FF3103F08FFD0028F8D198F8EB
:10FE200000300197002BF3D101A94846FAF7F4FA04
:10FE3000019D31462846002DEAD0336998470028B5
:10FE4000EDD0284608F05EFC98F800300197002BB2
:10FE5000DED1E9E7DCA1002020A3002028A10020BA
:10FE6000014B186803F094BDDCA10020014B186819
:10FE700003F08EBDD8A1002008B5FAF7FDFC0306FB
:10FE800000D408BD024B1868BDE8084003F080BDEF
:10FE9000DCA100202DE9F0410446AAB0002800F0C2
:10FEA000C980684B684A694E47F27341C4E905232B
:10FEB000E1856422002111A810F077FE04AB0093C5
:10FEC000634A73604FF400033260B3604FF47A7298
:10FED000604B02924FF00608F3605F4BCDF8048050
:10FEE0005E4933614FF4C0630025736140220123F2
:10FEF00004915B48ADF81450A021FBF795FA304609
:10FF0000FAF78EF8574B294634220746184610F068
:10FF10004CFE212240F8042C4FF44002026152486A
:10FF200008F08CF8736884F82C80197884F826100F
:10FF3000597884F82710997884F82810D97884F8AB
:10FF40002910197994F82D2084F82A105B7984F807
:10FF50002B3042F00A0240F2DC5384F82D20A384B7
:10FF6000012106A80695079503F0BAFC3F4E012132
:10FF7000306008A8CDE9085503F0B2FC03463068AC
:10FF80003B4E2946336003F0D7FC2946394D306893
:10FF900003F0D2FC0FCD0DF1280CACE80F0095E872
:10FFA00007008CE8070021460AA803F007FC324945
:10FFB0003248F9F785F83148F9F79AF858BB27BB6A
:10FFC0002E48F9F7C9F8012825DD033802282CD876
:10FFD0002B4A2C4B52F8206053F820501B4811A993
:10FFE000FAF7A0FB11A91948CDE91656FAF704FC57
:10FFF0001648FAF739F9204608F008FA204608F0C2
:020000040801F1
:100000003BFA00202AB0BDE8F081F7F77FFC002022
:100010002AB0BDE8F081204608F052FA204608F0E8
:100020000FFA00202AB0BDE8F0814FF480454FF46C
:100030000066D3E7144B1549154840F20D2210F025
:10004000AFFC2EE7A5FC00084DE1010828A1002027
:1000500000800240E0A1002080A200200080E1009A
:10006000A09B0020F4A00020DC690208DCA1002095
:10007000D8A100203836020884030020D0A0002038
:10008000D0690208C4690208D83E0208F43E02089A
:10009000043F0208F9F7D4B8F0B53B4B02688DB0C5
:1000A00000249A42CDE90644CDE908440A9401D0DF
:1000B0000DB0F0BDA3F5904300941A6B334842F0A5
:1000C00000721A631A6B02F000720092009A019497
:1000D0001A6B42F080621A631A6B02F0806201921E
:1000E000019A02941A6B42F000621A631A6B02F0D2
:1000F00000620292029A03941A6B42F004021A639D
:100100001A6B02F004020392039A04941A6B42F0F1
:1001100001021A631A6B02F001020492049A059418
:100120001A6B42F040021A631B6B03F04003322249
:10013000059303260B2506A90223CDE906230227F2
:10014000059BCDE90965FAF79BFB862306A91048B4
:100150000A95CDE90637CDE90846FAF791FB4FF449
:10016000D04306A90B480693CDE9084607970A95A0
:10017000FAF786FB224606213D20F9F7BFFA3D201B
:10018000F9F7F8FA0DB0F0BD008002400008024017
:1001900000000240001802402DE9F04F9BB00027FC
:1001A000044664220021684610F0FFFCDFF894B09A
:1001B000DFF894A0214D224EB946B84604E001284C
:1001C0000DDC642003F02AFB2846F8F7C5FF94F8FD
:1001D0002D305A07F3D5012822DD5B07F1D4023810
:1001E000032819D85BF820705AF8209069463046E9
:1001F000FAF798FA69463046CDE90579FAF7FCFA3C
:100200003046FAF731F8204608F036F9204608F073
:10021000FDF84FF00108D4E7B8F1000FD1D0E5E7C1
:100220003046FAF771F8204608F00AF9204608F03F
:1002300047F9E36920469847C3E700BFD0A00020F4
:1002400028A10020B4690208A469020810B5044678
:1002500082B00D4807F03AFF034678B100F1200262
:100260000A4922604FF4C06019610021CDE90020E5
:100270004122084608F094F902B010BD044A2060FB
:100280000121117002B010BDDC690208CDFD00082B
:1002900020A3002030B4002542F8205CA2F1200405
:1002A00022F8163C22F8185C026862B10A681460F1
:1002B0000C6002682AB11189194411811268002A60
:1002C000F9D130BC70470460F2E700BF08F01ABAF9
:1002D000D0F8D43200EB830010B5D0F8C04284B11E
:1002E000D0F8C4325BB194F80002FF2807D09B68B5
:1002F00094F8012221469847FF2384F80032002019
:1003000010BD032010BD00BF0A23038000487047C2
:100310001404002070B5822106460F4800F0BAFB95
:10032000012105460C4800F0B5FB812104460A482E
:1003300000F0B0FB0DB11022AA711CB100224021C7
:100340002171627118B10022402101714271432371
:100350000148338070BD00BF98030020FFF7DABF6B
:1003600070B5822106460F4800F094FB0121054636
:100370000C4800F08FFB812104460A4800F08AFBFC
:100380000DB11022AA711CB10021022221716271EB
:1003900018B10021022201714271432301483380C8
:1003A00070BD00BF9803002038B5D0F8D432B03308
:1003B00050F8235095B104460FF04AFBD4F8D432DC
:1003C000C5F80C0204EB8304D5F80402D4F8C43257
:1003D00005F50371DB689847002038BD032038BD60
:1003E00070B5D0F8D442D0F8C86200EB840EDEF8C5
:1003F000C05245B301F00F0404EB840C00EB8C0CED
:100400000A46DCF814306BB9DEF8C4321B690021EF
:10041000C5F8141223B1D5F8080205F50471984700
:10042000002070BD04EBC40406EB8406F469B3FB42
:10043000F4F604FB1633002BE6D1CCF814301A4640
:100440000FF0EEFAECE7032070BD00BF70B5D0F8F6
:10045000D43200EB830382B0D3F8C06200228DF85F
:100460000520ADF8062066B191F800C01CF06002CE
:1004700004460D461ED0202A06D02946204600F00C
:10048000C9FD032002B070BDCA8891F801E07AB3BB
:100490001CF0800F4CD0D3F8C43231469B687046B4
:1004A0009847EA88072A314628BF0722204600F0ED
:1004B000E9FD22E04B780B2BDFD801A252F823F0A4
:1004C00009050108FB0401087B0401087B040108FD
:1004D0007B0401087B0401087B0401087B040108FC
:1004E0007B0401087B0401081D050108FF040108C5
:1004F000D3F8C43270469B6898470020C2E790F852
:100500009C32032BF9D0B8E790F89C32032BB4D17E
:1005100002220DF1060100F0B5FDEEE790F89C32E5
:10052000032BAAD101220DF1050100F0ABFDE4E798
:10053000402A28BF402286F800E286F80122314690
:1005400000F0B6FDD9E700BF38B50446002581218B
:100550000FF022FA012184F8375020460FF01CFAE0
:10056000822184F8775120460FF016FAD4F8D4325D
:1005700084F84B5004EB83036564D3F8C0228AB13E
:10058000D3F8C4325B689847D4F8D432B03354F807
:1005900023000FF065FAD4F8D432B03344F8235076
:1005A000C4F8BC52002038BDF8B504464FF40770BB
:1005B0000FF052FA054600285BD04FF40772002175
:1005C00010F0F3FAD4F8D432B03344F82350237C3B
:1005D000C4F8BC52B3B340230222812120460FF05D
:1005E000CDF90121402384F83710022220460FF074
:1005F000C5F901271023032263648221082384F8AC
:10060000777120460FF0BAF9D4F8D43284F84B70E1
:1006100004EB83030026D3F8C432C5F804621B68D8
:100620009847D5F80422C5F81462C5F818622AB3B1
:10063000237CC3B94FF40073394620460FF0FCF910
:100640000020F8BD4FF400730222812120460FF0F4
:1006500095F901214FF4007384F8371002222046E7
:100660000FF08CF9C5E74023394620460FF0E4F936
:10067000E6E7D4F8D432B03344F823000220F8BDC2
:10068000034639B1D0F8D42203EB82030020C3F82B
:10069000C412704703207047D0F8D432B03350F8FA
:1006A00023302BB1C3F80812C3F810220020704782
:1006B00003207047D0F8D432B03350F823301BB148
:1006C000C3F804120020704703207047D0F8D432DA
:1006D000B03350F8232092B110B5D2F814420CB1C7
:1006E000012010BD0123C2F81432D2F81032D2F822
:1006F0000822836281210FF093F9204610BD032068
:10070000704700BFD0F8D422B03250F822208AB10E
:1007100008B5037CD2F804222BB1402301210FF04D
:100720008BF9002008BD4FF4007301210FF084F90C
:10073000002008BD0320704778B10023C0F8B8320C
:10074000C0F8C432C0F8D03209B1C0F8B4120123E5
:1007500080F89C3202700FF0D3B80320704700BFBE
:1007600010B582B00023ADF8063089B1CB6AC0F86D
:10077000B812044623B10DF106009847C4F8D00220
:10078000D4F8D83200200133C4F8D83202B010BDFA
:10079000032002B010BD00BF0FF0E4B8D0F8B832AB
:1007A0000BB11B6818471846704700BF08B5D0F852
:1007B000B8325B689847002818BF032008BD00BF07
:1007C00038B5044600F2AA25284600F017FC94F834
:1007D000AA12B4F8B022C4F898220123C4F89432C3
:1007E00001F01F03012B0ED0022B06D08BB9294636
:1007F0002046BDE8384000F063B929462046BDE8F0
:10080000384000F049BB29462046BDE8384000F09A
:1008100003BB204601F08001BDE838400FF0C8B8A6
:1008200010B5044629B9D0F89422032A10D000202C
:1008300010BD90F89C32032BF9D1D0F8B8329B69E7
:10084000002BF4D00022BDE81040C0F8D422184795
:10085000B0F860210B46D0F85811914208D890F8B2
:100860009C22032A12D0204600F03AFC002010BD42
:100870008B1AD0F86411C0F8583111449A42C0F86C
:10088000641138BF1A4600F023FCD0E7D0F8B82234
:100890001269002AE7D0C0F8D4329047E3E700BFDE
:1008A00070B5044659B9D0F89432022B16D094F89A
:1008B000A03213B1002384F8A032002070BD90F85C
:1008C0009C32032BF9D1D0F8B8325B69002BF4D0FD
:1008D0000022BDE87040C0F8D42218478269038C1A
:1008E0009A420D4610D81DD094F89C32032B26D086
:1008F000802120460FF05CF8204600F0FDFB94F8C4
:10090000A032002BD9D0D5E7416AD21A19448261AE
:10091000416200F0C5FB2B462A46294620460FF0CF
:100920008BF8C4E743699A42DED8D0F89822934204
:10093000DAD20A4600F0B4FBC4F89852EBE7D4F8D8
:10094000B832DB68002BD3D00022C4F8D422204672
:100950009847CDE7F8B5D0F8B8320021012280F8E9
:100960009C2204464160C0F89412C0F8A41280F89A
:10097000A0121BB15B680BB19847B8B900270022E1
:10098000402511460126402320460EF0F7FF84F84B
:100990006361A4F860512B460022802120460EF0AE
:1009A000EDFF84F8236025843846F8BD0327E6E789
:1009B00001740020704700BF90F89C32042B04D0D3
:1009C00090F89C32DBB280F89D32042380F89C3290
:1009D0000020704790F89C32042B04D190F89D328F
:1009E000DBB280F89C320020704700BF90F89C2258
:1009F000032A01D00020704708B5D0F8B83213B1EF
:100A0000DB6903B19847002008BD00BFD0F8D422AD
:100A1000AE3250F8222062B108B590F89C32032B18
:100A200001D0002008BD136A002BFAD0984700209F
:100A300008BD0320704700BFD0F8D422AE3250F872
:100A4000222062B108B590F89C32032B01D000201F
:100A500008BD536A002BFAD09847002008BD032038
:100A6000704700BF00207047D0F8B822012180F8FD
:100A70009C1242B108B552680179904708B900202C
:100A800008BD032008BD0020704700BF002070474C
:100A9000002070470278B0F802C09445134603D88E
:100AA0000CE09C450AD90278104413444278052A88
:100AB0009BB2F6D182788A42F3D17047002070470A
:100AC00070B50B7803F06003202B82B00D4604460E
:100AD00028D0402B26D05BB1802120460EF068FF45
:100AE000002120460EF064FF0025284602B070BDAC
:100AF0004B78092BF0D801A252F823F0750B0108AE
:100B00009D0B0108D90A0108BB0B0108D90A01088D
:100B1000D30B0108150C0108D90A0108490C01087A
:100B20003D0B0108D4F8D432AE33294654F82330B3
:100B30009B68204602B0BDE8704018478978B54DE3
:100B40000129297000F2418190F89C32022BDEB21B
:100B500000F02081032E00F0FB8080210EF028FFA2
:100B6000002120460EF024FF29782046FFF71EFEC4
:100B70000325BAE790F89C32013B022BACD8CA8817
:100B8000022AA9D1D0F8A4320146002B0CBF0123C0
:100B9000032341F80C3F00F075FAA5E790F89C326A
:100BA000013B022B98D84B88012B9DD10023C4F820
:100BB000A432204600F094FA96E74B88012BF6D039
:100BC000022B89D18B881B0A80F8A03200F088FAAA
:100BD0008AE78B88002B7FF47FAFCB88002B7FF4D4
:100BE0007BAF4B887F2B3FF677AF90F89C22032A90
:100BF0003FF472AFDDB280F89E5229460EF004FF3A
:100C0000204600F06DFA002D00F0FF80022384F8EA
:100C10009C3269E74A88130A0021013BADF80610AF
:100C2000062B3FF659AF01A151F823F0EF0C010854
:100C3000D50C0108C30C0108D90A0108D90A01081A
:100C4000AD0C0108710C0108CA88012A7FF444AF79
:100C500090F89C32022BD9B200F2B08000293FF408
:100C60003BAF0146002341F8083F00F00BFA3BE799
:100C7000037C002B7FF430AFD0F8B8320DF10600C2
:100C80001B6B984707234370EB88002B91D0BDF86E
:100C90000620002A3FF420AF9A4228BF1A46014698
:100CA0002046ADF8062000F0EDF91DE7037C002B8F
:100CB0007FF412AFD0F8B8320DF106005B6B9847A5
:100CC000E2E7D2B2052A3FF607AFDFE802F03B3594
:100CD0002F292318027CD0F8B832002A40F08780F0
:100CE0009B6A0DF10600984702234370CCE7D0F8C9
:100CF000B432007C1B680DF106019847C4E7D0F8B8
:100D0000B4329B69002B3FF4E7AE207C0DF1060165
:100D10009847B9E7D0F8B4325B69002BF5D1DBE630
:100D2000D0F8B4321B69002BEFD1D5E6D0F8B4323D
:100D3000DB68002BE9D1CFE6D0F8B4329B68002BFA
:100D4000E3D1C9E6D0F8B4325B68002BDDD1C3E64D
:100D5000002942D0416801293FF42BAFC9B2FFF707
:100D600025FD297861602046FFF718FD054600281B
:100D70003FF41FAF802120460EF01AFE00212046CE
:100D80000EF016FE21792046FFF710FD022384F8AD
:100D90009C32AAE600293FF40CAF01214160FFF725
:100DA000FDFC054650B3802120460EF001FE0021D7
:100DB00020460EF0FDFD84F89C6296E603297FF440
:100DC0008BAE011D00F05EF98EE680210EF0F0FD85
:100DD000002120460EF0ECFDCAE6022380F89C328A
:100DE0004160FFF7E3FC204600F07AF97CE6DB6A1D
:100DF0000DF1060098470223437045E7204600F0B6
:100E00006FF9032384F89C326EE6012384F89C3248
:100E10006AE600BFABEC002070B50B785A060D46B1
:100E200004460DD503F06002402A09D080210EF05F
:100E3000BFFD002120460EF0BBFD0026304670BDF0
:100E400094F89C32013B022B02D82979012908D958
:100E5000802120460EF0ACFD002120460EF0A8FDBA
:100E6000EBE72046FFF712FE90B9D4F8B8329B6842
:100E700073B1C4F8D402294620469847EB88064649
:100E8000002BDBD10028D9D1204600F029F9D5E785
:100E90000326304670BD00BF30B50C468A882378E3
:100EA00003F06003202B83B00546D1B24DD0402B18
:100EB0004BD053B1802128460EF07AFD0021284600
:100EC0000EF076FD002003B030BD6378012B2BD0EF
:100ED000032B4CD0002BEDD190F89C32022BD8B2D2
:100EE0005FD00328E6D101F00F0303EB8303120662
:100EF00005EB830365D493F86331002BDAD0142417
:100F000004FB015404F5AA74002968D028460EF0A9
:100F100067FD00286BD00123A373022204F10E01A8
:100F2000284600F0AFF8CDE790F89C32022BDAB2F9
:100F30002ED0032ABED16388002BC3D14B0651D1DA
:100F40002846019100F0CCF801992846FFF7A0FD52
:100F50000028B7D1D5F8B832C5F8D4029B68002B69
:100F6000B0D02146284603B0BDE83040184790F87D
:100F70009C32022BDAB20BD0032A9BD163881BB9B7
:100F8000480601D0E388A3B3284600F0A9F899E702
:100F90004A068FD00EF00CFD802128460EF008FD89
:100FA00090E7480686D111064CBF05F1140105F5FE
:100FB000AA71002301F80E3F0222284600F062F8D1
:100FC00080E793F82330002B3FF474AF01F07F04E7
:100FD000013404EB8404802905EB840496D10023BA
:100FE000A3739AE701910EF0EFFC0199A8E7A073B3
:100FF00093E728460EF0DCFCC6E700BF0B780370D1
:101000004B7843704B8843808B888380CB88C38028
:10101000704700BF10B5802104460EF0C9FC204681
:101020000021BDE810400EF0C3BC00BF30B370B566
:1010300003780E46144605460BB3034613F8011F0A
:101040000029FBD1681CEFF7CDF8431CDBB201335C
:101050005B00DAB223800323327073702C7864B1A2
:101060002846022300215A1CD2B2F454B15410F87D
:10107000014F0233DBB2002CF5D170BD7047022264
:101080001346E7E708B513460A460221C0E90533CF
:10109000C0F89412426200210EF0C2FC002008BD8C
:1010A00008B513460A4600210EF0BAFC002008BD20
:1010B00008B513460A460321C0E95533C0F8941217
:1010C000C0F8642100210EF0B7FC002008BD00BF6D
:1010D00008B513460A4600210EF0AEFC002008BDFC
:1010E00008B504210023C0F894121A4619460EF0E0
:1010F00097FC002008BD00BF08B505210023C0F8FB
:1011000094121A4619460EF097FC002008BD00BF45
:10111000034B03EB800203445268187A5368184764
:10112000D4EC002038B5084D2B5C5BB905EB800290
:101130002B1852680446187A1368984708B9012397
:101140002B5538BD002038BDD4EC002030B4054C00
:1011500004EB800504446D68207AAC68A44630BC7A
:10116000604700BFD4EC002030B4054C04EB800590
:1011700004446D68207AEC68A44630BC604700BF28
:10118000D4EC0020044B03EB000C03EB80039CF831
:1011900008005B681B691847D4EC0020264A1368D6
:1011A00070B4ABB10468A34209D01369ABB1A342D8
:1011B0003AD002290CBF0020122070BC704784680E
:1011C0005568A5420CD015693DB1AB42F1D110E094
:1011D000146914B10568A5420DD0002070BC704799
:1011E00045699668AE4225D01569002DF5D09D421F
:1011F000DFD1002501E0846801255369A34202D0B4
:10120000002DD6D0E9E7946943699C42F8D10123C7
:1012100069B902EB031270BC9089A0F58070B0FA36
:1012200080F040090001704784680025E5E7102040
:1012300070BC70470023EBE7ACEC00200246294B62
:10124000F0B418681568854224D01C69AC4206D0F9
:1012500000282FD0002C41D00020F0BC70475E69E0
:101260009768BE42F4D19E695769BE4208BF4FF0ED
:10127000010CEDD103EB0C124FEA0C149289A1B1D1
:10128000002AE9D10CF101004FF480722344F0BC34
:101290009A81704794685E68A642D6D154699E6868
:1012A000A642D2D14FF0000CE4E7013292B20CF129
:1012B0000100EBE7844601204FEA0C1400291D5180
:1012C0009568526903EB0C11C1E901524FF000021D
:1012D0008A8114BF4FF480720122D7E702204FF0B9
:1012E000010CE9E7ACEC0020016899B191F800C06D
:1012F000BCF11F0F13D90A46634603E012F8013F01
:101300001F2B0CD93A2BF9D1BCF1300F02D101318E
:101310008A4202D04FF0FF30704701320260002055
:10132000704700BFF8B5C3780BB90020F8BD456B16
:1013300000F138070446012340782A463946FFF772
:1013400013FFA8B9A26A236AE070AA1A9A42ECD2E3
:10135000A678012E01D8E8E7236A60781D442A4662
:1013600001233946013EFFF7FFFE012EF4D1DCE7F1
:101370000120F8BD2DE9F0410026D0F800808E75DF
:10138000C369002B5AD0036B013307460D461CD0AE
:10139000D8F80C30188898B101F1150601240AE03C
:1013A000412C0DD006F8010FD8F80C3033F814009A
:1013B000621C30B11446002102F05CF90028EFD124
:1013C00000242C440023A375AE7D3F6A00237C1EBD
:1013D00018464FF0E50C14F8011F202900F1010018
:1013E0001DD0052903F101022AD0092834D02B444D
:1013F00059726EBBA1F1410EBEF1190F27D8082812
:1014000097F80CE057D81EF0080F18BF20319975D7
:1014100014F8011F2029134600F10100E1D10B2827
:10142000D9D12B44B6B300225A72FB7A2B72FB69D6
:101430002B60D7F81630EB801B0CAB80BDE8F08139
:1014400009282DD02B4483F809C00EB9E5219975E0
:101450000B281346BFD1E4E72A4405EB030E4FF0F7
:101460002E0896B98EF816808EF80980A1F1410EEB
:10147000BEF1190F517205D897F80CE01EF0100F4D
:1014800018BF203191750233A5E78EF80980023329
:101490005172A0E79E753A7B002A08BF2B46C2E72F
:1014A0002A447EB1E9184FF02E0E81F809E0E521BB
:1014B000023351728FE71EF0100FC8D02031C9B22D
:1014C0009975C5E705EB030E71464FF02E088EF8AF
:1014D00016804EF22E5EA1F809E0E52102339175E7
:1014E00079E700BF38B5436B8B4201D1002038BD8E
:1014F00005460C46FFF716FF0028F8D1224668780B
:10150000012305F13801FFF721FE00281CBF4FF031
:10151000FF3401206C6338BDF8B50546FFF702FFC4
:1015200050B92B78032B08D0002268781146FFF7BA
:1015300029FE003818BF0120F8BD2E79012EF3D105
:1015400005F13807014604464FF4007238460FF0A3
:101550002CFB4AF65523A5F836320C4BAB6303F14E
:10156000FF536A6AA869C5F8200203F500532033C7
:10157000C5F81C3201326B69C5F8243268786A6399
:1015800033463946FFF7F0FD2C71CDE752526141E9
:1015900038B50D4640B1036804462BB11A781AB12C
:1015A0008188DA88914203D0092000232B6038BD5E
:1015B000186902F0DDF8034668B123685878FFF730
:1015C000A7FD10F001002368F0D0002BECD01869C3
:1015D00002F0D8F8E8E70F20E8E700BF70B54FF059
:1015E000FF360023B1420446C370466322D1B4F8EB
:1015F00036224AF655239A421AD194F83830E92B0C
:1016000007D0A36B134A03F0FF13934201D00220CB
:1016100070BDD4F86E30104A23F07F43934217D048
:10162000D4F88A000D4BC01A18BF0120400070BDCD
:10163000032070BD0D460A464078012304F13801AD
:10164000FFF784FD10B16663042070BD6563CEE7CB
:10165000002070BDEB0090004641540046415433D9
:10166000F0B5002385B00B600E461746FFF73CFE31
:10167000041EC0F2C580944B53F82450002D00F096
:10168000BC80286902F074F810B90F2005B0F0BDD5
:1016900035602B7807F0FE07002B40F08680E0B223
:1016A00000232B706870FFF73DFDC60700F1B28084
:1016B00017B1440700F19F8000212846FFF78EFFF5
:1016C00002287DD0042800F0A980012898BF0026B8
:1016D00000F28E80B5F84330B3F5007F40F088808B
:1016E000B5F84E10002900F0978095F8482029623F
:1016F000531E012BAA707BD895F845306B81002BC7
:1017000076D0581E184273D1B5F849702F8138072A
:101710006ED1B5F84B0000B9A86DB5F846C0BCF164
:10172000000F65D001FB02F20CEB17141444A04229
:101730005ED3001B9842B0FBF3FE59D30CEB0603BB
:101740004FF6F57CE64534440EF1020068D9AB62F1
:10175000B5F862302C633B43E8616E6248D1830088
:1017600003F2FF136A6EEA62B1EB532F40D3B5F870
:1017700068204FF0FF338021012AC5E90533297124
:101780007FD003205149524A28700B8810680133DA
:101790009BB285420B80EB8004BF0023136013696A
:1017A0009D420BD10023136108E06878FFF7B0FC7D
:1017B000C3073FF574AF0FB147071CD4002065E79E
:1017C0006C4605F5FB7305F2362021461A7902B105
:1017D0009A6841F8042B10338342F7D104F11007C3
:1017E00054F8046B032076B9BC42F9D1042815D013
:1017F0000D2005B0F0BD0A2048E70C2005B0F0BD73
:101800000B2005B0F0BD31462846FFF7E7FE012862
:10181000EAD85FE7032039E7E96D66E7012035E79D
:1018200040F6F57CE6456E622C63E861AB6216D843
:10183000002FDDD01A4400F0010303F2FF1300EB88
:10184000400003EB5003B1EB532FEA62D0D34FF0CB
:10185000FF338022C5E905332A71012092E7002F6A
:10186000C6D04000134400F2FF12B1EB522FEB62DE
:10187000BED34FF0FF338022C5E905332A71022021
:1018800080E7711C2846FFF72DFE00287FF479AF12
:10189000B5F8361228714AF6552291427FF471AF9D
:1018A000AA6B0C4B9A427FF46CAF03F1FF53D5F84F
:1018B0001C2203F5005320339A427FF462AFD5E92E
:1018C0008832C5E905235CE7D0EC0020CCEC002091
:1018D000ACEC0020525261412DE9F8430778022F09
:1018E00004460D46164642D0032F2ED0012F53D169
:1018F000836A01EB510803EB5829436B99454ED19C
:1019000000F1380708F1010915F00105C8F30808CE
:10191000F1B24FEA592274D017F8083003F00F03E0
:1019200043EA011307F808300123E370A36A02EBCE
:101930000308636B98456ED1C9F308094F44C6F399
:10194000071301223B70E27023E0826A436B02EBD3
:10195000D118984545D100F13807AD0005F4FE7562
:1019600001227B5966F31B037B51E27011E0826A0E
:10197000436B02EB1128984522D100F138076D0026
:1019800005F4FF757A197E550123C6F307265670B4
:10199000E3700020BDE8F8830220BDE8F883FFF77C
:1019A000C1FC0028F9D13B4604F1380760784A466B
:1019B0003946FFF7CBFB00284BD1C4F83490A1E7A0
:1019C000FFF7B0FC0028E8D104F138076078012364
:1019D00042463946FFF7BAFB00283AD1C4F83480B2
:1019E000CDE7FFF79FFC0028D7D104F138076078D6
:1019F000012342463946FFF7A9FB50BBC4F83480A7
:101A0000ABE707F808100123E370A36A02EB0308B1
:101A1000636B434513D02046FFF784FC0028BCD1FC
:101A20006078012342463946FFF790FB88B9C9F335
:101A30000809C4F834804F44002D80D102E0C9F376
:101A400008094F443B78C6F3032623F00F033343C2
:101A500077E74FF0FF33636301209EE701292BD91D
:101A6000C36999422DE9F0410C46054602D3012095
:101A7000BDE8F0810678022E2ED0032E1ED0012E56
:101A8000F5D1836A01EB5107416B03EB5728884579
:101A90002ED1C7F3080207F101082A4403EB5827A7
:101AA0008F4292F838605AD02846FFF73BFC002856
:101AB0004CD04FF0FF30DBE701207047866A436B64
:101AC00006EBD1169E4233D1A40004F4FE742544E3
:101AD000A86B20F07040CBE7866A436B06EB1126BB
:101AE0009E4217D1630003F4FF732B44188FBFE7A6
:101AF000FFF718FC0028DCD168783346424605F130
:101B00003801FFF723FB002836D1AB6AC5F83480D3
:101B10004146BEE7FFF706FC0028CAD168780123DA
:101B2000324605F13801FFF711FB28BB6E63D9E798
:101B3000FFF7F8FB0028BCD168780123324605F195
:101B40003801FFF703FBB8B96E63BDE7687801237E
:101B50003A4605F13801FFF7F9FA68B96F63C8F33F
:101B600008072F4497F8383046EA0320E3074CBFB4
:101B70000009C0F30B007BE74FF0FF336B6398E77E
:101B80000129F8B505680E4628D9EB698B4225D99D
:101B90000746114622BB284611E0FFF79DFEF0B92B
:101BA000D5E90632911E8B4205D22979013341F0E5
:101BB00001012971AB61A2421FD93868264631461E
:101BC000FFF74CFF0446002231462846ACB1012CF9
:101BD00004D0631C13D0EB699E42DED30220F8BD13
:101BE000012AFBD09342F9D94FF0FF322846FFF784
:101BF00073FE0028F3D13868E1E70020F8BD01202A
:101C0000F8BD00BF2DE9F041076806468846002967
